:1000000000000120C501000041020000F797010037
:100010004502000047020000490200000000000005
:10002000000000000000000000000000D5250100D5
:100030004D02000000000000F5250100CBAF0100DB
:100040007B7C0100837C01008B7C0100937C0100A0
:100050009B7C0100A37C0100AB7C0100B37C010010
:10006000BB7C0100C37C0100CB7C0100D37C010080
:10007000DB7C0100E37C0100EB7C0100F37C0100F0
:10008000FB7C0100037D01000B7D0100137D01005D
:100090001B7D0100237D01002B7D0100337D0100CC
:1000A0003B7D0100437D01004B7D0100537D01003C
:1000B0005B7D0100637D01006B7D0100F1EE0000BE
:1000C000737D0100FDC900007B7D0100837D01007F
:1000D0008B7D0100937D01009B7D0100A37D0100CC
:1000E000AB7D0100B37D0100BB7D0100C37D01003C
:1000F000CB7D0100D37D0100DB7D0100E37D0100AC
:100100002DB40000EB7D0100F37D0100FB7D0100BB
:10011000037E0100452200000B7E0100137E0100DA
:100120001B7E0100237E01002B7E0100F92C0000C4
:10013000337E01003B7E0100437E01004B7E0100C7
:10014000537E01005B7E0100637E01006B7E010037
:10015000737E01007B7E0100837E01008B7E0100A7
:10016000937E01009B7E0100A37E0100AB7E010017
:10017000B37E0100BB7E0100C37E0100CB7E010087
:10018000D37E0100DB7E010014010200000000208C
:1001900054020000140102000000FF1F00000000D4
:1001A0001401020000000014000000000004002000
:1001B000EC3100000000FF1F0000000000000014F0
:1001C0000000000010B572B613F0AEFF0D4B07E053
:1001D00003F10C049A685968186800F019F823466E
:1001E000094A9342F4D306E01C46596854F8080BB8
:1001F00000F01DF82346054A9342F5D362B617F086
:10020000F7FEFEE788010000AC010000C401000019
:10021000002393420AD210B450F8044B41F8044B27
:1002200004339342F8D35DF8044B704770470023C2
:1002300003E0002240F8042B04338B42F9D37047CB
:10024000FEE7FEE7FEE7FEE7FEE7FEE7FEE7FEE786
:10025000FEE7FEE7FFFFFFFFFFFFFFFFFFFFFFFFE0
:10026000FFFFFFFFFFFFFFFFFFFFFFFFFFFFFFFF9E
:10027000FFFFFFFFFFFFFFFFFFFFFFFFFFFFFFFF8E
:10028000FFFFFFFFFFFFFFFFFFFFFFFFFFFFFFFF7E
:10029000FFFFFFFFFFFFFFFFFFFFFFFFFFFFFFFF6E
:1002A000FFFFFFFFFFFFFFFFFFFFFFFFFFFFFFFF5E
:1002B000FFFFFFFFFFFFFFFFFFFFFFFFFFFFFFFF4E
:1002C000FFFFFFFFFFFFFFFFFFFFFFFFFFFFFFFF3E
:1002D000FFFFFFFFFFFFFFFFFFFFFFFFFFFFFFFF2E
:1002E000FFFFFFFFFFFFFFFFFFFFFFFFFFFFFFFF1E
:1002F000FFFFFFFFFFFFFFFFFFFFFFFFFFFFFFFF0E
:10030000FFFFFFFFFFFFFFFFFFFFFFFFFFFFFFFFFD
:10031000FFFFFFFFFFFFFFFFFFFFFFFFFFFFFFFFED
:10032000FFFFFFFFFFFFFFFFFFFFFFFFFFFFFFFFDD
:10033000FFFFFFFFFFFFFFFFFFFFFFFFFFFFFFFFCD
:10034000FFFFFFFFFFFFFFFFFFFFFFFFFFFFFFFFBD
:10035000FFFFFFFFFFFFFFFFFFFFFFFFFFFFFFFFAD
:10036000FFFFFFFFFFFFFFFFFFFFFFFFFFFFFFFF9D
:10037000FFFFFFFFFFFFFFFFFFFFFFFFFFFFFFFF8D
:10038000FFFFFFFFFFFFFFFFFFFFFFFFFFFFFFFF7D
:10039000FFFFFFFFFFFFFFFFFFFFFFFFFFFFFFFF6D
:1003A000FFFFFFFFFFFFFFFFFFFFFFFFFFFFFFFF5D
:1003B000FFFFFFFFFFFFFFFFFFFFFFFFFFFFFFFF4D
:1003C000FFFFFFFFFFFFFFFFFFFFFFFFFFFFFFFF3D
:1003D000FFFFFFFFFFFFFFFFFFFFFFFFFFFFFFFF2D
:1003E000FFFFFFFFFFFFFFFFFFFFFFFFFFFFFFFF1D
:1003F000FFFFFFFFFFFFFFFFFFFFFFFFFFFFFFFF0D
:10040000FFFFFFFFFFFFFFFFFFFFFFFFFEFFFFFFFD
:1004100001F0FF01102A2BDB10F0070F08D010F8B5
:10042000013B013A8B422DD010F0070F42B3F6D1B9
:10043000F0B441EA012141EA014122F007047FF0D2
:1004400000070023F0E80256083C85EA010586EA29
:10045000010685FA47F5A3FA87F586FA47F6A5FA65
:1004600087F68EB9EED1F0BC01F0FF0102F0070271
:1004700032B110F8013B013A83EA010313B1F8D11C
:100480000020704701387047002D06BF35460338FD
:10049000073815F0010F07D1013015F4807F02BF36
:1004A000013015F4C03F0130F0BC0138704700BF87
:1004B00080B483B000AF78607B68002B01D101234A
:1004C00003E07B68044A1A60002318460C37BD46D7
:1004D0005DF8047B704700BF0000FFFF80B586B069
:1004E00000AFF8607B600B46FB721346BB72FB7A71
:1004F0005A00BB7A13437B6107F11003184615F0CD
:1005000082FBFA687B691B01134403F128025379CB
:1005100043F040035371FB685B6823F4FF7323F0DF
:100520000103FA7A520102F4F0721A43BB7A1B01FA
:1005300003F010031A43F9687B691B010B4428334D
:100540005B79C3F30013DBB2DB00134304331A46B9
:100550007B6813603B6A1A04204B1340F9687A6980
:1005600012010A4428325279C2F3C002D2B2920177
:100570001A43FB685B6823F4FF7323F00103F97AE5
:10058000490101F4F0711943BB7A1B0103F0100318
:100590001943F8687B691B01034428335B79C3F373
:1005A0000013DBB2DB000B43194642F088030B60FB
:1005B0003B69184615F035FBFB689B6893F894304F
:1005C000DAB2FB689B6822F02002D2B283F8942052
:1005D000002318461837BD4680BD00BF0000FF034A
:1005E00080B586B000AF0346B9607A60FB732D4BCF
:1005F0003B61FB7B002B02D1FB7B002B01D0062350
:100600004BE0FB7BA42202FB03F3274A13447B61EC
:100610007B69FA7B83F8A220FB7B9B0018333B4469
:1006200053F8083C1A467B699A60FB7B9B011F4A82
:100630001A447B69DA617B699B68FF2283F880201A
:1006400000220121786900F035F8FB7B5B02184A33
:100650001A447B695A607B695B681A0A7B699B68EC
:10066000D2B283F89C207B695B681A0C7B699B681B
:10067000D2B283F8B0207B695B681A0E7B699B68F5
:10068000D2B283F8B420786915F013FB7B687A69DD
:100690001A607B69BA681A60002318461837BD468D
:1006A00080BD00BF0020074000060020A4060020F7
:1006B0000004002080B58AB000AFF8600B467A6075
:1006C000FB72FB683B62012387F82730FB68002B35
:1006D00001D103233EE1FB7A122B00F2288101A213
:1006E00052F823F03107000097070000DB070000F5
:1006F000F30700001308000033080000530800004F
:100700006B080000B30800002F0900002F0900004B
:100710002F0900002F0900002F090000D108000058
:10072000170900002F0900002F0900002F09000001
:100730003B6A9B68002283F800213B6A9B681B7F11
:10074000DBB203F00403002B09D03B6A9B681B7FDC
:10075000DAB23B6A9B6862F07F02D2B21A773B6AD8
:100760009B6893F80831DAB23B6A9B6842F010024A
:10077000D2B283F808213B6A9B6893F89430DAB2CE
:100780003B6A9B6842F00102D2B283F894200023B6
:1007900087F82730DCE03B6A9B681B7FDBB203F005
:1007A0000403002B09D03B6A9B681B7FDAB23B6ACB
:1007B0009B6802F07F02D2B21A773B6A9B6893F87B
:1007C0000831DAB23B6A9B6822F01002D2B283F899
:1007D0000821002387F82730BAE07B68002B00F05F
:1007E000A8807968386A15F010FB034687F827302F
:1007F0009FE07B68002B00F09E807B68FB61FB69BB
:100800001B781946386A15F096FB034687F827309F
:1008100091E07B68002B00F090807B68FB61FB69B6
:100820001B781946386A15F0B4FB034687F8273061
:1008300083E07B68002B00F082807B68FB61FB69B2
:100840001B781946386A15F000FC034687F82730F4
:1008500075E07B68002B74D07B687B617B6901222B
:100860001A80002387F827306BE07B68002B6AD062
:100870007B68BB61BB691B7803F00C03002B62D162
:10088000BB691B785B0003F01E03BA691278D209BA
:10089000D2B213433A6A1B01134428335B79C3F382
:1008A0008003DBB29AB2BB695A80002387F82730F5
:1008B00049E07B68002B48D07B68FB613B6A9B6802
:1008C000FA69127883F89820002387F827303CE0F3
:1008D000002387F8263013E097F8263063F07F0373
:1008E000DBB21946386A15F026FB97F82630194610
:1008F000386A15F020FB97F82630013387F8263048
:1009000097F82630032BE7D9386A15F0D2F900237F
:1009100087F827301CE07B68002B18D07B68FB61D0
:10092000FB6900221A70002387F827300FE000BF10
:100930000EE000BF0CE000BF0AE000BF08E000BF0F
:1009400006E000BF04E000BF02E000BF00E000BF1F
:1009500097F8273018462837BD4680BD90B5A7B018
:1009600002AFF860B9607A600023FB670023BB67C1
:10097000052387F88F30BB685B68B3F1FF3F02D077
:100980007B68002B02D197F88F309FE17B68C7F816
:100990008830D7F888309B68C7F8843007F1770330
:1009A0001A460621F86800F059FABB681B7A002B3A
:1009B00000F01781BB685B68082B03D1BB681B681C
:1009C000002B02D197F88F3080E1BB681B68C7F815
:1009D0008030D7F880305A88D7F884305A80D7F8DA
:1009E00080309A88D7F884309A80D7F88030DA88B7
:1009F000D7F88430DA80D7F880305A78D7F8843046
:100A00005A70D7F880301A78D7F884301A70D7F82F
:100A100084301B7803F06003002B23D1D7F8843097
:100A20005B780C2B00F2CB80D7F884305B781A46C9
:100A3000A84B53F82230002B00F0C180D7F8843047
:100A40005B781A46A34B53F8224007F1780307F16D
:100A50007C02D7F88410D7F88800A047034687F8AF
:100A60008F30ACE0D7F88430DB88002B64D0D7F827
:100A700084301B785BB2002B5EDBD7F88430DB88D8
:100A8000002B21D0D7F884301B7803F02003002BF3
:100A90001AD00023BB66012387F87030D7F8843062
:100AA0007B66D7F88430DB88FB6607F164031A465F
:100AB0000121F86801F09AF9034687F88F30FB6E40
:100AC000BB67BB6EFB6725E0D7F88430DB88002B63
:100AD00020D0D7F884301B7803F04003002B19D0C6
:100AE0000023BB65012387F86030D7F884307B652D
:100AF000D7F88430DB88FB6507F154031A461321CD
:100B0000F86817F041F8034687F88F30FB6DBB6734
:100B1000BB6DFB6797F88F30002B50D1FA6FD7F879
:100B20008430DB880021F86816F0B5FD034687F8AD
:100B30008F3097F88F30C9E0D7F884301B7803F0F6
:100B40002003002B1AD00023BB64012387F8503008
:100B5000D7F884307B64D7F88430DB88FB6407F1F6
:100B600044031A460121F86801F040F9034687F86A
:100B70008F30FB6CBB67BB6CFB6720E0D7F8843021
:100B80001B7803F04003002B19D00023BB63012323
:100B900087F84030D7F884307B63D7F88430DB881F
:100BA000FB6307F134031A461321F86816F0ECFFD3
:100BB000034687F88F30FB6BBB67BB6BFB6797F80F
:100BC0008F2007F17803019307F17C030093002342
:100BD000D7F88410F86816F058FA034687F88F3073
:100BE00072E097F87730032B13D1D7F884305B7815
:100BF0001A46384B53F8224007F1780307F17C027C
:100C0000D7F88410D7F88800A047034687F88F30BC
:100C10005AE0BB685B68002B56D0D7F88430DB887D
:100C2000002B51D0D7F884301B785BB2002B4BDB04
:100C3000D7F884301B7803F02003002B16D0BB6854
:100C40001B68BB62002387F83030D7F884307B62A2
:100C5000BB685B68FB6207F124031A460121F86850
:100C600001F0C4F8034687F88F301CE0D7F88430D1
:100C70001B7803F04003002B15D0BB681B68BB61D9
:100C8000002387F82030D7F884307B61BB685B682D
:100C9000FB6107F114031A461321F86816F074FF7C
:100CA000034687F88F3097F88F2007F17803019378
:100CB00007F17C0300930123D7F88410F86816F03D
:100CC000E4F9034687F88F3097F88F301846943749
:100CD000BD4690BD44C5010080B588B000AF7860C6
:100CE00039601B4BFB603B683B6101233B77002372
:100CF000FB7600237B778023BB7640233B8307F181
:100D00000C0207F118031946786816F0DAFC03465E
:100D1000FB77FB7F002B01D0FB7F15E00023BB7628
:100D200007F10C0207F118031946786816F0C9FCA0
:100D30000346FB77FB7F002B05D08021786816F0F7
:100D40001FFDFB7F00E0002318462037BD4680BD15
:100D50005D09000080B584B000AF03463960FB71C7
:100D600007F10803184614F04EFF0023FB601EE055
:100D70002B49FA681346DB009B1A1B010B441B68C6
:100D8000002B11D02649FA681346DB009B1A1B0181
:100D90000B446D331B78FA799A4205D1BB6818462B
:100DA00014F03FFF012336E0FB680133FB60FB6872
:100DB000002BDDD00023FB6025E01949FA681346BB
:100DC000DB009B1A1B010B441B68002B18D1144934
:100DD000FA681346DB009B1A1B010B446D33FA794A
:100DE0001A70FA681346DB009B1A1B010C4A1A445E
:100DF0003B681A60BB68184614F013FF00230AE032
:100E0000FB680133FB60FB68002BD6D0BB6818463B
:100E100014F007FF022318461037BD4680BD00BFFF
:100E2000E406002080B485B000AF03463960FB7152
:100E30000623FB73FB79012B05D83B68064A1A6031
:100E40000023FB7300E000BFFB7B18461437BD4650
:100E50005DF8047B704700BF78C5010080B586B09F
:100E600000AFF8600B467A60FB720123FB757B686C
:100E7000002B01D1042353E0FB7A023B062B4DD813
:100E800001A252F823F000BFA50E0000B50E00002D
:100E9000ED0E0000FD0E0000C50E0000D90E000092
:100EA0000D0F00007A680F21F86816F0E8F9034684
:100EB000FB7534E07A681021F86816F0E0F9034613
:100EC000FB752CE07B683B610023FB75FB6893F8A6
:100ED0006E203B691A7022E07B683B610023FB7542
:100EE000FB6893F86C203B691A7018E07A68062159
:100EF000F86816F0C4F90346FB7510E07A6807211C
:100F0000F86816F0BCF90346FB7508E07A68092119
:100F1000F86816F0B4F90346FB7500E000BFFB7DEE
:100F200018461837BD4680BD80B586B000AFF86062
:100F30000B467A60FB720123FB75FB7A033B0B2B9C
:100F400072D801A252F823F0790F00002910000096
:100F500029100000890F00009F0F000029100000D9
:100F6000291000000910000019100000E90F00000E
:100F700029100000F90F00007A681121F86816F0B6
:100F80007EF90346FB7554E07B68002B4ED00023AE
:100F9000FB757B681A78FB6883F86E2046E0FB6877
:100FA00093F86E30032B15D07B68002B40D00023C4
:100FB000FB757B681A78FB6883F86C20FB6803225A
:100FC00083F86E20FB686C331A461421F86816F01B
:100FD00056F92DE0FB686C331A460821F86816F0C4
:100FE0004EF90346FB7523E07A680A21F86816F08B
:100FF00046F90346FB751CE07A680B21F86816F089
:101000003EF90346FB7514E07A680C21F86816F087
:1010100036F90346FB750CE07A680D21F86816F086
:101020002EF90346FB7504E000BF02E000BF00E0BC
:1010300000BFFB7D18461837BD4680BD80B485B023
:1010400000AF78600023FB6017E01149FA6813468F
:101050001B0113449B000B441B68002B0AD1FA6848
:1010600013461B0113449B00094A1A447B681A600B
:10107000002306E0FB680133FB60FB68002BE4D033
:10108000022318461437BD465DF8047B704700BF45
:101090005407002080B596B000AF786000237B65D0
:1010A000012387F853307B68002B02D197F8533027
:1010B000BAE17B6893F84030002B08D07B6893F846
:1010C00040207B685B689B685B799A4202D997F8FD
:1010D0005330A9E17B685B689B681A687B6893F86A
:1010E000403003F10053013BDB0013447B630023DA
:1010F000FB644DE07B6B5968FA6C13465B0013444C
:101100009B000B441B78022B3FD10023BB6422E0E1
:101110007B6B5968FA6C13465B0013449B000B44CD
:101120005A68BB6C1B0113441A787B6893F84230F1
:101130009A420DD17B6B5968FA6C13465B001344DD
:101140009B000B445A68BB6C1B0113447B650FE08A
:10115000BB6C0133BB647B6B5968FA6C13465B0054
:1011600013449B000B441B7A1A46BB6C9342CFD3AB
:101170007B6B5968FA6C13465B0013449B000B446D
:10118000DA787B6883F8412008E0FB6C0133FB646C
:101190007B6B1B781A46FB6C9342ABD37B6D002BA9
:1011A00002D197F853303FE17B687A6D9A60002353
:1011B0007B6461E0002387F830307B6D99687A6C3E
:1011C00013465B0013445B000B441B7987F83130F6
:1011D0007B6D99687A6C13465B0013445B000B448B
:1011E0001B7887F82E307B6D99687A6C13465B000C
:1011F00013445B000B445B88BB857B6D99687A6CFC
:1012000013465B0013445B000B445B7887F82F3078
:1012100097F82E30DB09DBB2012B1CD197F82F3069
:10122000032B18D197F82E3003F00F03DAB27B6846
:1012300083F83D207B68002283F83E207B684FF0D6
:10124000FF325A637B68002283F83C207B680022CF
:101250009A63774B3B627B687B627B681B6807F114
:10126000200207F12C01184616F02BFA034687F8E6
:1012700053307B6C01337B647B6D1B791A467B6C2E
:10128000934297D300233B6442E07B6B59683A6CEE
:1012900013465B0013449B000B441B780A2B34D18C
:1012A0000023FB6323E07B6B59683A6C13465B00B9
:1012B00013449B000B445A68FB6B1B0113441A78C0
:1012C0007B6893F842309A420ED17B6B59683A6C36
:1012D00013465B0013449B000B445A68FB6B1B01D5
:1012E00013447B6500BF19E0FB6B0133FB637B6B31
:1012F00059683A6C13465B0013449B000B441B7AFD
:101300001A46FB6B9342CED308E03B6C01333B643F
:101310007B6B1B781A463B6C9342B6D37B687A6D25
:10132000DA600023BB6377E000233B777B6D99682D
:10133000BA6B13465B0013445B000B441B797B774D
:101340007B6D9968BA6B13465B0013445B000B44DA
:101350001B78BB767B6D9968BA6B13465B001344B0
:101360005B000B445B883B837B6D9968BA6B1346CB
:101370005B0013445B000B445B78FB76BB7EDB09B0
:10138000DBB2012B18D1FB7E022B15D1BB7E03F003
:101390000F03DAB27B685A777B6800229A777B6802
:1013A0004FF0FF325A617B6800221A777B68002277
:1013B0009A61204BFB601EE0BB7E5BB2002B1ADB08
:1013C000FB7E022B17D1BB7E03F00F03DAB27B68E2
:1013D00083F82D207B68002283F82E207B684FF055
:1013E000FF325A627B68002283F82C207B6800223F
:1013F0009A62114BFB607B683B617B681B6807F15D
:101400000C0207F11801184616F05BF9034687F83D
:101410005330BB6B0133BB637B6D1B791A46BB6BCF
:10142000934281D397F8533018465837BD4680BD54
:10143000C3780100177901006979010080B59AB07D
:1014400000AFF860B9607A60012387F867307B6885
:10145000002B02D0FB68002B01D1032309E3FB68BA
:101460003B65BB68013B052B00F2EE8201A252F8FE
:1014700023F000BF6D1800008D14000097140000C9
:10148000F114000065150000451600003B6D0022B8
:1014900083F84020EBE27B68FB643B6D5B68002BCC
:1014A00000F0D482FB6C1A783B6D93F840309A427E
:1014B00000F0CE82386D16F081FA034687F8673067
:1014C000FB6C1A783B6D83F840203B6D002283F85B
:1014D0004220386DFFF7DEFD034687F8673097F846
:1014E0006730002B00F0B682924814F085F9B1E223
:1014F0003B6D5B68002B00F0AF827B681B88A7F810
:101500004A30B7F84A3087F849303B6D93F84120AC
:10151000B7F84A301B0A9BB2DBB29A4240F09E8277
:101520003B6D93F8423097F849209A4200F0988238
:10153000386D16F043FA034687F867303B6D97F82D
:10154000492083F84220386DFFF7A4FD034687F851
:10155000673097F86730002B00F08482764814F0EB
:101560004BF97FE23B6D5B68002B00F07D823B6DA9
:101570009B68002B00F078823B6DDB68002B00F04D
:1015800073827B68FB6400233B661FE0FB6C197869
:101590003B6D9B6898683A6E13465B0013445B0092
:1015A00003441B7899420ED13B6D012283F83C2005
:1015B0003B6D1A68FB6C1B781946104616F038F91B
:1015C000034687F867303B6E01333B663B6D9B6893
:1015D0001B791A463B6E9342D8D30023FB6529E062
:1015E000FB6C19783B6DDB689868FA6D13465B00FD
:1015F00013445B0003441B78994218D1FB6C1B78A1
:10160000DB09DBB2012B03D13B6D01221A7703E02A
:101610003B6D012283F82C203B6D1A68FB6C1B7814
:101620001946104616F004F9034687F86730FB6D3B
:101630000133FB653B6DDB681B791A46FB6D9342FA
:10164000CED314E23B6D5B68002B00F00D823B6D46
:101650009B68002B00F008823B6DDB68002B00F0DC
:1016600003827B68FB640023BB6559E0FB6C19783F
:101670003B6D9B689868BA6D13465B0013445B0032
:1016800003441B78994248D13B6D1A68FB6C1B7868
:101690001946104616F0E4F8034687F86730FB6CED
:1016A0001B78DB09DBB2012B37D13B6D93F83C3063
:1016B000002B32D03B6D002283F83C203B6D5B6BEE
:1016C000B3F1FF3F29D03B6D18683B6D93F83D1097
:1016D0003B6D5A6B3B6D9B6B15F0C4FF034687F85F
:1016E000673097F86730002B10D03B6D5B6BBB62A7
:1016F0003B6D9B6BFB62002387F830303B6D1B68B2
:1017000007F12801FA68184616F005F93B6D4FF00D
:10171000FF325A633B6D00229A63BB6D0133BB6598
:101720003B6D9B681B791A46BB6D93429ED3002389
:101730007B6592E090C50100D8C50100FB6C19786B
:101740003B6DDB6898687A6D13465B0013445B0061
:1017500003441B7899427DD13B6D1A68FB6C1B7862
:101760001946104616F07CF8034687F86730FB6C84
:101770001B78DB09DBB2012B35D13B6D1B7F002BC6
:1017800068D03B6D00221A773B6D5B69B3F1FF3F78
:1017900060D03B6D18683B6D597F3B6D5A693B6D5E
:1017A0009B6915F05FFF034687F8673097F867304D
:1017B000002B10D03B6D5B69FB613B6D9B693B620D
:1017C000002387F824303B6D1B6807F11C01FA6881
:1017D000184616F0A0F83B6D4FF0FF325A613B6D92
:1017E00000229A6136E03B6D93F82C30002B31D00B
:1017F0003B6D002283F82C203B6D5B6AB3F1FF3F09
:1018000028D03B6D18683B6D93F82D103B6D5A6ADC
:101810003B6D9B6A15F03FFF034687F8673097F8EA
:101820006730002B0FD03B6D5B6A3B613B6D9B6A61
:101830007B6100233B763B6D1B6807F11001FA6862
:10184000184616F091F83B6D4FF0FF325A623B6D2F
:1018500000229A627B6D01337B653B6DDB681B79EF
:101860001A467B6D9342FFF469AF00E17B68002B61
:1018700000F0E8807B687B647B6C1B689B88DBB234
:101880003A6D92F84120934240F0F0807B6C1B68E7
:101890001B7803F06003202B40F0D4807B6C043372
:1018A0007B637B6C0833BB637B6C1B689B88BB874B
:1018B0007B6C1B685B88FB877B6C1B7B87F84030ED
:1018C0007B6C1B685B78232B00F2B88001A252F876
:1018D00023F000BF651900007D1900009519000074
:1018E000AD190000C51900003D1A00003D1A0000A6
:1018F0003D1A00003D1A00003D1A00003D1A00008C
:101900003D1A00003D1A00003D1A00003D1A00007B
:101910003D1A00003D1A00003D1A00003D1A00006B
:101920003D1A00003D1A00003D1A00003D1A00005B
:101930003D1A00003D1A00003D1A00003D1A00004B
:101940003D1A00003D1A00003D1A00003D1A00003B
:101950003D1A0000F5190000DD1900000D1A000005
:10196000251A00003B6D5B681B68386D07F1340277
:1019700004219847034687F8673064E03B6D5B6855
:101980001B68386D07F1340205219847034687F834
:10199000673058E03B6D5B681B68386D07F13402B7
:1019A00006219847034687F867304CE03B6D5B683B
:1019B0001B68386D07F1340207219847034687F802
:1019C000673040E03B6D5B681B68386D07F134029F
:1019D00008219847034687F8673034E03B6D5B6821
:1019E0001B68386D07F1340209219847034687F8D0
:1019F000673028E03B6D5B681B68386D07F1340287
:101A00000A219847034687F867301CE03B6D5B6806
:101A10001B68386D07F134020B219847034687F89D
:101A2000673010E03B6D5B681B68386D07F134026E
:101A30000C219847034687F8673004E0052387F8B0
:101A4000673000E000BF12E000BF10E000BF0EE012
:101A500000BF0CE000BF0AE000BF08E000BF06E0E6
:101A600000BF04E000BF02E000BF00E000BF97F845
:101A7000673018466837BD4680BD00BF80B586B068
:101A800000AF0346B9607A60FB730123FB7507F171
:101A900010031846FFF7D2FA0346FB75FB7D002BB7
:101AA00001D0FB7D44E03B691A46FB7B114618469A
:101AB00000F060F90346FB75FB7D002B01D0FB7D38
:101AC00036E03B691B68002B01D1032330E03B6902
:101AD000BA685A603B69002283F840203B69FF22C4
:101AE00083F842203B6910331846FEF7E1FC0346B9
:101AF000002B02D0104813F07FFE3B6920331846BC
:101B0000FEF7D6FC0346002B02D00B4813F074FE00
:101B10003B6930331846FEF7CBFC0346002B02D05E
:101B2000054813F069FE3B691A467B681A60FB7D25
:101B300018461837BD4680BD1CC6010080B584B06C
:101B400000AF78600123FB737B68BB60BB68002B30
:101B500001D1032329E0BB681B69184614F06CF817
:101B60000346002B02D0134813F046FEBB681B6AE5
:101B7000184614F061F80346002B02D00D4813F00C
:101B80003BFEBB681B6B184614F056F80346002B4F
:101B900002D0084813F030FEB86815F00FFF034676
:101BA000FB73B86815F074FEFB7B18461037BD4612
:101BB00080BD00BF30C6010080B584B000AF0346D1
:101BC0003960FB7107F10803184614F01CF8002374
:101BD000FB6018E0284AFB681B0113441B68002BBC
:101BE0000ED0254AFB681B0113440E331B78FA798B
:101BF0009A4205D1BB68184614F013F8012337E068
:101C0000FB680133FB60FB68002BE3D00023FB6023
:101C100026E0194AFB681B0113441B68002B1CD1EA
:101C2000154AFB681B0113440E33FA791A70FB68DE
:101C3000DB00124A1A441049FB681B010B440833AD
:101C40001A60FB681B010C4A1A443B681A60BB68A7
:101C5000184613F0E6FF00230AE0FB680133FB603F
:101C6000FB68002BD5D0BB68184613F0DAFF0223BF
:101C700018461037BD4680BD98070020A8070020F1
:101C800080B584B000AF0346FB710023FB6007F111
:101C90000803184613F0B7FF2CE01C4AFB681B0131
:101CA00013441B68002B22D0184AFB681B01134405
:101CB0000E331B78FA799A4219D1144AFB681B013A
:101CC000134400221A60114AFB681B0113440433B9
:101CD00000221A600D4AFB681B0113440E330022D8
:101CE0001A70BB68184613F09CFF00230AE0FB68DB
:101CF0000133FB60FB68002BCFD0BB68184613F0A4
:101D000090FF042318461037BD4680BD9807002079
:101D100080B584B000AF786039600023FB6007F1C4
:101D20000803184613F06FFF16E0114AFB681B0109
:101D300013441B687A689A420BD1FB681B010C4A5A
:101D40001A443B681A60BB68184613F06AFF002308
:101D50000AE0FB680133FB60FB68002BE5D0BB6841
:101D6000184613F05EFF042318461037BD4680BDA9
:101D70009807002080B584B000AF03463960FB713E
:101D80000023FB6007F10803184613F03CFF1FE037
:101D9000154AFB681B0113441B68002B15D0124A1F
:101DA000FB681B0113440E331B78FA799A420CD15D
:101DB0000D4AFB681B0113441A683B681A60BB6834
:101DC000184613F02EFF00230AE0FB680133FB6086
:101DD000FB68002BDCD0BB68184613F022FF0423FD
:101DE00018461037BD4680BD9807002090B587B0D3
:101DF00000AFF8600B467A60FB7201233B7501234C
:101E00007B757B68002B01D1042359E007F1100397
:101E10001946F868FFF77CFF03463B753B7D002BB6
:101E200001D004234CE00023BB7542E00023FB7586
:101E300037E0FB7D244A1B0113440C3319783B69BE
:101E40005B681868BA7D13465B0013449B0003442B
:101E50009B681B79994221D1FB7D1B4A1B011344CE
:101E600008331C683B695B681968BA7D13465B00E0
:101E700013449B000B445B681846FB7A7A6819464A
:101E8000A04703463B753B7D052B01D1052317E099
:101E90003B7D002B09D100237B7506E0FB7D0133E0
:101EA000FB75FB7D012BC4D900E000BFBB7D013376
:101EB000BB753B695B681B7ABA7D9A42B6D37B7D62
:101EC00018461C37BD4690BD48C6010090B587B086
:101ED00000AF0346B9607A60FB7301237B757B68B2
:101EE000002B06D0BB68002B03D0BB685B68002BBF
:101EF00001D1042370E007F11002FB7B1146184664
:101F0000FFF75AFE03467B757B7D002B01D07B7D5E
:101F100062E03B69BA685A603B691A46FB7B30490C
:101F2000184615F0BDFA03467B757B7D002B0AD061
:101F30003B691B68184615F074FBFB7B1846FFF7DE
:101F40009FFE7B7D48E00023BB753AE00023FB75D4
:101F500031E03B695B681968BA7D13465B00134446
:101F60009B000B449B681A79FB7D1E491B010B44A7
:101F70000C331B789A421BD1FB7D1A4A1B01134478
:101F80001C683B695B681968BA7D13465B001344A3
:101F90009B00C8183B695B681968BA7D13465B00F3
:101FA00013449B000B441A1DFB7B01461846A047B7
:101FB000FB7D0133FB75FB7D012BCAD9BB7D013352
:101FC000BB753B695B681B7ABA7D9A42BED33B699D
:101FD0001A687B681A607B7D18461C37BD4690BD29
:101FE000897B010048C6010080B483B000AF7860EF
:101FF00039603B68054A1A603B6812225A60002328
:1020000018460C37BD465DF8047B70475C00002025
:1020100080B483B000AF786039603B681B7A002BD6
:1020200007D13B68064A1A603B6843225A60002386
:1020300000E0052318460C37BD465DF8047B704769
:102040007000002080B485B000AF786039603B68D4
:102050009B7A002B08D12A4B1A683B681A60284BE0
:102060005A683B685A6044E00023FB730323BB7348
:1020700017E03B681989224B9868FA7B13465B008E
:1020800013449B0003441B89994207D13B689B7A08
:10209000022B0AD83B689B7ABB7306E0FB7B0133BB
:1020A000FB73FB7B002BE4D000E000BFBB7B032B6A
:1020B00001D105231EE0124B9968FA7B13465B00A1
:1020C00013449B000B441A68BB7B9B0013441A68A3
:1020D0003B681A600A4B9968FA7B13465B0013440D
:1020E0009B000B445A68BB7B9B0013441A683B68F7
:1020F0005A60002318461437BD465DF8047B7047CC
:102100003001002080B483B000AF0346FB7197F923
:102110000730002B0BDBFB7903F01F02074997F90F
:1021200007305B09012000FA02F241F8232000BFCA
:102130000C37BD465DF8047B704700BF00E100E04E
:1021400080B483B000AF03463960FB7197F9073064
:10215000002B0ADB3B68DAB20C4997F90730120111
:10216000D2B20B4483F800230AE03B68DAB2084994
:10217000FB7903F00F03043B1201D2B20B441A7631
:1021800000BF0C37BD465DF8047B704700E100E0FE
:1021900000ED00E080B582B000AF78600D4B1B68A9
:1021A00018460BF0BBFD0346002B03D17B680022D1
:1021B0001A700CE0074B1B68796818460BF01EFE7E
:1021C0000346002B03D07B6800221A7000BF08373B
:1021D000BD4680BDB007002080B584B000AF034687
:1021E000FB713223FB6008E0012010F07FFBFB68ED
:1021F000002B0DDDFB68013BFB60084B1B68FA1DE3
:10220000114618460BF0A6FD0346002BECD100E06A
:1022100000BF00BF1037BD4680BD00BFB40700201F
:1022200080B500AF064B1B6818460BF077FD0346E0
:10223000002B14BF01230023DBB2184680BD00BF72
:10224000B007002080B500AF044B1B68184614F09F
:102250002EFCBFF34F8F00BF00BF80BDB80700202A
:1022600080B58CB000AFF860B9607A60012387F860
:102270002F30954B7B627B683B627B68FB61BB6860
:10228000013B0B2B00F2AC8101A252F823F000BFFE
:10229000C12200003F230000A7230000E125000029
:1022A000E1250000B723000005240000E12500001F
:1022B0003F2400005724000079240000E12500009D
:1022C000FB695B68002B15D0FB695B687F4A52880D
:1022D000B3FBF2F101FB02F29B1A002B0AD100239F
:1022E00000220221F86815F0C0FB034687F82F3062
:1022F00000BF77E1764B1B7ADBB2012B40F0728195
:10230000734B9B7ADBB2012B40F06C81FB691B683D
:10231000002B09D1FB691B68002B40F06381FB692E
:102320005B68002B40F05E81684B5B88694A032143
:10233000F86815F0EBFB034687F82F3052E1644B49
:102340001B7ADBB2012B40F04F81614B9B7ADBB2F1
:10235000012B40F04981FB695B683B613B69002BC5
:1023600016D03B69B3F1FF3F12D00023BB620BE0F4
:10237000594B1A68BB6A57490B44194610460BF073
:10238000E9FCBB6A0133BB62BA6A3B699A42EFD38C
:102390004E4B5B884F4A0321F86815F0B7FB0346A4
:1023A00087F82F3020E1FB68002283F843200023C8
:1023B00087F82F3019E13B6A5B89012B0DD13B6A0D
:1023C0001B7B012B04D13B6A1B68444A1A6015E051
:1023D0003B6A5B6800221A6010E03B6A5B89022B53
:1023E0000CD13B6A1B7B012B04D13B6A1B683C4A26
:1023F0001A6003E03B6A5B6800221A60002387F8DA
:102400002F30F2E03B6A5B89012B08D13B6A1B68E5
:10241000324A1A603B6A5B6802221A600BE03B6A30
:102420005B89022B07D13B6A1B682D4A1A603B6A05
:102430005B6802221A60002387F82F30D5E03B6AE0
:102440001B68284A1A603B6A5B6807221A600023EF
:1024500087F82F30C9E03B6A1B7B012B04D13B6A14
:102460001B68204A1A6003E03B6A5B6800221A601E
:10247000002387F82F30B8E03B6A5B89DAB2124B51
:102480009A737B6A9B7B03F00203002B07D07B6A65
:102490001B8A43F002039AB27B6A1A8206E07B6AC7
:1024A0001B8A23F002039AB27B6A1A827B6A9B7BA7
:1024B00003F00103002B17D07B6A1B8A43F0010352
:1024C0009AB27B6A1A8216E0D0070020080000202A
:1024D000B8070020E4070020B0070020C80700204C
:1024E000CC070020400100207B6A1B8A23F00103F7
:1024F0009AB27B6A1A827B6A9B7B03F00103002BF2
:1025000014BF01230023DAB27B6A9A727B6A1B8AAA
:10251000DBB218460AF050F97B6AA1221A707B6A76
:1025200020225A707B6A00229A707B6A0022DA703D
:102530007B6A00221A717B6A00225A717B6A02222E
:102540009A717B6A0022DA713B6A1B89DAB27B6A74
:102550001A717B6A0833BB617B6A1B8ADAB2BB697A
:102560001A707B6A1B8A1B0A9AB2BB690133D2B20A
:102570001A700A237B61FB6893F84330002B13D158
:102580007A6A7B690121F86815F06FFA034687F8CB
:102590002F3097F82F30002B02D0174813F02CF96A
:1025A000FB68012283F843207B6A9B7B03F00103D5
:1025B000002B08D1114B1B7ADBB2002B0CD07B6AAD
:1025C0009B7B022B08D10D4B1B7ADBB2012B06D172
:1025D0000A4B01229A7202E0084B1B7A05E004E0E4
:1025E00000BF02E000BF00E000BF97F82F301846A0
:1025F0003037BD4680BD00BF7CC60100B807002053
:1026000080B588B000AFF860B9607A600123FB77CD
:102610007B68BB617B687B61BB68013B152B00F26B
:102620008C8001A252F823F0812600003B27000095
:102630003B2700003B2700003B2700003B27000012
:102640003B2700003B2700008F260000D326000018
:10265000FF26000013270000272700003B2700006B
:102660003B2700003B2700003B2700003B270000E2
:102670003B2700003B2700003B2700003B270000D2
:10268000354B00221A72344B0022DA725EE07B690D
:102690001B78002B06D1304B00221A722E4B0022E1
:1026A000DA7253E07B691B78012B0FD12A4B012290
:1026B0001A727B691A78284BDA72274B5868274BB5
:1026C0005B88274A032115F021FA3FE00523FB77B9
:1026D0003CE0214B1B7ADBB2002B30D0BB691B885E
:1026E0001B0A9BB2FB74BB691B88BB74FB7C012B70
:1026F00025D8FB7C184A1344BA7C1A731FE07B6808
:10270000002B1ED07968F868FFF76EFC0346FB7754
:1027100017E07B68002B16D07968F868FFF778FC23
:102720000346FB770FE07B68002B0ED07968F868D2
:10273000FFF788FC0346FB7707E000BF06E000BF19
:1027400004E000BF02E000BF00E000BFFB7F1846CE
:102750002037BD4680BD00BFB8070020080000201C
:10276000E407002080B582B000AF786015F06FFA02
:10277000054B1B68184614F046FF00F08BF8052047
:1027800010F0B4F8F9E700BFB807002080B584B0B6
:1027900002AF0021294815F03EFA294B00225A7257
:1027A000274B00221A72264B00225A60244B00222B
:1027B0001A60234A23490020FFF788FB0346002BB9
:1027C00003D0214813F018F807E0204813F014F85C
:1027D0001C4B1B685B681A4A536015F038FA184B9B
:1027E0001B68184614F00FFF3B4618460BF020FA02
:1027F00001237B604FF480433B603B4618460BF05F
:102800003DFA0346124A13603B4618460BF036FA6F
:102810000346104A1360002301930523009300230D
:1028200096220D490D4819F00FFB0346012B00D0ED
:10283000FEE700BF0837BD4680BD00BF00D00040A6
:10284000B807002054010020ACC60100C8C6010032
:10285000B0070020B4070020E8C60100652700008B
:1028600080B400AF0A4B1B7ADBB2012B06D1084BB8
:102870009B7ADBB2012B01D1012300E0002303F09E
:102880000103DBB21846BD465DF8047B704700BF0C
:10289000B807002080B582B000AF0123FB701C4B4D
:1028A0001B7ADBB2012B2FD1194B9B7ADBB2012BA8
:1028B0002AD1184B1B6818460BF030FA0346002B40
:1028C00022D000237B600BE0124B1A687B68124910
:1028D0000B44194610460BF091FA7B6801337B607C
:1028E0007B683F2B07D80B4B1B6818460BF016FA7A
:1028F0000346002BE8D1064B58687B68064A022144
:1029000015F0B3F80346FB7000BF0837BD4680BD25
:10291000B8070020B40700202408002080B582B04A
:1029200000AF78603960054A3968786817F068F94F
:10293000034618460837BD4680BD00BFECC60100FF
:1029400080B584B000AF78600023FB600FE00C49D5
:10295000FA6813465B0013449B000B441B685B68DA
:102960001946786816F0E6FFFB680133FB60FB68E8
:10297000012BECD900BF00BF1037BD4680BD00BFA2
:102980004CC7010090B585B000AF78600CF01CFA20
:1029900003465B681946204816F0CCFF0023FB6015
:1029A0000DE01E49FA6813465B0013449B000B447C
:1029B00004331B6800221A70FB680133FB60FB685C
:1029C000012BEED90023FB601FE01449FA6813467F
:1029D0005B0013449B000B44043318680F49FA68EA
:1029E00013465B0013449B000B44083319680B4CDF
:1029F000FA6813465B0013449B0023441A68084B93
:102A000017F07CF9FB680133FB60FB68012BDCD914
:102A100014200FF06BFFD5E764C701004CC701001D
:102A2000ECC6010080B582B002AF002301930223FF
:102A300000930023C8220A490A4819F005FA034600
:102A4000012B00D0FEE70BF039FF034618460CF0CF
:102A5000ABF9054809F064FE00BFBD4680BD00BF6C
:102A60007CC701008529000038C7010080B483B00D
:102A700000AF0346FB7197F90730002B0BDBFB79A6
:102A800003F01F02074997F907305B09012000FA9C
:102A900002F241F8232000BF0C37BD465DF8047BED
:102AA000704700BF00E100E080B483B000AF034690
:102AB0003960FB7197F90730002B0ADB3B68DAB20B
:102AC0000C4997F907301201D2B20B4483F8002366
:102AD0000AE03B68DAB20849FB7903F00F03043BD4
:102AE0001201D2B20B441A7600BF0C37BD465DF816
:102AF000047B704700E100E000ED00E080B586B0A7
:102B000000AFF860B9607A607B68002B06D10A4B91
:102B10000A4A4FF484710A4812F046F9BB689B00D8
:102B2000FA6813447B617B697A6812881A8000BF57
:102B30001837BD4680BD00BFB0C8010054C80100B1
:102B400084C7010080B582B000AF00237B60084BD2
:102B50001B68184609F0E0FB0346002B03D07B6896
:102B600043F001037B607B6818460837BD4680BD93
:102B70006408002080B584B002AF03463960FB7161
:102B8000FB79042B34D801A252F823F0A12B0000CA
:102B9000B12B0000C12B0000D12B0000E12B000065
:102BA00039681C4818F0CBF9022004F0F9F82DE040
:102BB0003968194818F0C3F9032004F0F1F825E04A
:102BC0003968164818F0BBF9052004F0E9F81DE053
:102BD0003968134818F0B3F9062004F0E1F815E05D
:102BE0003968104818F0ABF9042004F0D9F80DE06A
:102BF0000D4B98686423009300230022032110F0FA
:102C0000D5FF3968094818F09AF900BF00BF0837A6
:102C1000BD4680BDC0C70100D0C70100E0C70100AC
:102C2000F4C7010008C801006001002018C80100B5
:102C300080B582B000AF7860034809F0E3FB00BFC5
:102C40000837BD4680BD00BF6001002090B587B049
:102C500002AF78600B46FB700023BB60224B1B78F1
:102C6000002B3DD1204A7B68D3601F4B01221A7094
:102C70001D4809F0C7FBFB78002B0ED01A4B9C684F
:102C80000FF0CEFF024607F1080300210091062154
:102C9000204610F08BFFF8600CE0134B9C680FF09F
:102CA000AFFF02466423009300230121204610F069
:102CB0007DFFF860FB68012B05D00C4B0C4A962178
:102CC0000C4812F071F8FB78002B09D0BB68002B80
:102CD00004D00EF05FF80FF03BFC01E00EF03EF880
:102CE00000BF1437BD4690BD6001002024C801001C
:102CF00044C8010030C8010080B582B000AF0C4864
:102D000002F036F878607B6803F48043002B08D02B
:102D10004FF48041064802F043F801210120FFF7FB
:102D200095FFBFF34F8F00BF00BF0837BD4680BD82
:102D300000F00F4080B500AF034B1B68184616F03B
:102D4000E1FB00BF80BD00BF6408002080B588B0F3
:102D500002AF3B1D184609F0C1FA01233B711E4B1F
:102D6000BB601E4BFB600E233B613B1D184609F008
:102D7000FDFA03461A4A13600E21184815F026F989
:102D800003463B803B7843F003033B703B461A46C7
:102D90000E211248FFF7B2FE0A220E210F4815F04D
:102DA000F8F805213B20FFF77FFE3B2015F0DBF80C
:102DB0000C4B00930223012214210B4819F09DF9BA
:102DC00003460A4A9360094B9B68002B00D1FEE73B
:102DD00000BF1837BD4680BD00F00F400090044092
:102DE00064080020312C00003CC801006001002074
:102DF00080B586B000AF3B1D18460AF0BDFC01232C
:102E00003B710F4BBB600F4BFB600D233B613B1DC8
:102E100018460AF0CFFC03460B4A13600B4BBB600D
:102E20000B4BFB6000233B613B1D18460AF0C2FCC4
:102E30000346084A136000BF1837BD4680BD00BF77
:102E400000F00F400090044068080020C0F00F40E0
:102E500000C004406C08002080B500AF2C4815F07D
:102E6000D4F82C4815F0D1F82B4815F0CEF82B48A3
:102E700015F0CBF82A4815F0C8F816F0DAFC16F071
:102E800008FD16F038FB0CF039FC17F043FD16F086
:102E9000C9FC16F0A9FC16F035FD17F0ACFD03F0E7
:102EA000F5FF0CF0F3F816F048FBFFF76FFCFFF7A7
:102EB0009FFFFFF74BFF08F0C5FB16F077FA06F00F
:102EC00007FE0AF0BBF904F003F905F04FFD15F019
:102ED000B6F805F079FCFFF7A5FD07F015FE09F03F
:102EE000A5F806F061FA04F0DFFC03F08BFA03F0BA
:102EF000CDFF07F087FF08F03DF903F013FF15F051
:102F0000F9FD03F02BF815F0DAFC00BF80BD00BF1F
:102F1000090038100A0038100B0038100C00381067
:102F20000D00381080B584B000AF78600023FB60DE
:102F300009E00E4AFB6852F823307A689A4206D0BC
:102F4000FB680133FB60FB68012BF2D900E000BF96
:102F5000FB68012B05D9064B064A4A21064811F0A9
:102F600023FFFB6818461037BD4680BD68C80100C6
:102F700078C80100D8C801009CC8010080B584B0A1
:102F800000AF786039603B68002B05D13E4B3F4A6B
:102F900051213F4811F008FF7868FFF7C3FF03464F
:102FA0003C4A52F82330184615F068F83B685B78C5
:102FB00003F003023B681B799B0003F00C031343EF
:102FC000FB603B685B79042B03D0FB6843F0100384
:102FD000FB603B68DB785B0103F06003FA68134336
:102FE000FB603B68DB79002B03D0FB6843F0800378
:102FF000FB607B68FA689A607B68DB6823F00F03EC
:10300000FB603B685B79042B06D03B685B7903F07F
:103010000303FA681343FB603B689B79002B03D0E2
:10302000FB6843F00403FB603B689B78002B03D0F4
:10303000FB6843F00803FB607B68FA68DA607B6832
:103040001B6A23F00303FB603B681B7803F0030358
:10305000FA681343FB607B68FA681A623B681B7A64
:10306000002B06D07B685B6A43F008027B685A62DB
:1030700005E07B685B6A23F008027B685A6200BF48
:103080001037BD4680BD00BFA8C80100ECC80100D4
:103090009CC8010070C8010080B582B000AF7860A4
:1030A0007B68002B05D1124B124A9121124811F076
:1030B0007BFE7B6800221A707B6803225A707B6853
:1030C00001229A707B680322DA707B6801221A71F0
:1030D0007B6804225A717B6800229A717B68002207
:1030E000DA717B6800221A7200BF0837BD4680BDC6
:1030F000A8C80100F8C801009CC8010080B586B0CE
:1031000000AFF860B9607A60BB68012B06D9174B35
:10311000174A40F25711174811F046FE7B68002B02
:1031200006D1154B124A4FF4AC71124811F03CFE17
:103130007B681B6803F01F037B617B685B79002B56
:1031400003D07B6943F020037B617B681B79002BF4
:1031500003D07B6943F040037B61FB68BA687969FF
:1031600043F8221000BF1837BD4680BDB8C8010023
:1031700010C901009CC80100A8C8010080B584B036
:1031800000AF786039603B68012B06D90C4B0D4AC3
:1031900040F26D110C4811F007FE0023FB607B68C4
:1031A0003A6853F8223003F08003002B03D0FB6809
:1031B00043F08003FB60FB6818461037BD4680BDB6
:1031C000B8C8010028C901009CC8010080B483B0C0
:1031D00000AF7860084B1B6823F440227B689B0497
:1031E00003F44023044913430B6000BF0C37BD4672
:1031F0005DF8047B704700BF0070044080B483B06A
:1032000000AF78600A4B03F580535B6823F480328B
:103210007B681B0403F480330549134301F5805296
:10322000536000BF0C37BD465DF8047B704700BF9C
:103230000070044080B582B000AF174B1B7BDBB23F
:1032400003F00103002B02D0012B0ED01BE0134B27
:103250001B68002B05D1124B124AEC21124811F0C9
:10326000A3FD0E4B1B687B6010E0104B1B68002B0E
:1032700005D10F4B0B4AF1210B4811F095FD0B4B7B
:103280001B687B6002E000237B6000BF7B68184600
:103290000837BD4680BD00BF0040064070080020D2
:1032A00044C9010078C9010050C901007408002018
:1032B0005CC9010080B582B000AFFFF7BBFF78604A
:1032C0007B68002B01D17B6844E0244B1B78DBB288
:1032D000DB08DBB203F00703FB70FB787A6822FAA5
:1032E00003F37B601D4B5B78DBB21B09DBB203F0A1
:1032F0000303BB70194B1B7BDBB203F001037B7034
:10330000BB78002B24D07B78002B21D1FB78072BB6
:1033100014D0072B19DC052B02DC002B03DA14E098
:10332000062B04D011E07B685B097B6011E07B68B1
:103330000B4AA2FB03231B097B600AE07B68094A56
:10334000A2FB0323DB087B6003E000237B6000E03B
:1033500000BF7B6818460837BD4680BD0040064068
:10336000CDCCCCCCABAAAAAA80B400AF0C4B9B7935
:10337000DBB203F00103002B02D10A4B1B6809E00A
:10338000094B1A68064B1B7ADBB25B0803F0070394
:1033900022FA03F31846BD465DF8047B704700BF70
:1033A000004006408C0100209001002080B500AF55
:1033B000074B9B79DBB203F01003002B03D1FFF71F
:1033C00079FF034601E0034B1B68184680BD00BF30
:1033D000004006408C01002080B485B000AF7860CA
:1033E0007B6849F69702934202D80023FB7308E0FA
:1033F0007B68074A934202D80123FB7301E0022352
:10340000FB73FB7B18461437BD465DF8047B7047A1
:1034100000127A0080B500AF0B4B1B78DBB25BB2B9
:10342000002B0DDA094B1B68002B06D1084B094A0B
:1034300040F26D11084811F0B7FC044B1B6800E026
:103440000023184680BD00BF0050064070080020D1
:1034500044C9010090C9010050C9010080B582B083
:1034600000AF1A4B1B689B0C03F00303032B21D006
:10347000032B23D8002B02D0022B0CD01EE0FFF729
:10348000C9FF0346B3F5004F02D14FF4004300E0FB
:1034900000237B6015E00E4B1B68002B06D10D4B03
:1034A0000D4A40F281110D4811F07EFC084B1B685B
:1034B0007B6006E04FF47A737B6002E000237B6060
:1034C00000BF7B6818460837BD4680BD00700440C9
:1034D000740800205CC90100A8C9010050C901009E
:1034E00080B582B000AF0E4B03F580535B681B0CB8
:1034F00003F00103002B02D0012B04D007E000F001
:1035000067F9786006E000F0B3F9786002E0002324
:103510007B6000BF7B6818460837BD4680BD00BF92
:103520000070044080B584B000AF0346FB71FB79A6
:10353000132B00F2878001A252F823F08D35000092
:103540008D350000AB350000C9350000E7350000BF
:1035500045360000053600000D3600001536000027
:1035600045360000453600001D36000025360000B7
:103570002D36000035360000453600004536000087
:1035800045360000453600003D36000000F0EEF8FC
:103590000246304B03F580535B6C1B0F03F00F03A7
:1035A0000133B2FBF3F3FB604FE000F0DFF80246BB
:1035B000284B03F580535B6C1B0E03F00F030133A4
:1035C000B2FBF3F3FB6040E000F0D0F80246214B81
:1035D00003F580535B6C1B0D03F00F030133B2FB4B
:1035E000F3F3FB6031E000F0C1F80246194B03F53C
:1035F00080535B6C1B0C03F00F030133B2FBF3F33E
:10360000FB6022E0FFF76CFFF8601EE0FFF726FF8B
:10361000F8601AE0FFF7FEFEF86016E014F05FFEB7
:10362000F86012E000F012F9F8600EE000F0D0F857
:10363000F8600AE000F01CF9F86006E04FF47A73D5
:10364000FB6002E00023FB6000BFFB6818461037F8
:10365000BD4680BD0070044080B582B000AF786088
:10366000094A7B685B6802F5805253647B681B786B
:103670001846FFF7C3FD7B685B781846FFF7A6FD89
:1036800000BF0837BD4680BD0070044080B584B0DF
:1036900000AF786039600123FB732E4814F0C8FD39
:1036A0007B68002B0AD12C4B03F580535B682A4AB8
:1036B00023F4802302F58052536043E03B68274A9D
:1036C000934214D03B68254A93422CD83B68244A45
:1036D000934213D03B68224A934224D83B68214A44
:1036E000934219D03B68204A93420ED01BE01A4BFC
:1036F00003F580531A460923936417E0164B03F52C
:1037000080531A460223936410E0134B03F5805351
:103710001A460523936409E00F4B03F580531A46BC
:103720000023936402E00023FB7300BF0A4B03F500
:1037300080535B6823F4A02207497B68134301F59B
:1037400080525360034814F059FDFB7B1846103734
:10375000BD4680BD1200341000700440000E2707E3
:1037600000D8B805006CDC0200A24A0480B582B023
:1037700000AF164B9B79DBB29B0803F003033B6061
:103780003B68032B1AD801A252F823F0A53700009A
:10379000AD370000B53700009D37000000F068F835
:1037A00078600EE000F014F878600AE0FFF7DCFDC6
:1037B000786006E0FFF73EFD786002E000237B6062
:1037C00000BF7B6818460837BD4680BD00400640F4
:1037D00080B582B000AF1B4B5B78DBB203F0020315
:1037E000002B06D1174B9B79DBB203F02003002B93
:1037F00001D0002322E0FFF7D9FD78607B68002B21
:1038000001D17B681AE00F4BDB78DBB25B09DBB2DE
:1038100003F00303FB700B4BDB78DBB2DB09DBB29D
:1038200003F00103BB70FA78BB78074952001344D8
:1038300031F813301A467B6802FB03F31846083749
:10384000BD4680BD00400640C0C9010080B500AF44
:10385000064B1B78DBB203F00203002B01D10023DF
:1038600002E0FFF781FD0346184680BD0040064098
:1038700080B582B000AF184B9B79DBB203F04003F8
:10388000002B01D1002322E014F022FD78607B6838
:10389000002B06D1114B124A40F27A21114811F047
:1038A00083FA0D4B1B79DBB203F01F0301337A68F7
:1038B000B2FBF3F37B60084B5B79DBB203F01F03D1
:1038C00003F118027B6802FB03F37B607B681846F8
:1038D0000837BD4680BD00BF004006406CC90100EE
:1038E000D0C9010050C9010080B485B000AF0346C3
:1038F000FB71174B1B7BDBB203F00102FB799A4291
:1039000002D00123FB7301E00023FB73104B1B7BF0
:10391000DBB223F00103DAB2FB7903F00103DBB27F
:103920000B491343DBB20B73FB7B002B09D040F236
:10393000DC53BB6000E000BFBB685A1EBA60002BBE
:10394000F9D1002318461437BD465DF8047B704753
:103950000040064080B584B000AF78607B68002BE3
:1039600006D11E4B1E4A40F23A311E4811F01CFA95
:103970000023FB737B685B7803F01F03DAB2FB7BE9
:103980001343FB73184AFB7B1371174B5B79DBB254
:1039900023F01F03DAB27B689B7803F01F03DBB2CE
:1039A00011491343DBB24B710F4B1B79DAB27B68C1
:1039B0001B781343DBB20C4A43F04003DBB21371B4
:1039C00000BF094B9B79DBB203F04003002BF8D01A
:1039D00000BF00BF1037BD4680BD00BFB0C80100AA
:1039E000E4C9010050C901000040064080B584B020
:1039F00000AF78607B681B681846FFF7EDFC034654
:103A0000FB737B681B791946194814F047FC7B68E7
:103A100006331946164814F027FC164B5B78DBB2C8
:103A200023F03C03DAB2FB7B1B01DBB203F0300373
:103A3000DBB21343DAB27B685B790E491343DBB226
:103A40004B707B685B79002B0DD0094B1B78DBB288
:103A50005BB2002B07DA00BF064B9B79DBB203F0A9
:103A60000203002BF8D000BF1037BD4680BD00BF59
:103A7000005006400040064080B582B000AF0346CB
:103A80003960FB713B68002B06D1254B254A40F27B
:103A9000C651254811F088F9244B5B78DBB2234AE4
:103AA00023F00203DBB25370204B1B78DBB203F030
:103AB0003B03DBB21D4A63F07F03DBB2137000BF30
:103AC0001A4B9B79DBB203F01C03082BF8D1174B80
:103AD0005B79DBB2154A23F04003DBB2537100BFC0
:103AE000124B9B79DBB203F02003002BF8D138682E
:103AF000FFF730FF0D4B5B79DBB20C4A43F040031C
:103B0000DBB2537100BF094B9B79DBB203F020039A
:103B1000002BF8D0002318460837BD4680BD00BFF3
:103B2000B0C80100F8C9010050C9010000400640BA
:103B300080B582B000AF03463A60FB710B46BB71A3
:103B40003B68002B06D1134B134A4FF4CE61134848
:103B500011F02AF9FB791846FFF7C6FEBB793968E0
:103B60001846FFF789FF0E4B1B78DBB20C4A03F0B7
:103B70003F03DBB2137000BF094B9B79DBB29B089C
:103B800003F00303032BF7D1002318460837BD4683
:103B900080BD00BFB0C801000CCA010050C90100BF
:103BA0000040064080B582B000AF78603960786828
:103BB00014F0ACFB0346002B05D0094B1B68396899
:103BC0007868984704E0074B1B683968786898471D
:103BD000BFF34F8F00BF00BF0837BD4680BD00BF99
:103BE000840800208808002080B500AF094B1B68BE
:103BF000002B06D1084B094A40F2E161084811F058
:103C0000D3F8044B1B6819460648FFF7CBFF00BFEB
:103C100080BD00BF7808002050CA010080CA0100A2
:103C200044CA010000C0024080B500AF094B5B6888
:103C3000002B06D1084B094A40F2E961084811F00F
:103C4000B3F8044B5B6819460648FFF7ABFF00BFAB
:103C500080BD00BF7808002060CA010098CA01003A
:103C600044CA010000D0024080B500AF094B9B68F8
:103C7000002B06D1084B094A40F2F161084811F0C7
:103C800093F8044B9B6819460648FFF78BFF00BF6B
:103C900080BD00BF7808002070CA0100B0CA0100D2
:103CA00044CA010000C00A4080B586B000AF786009
:103CB0007B68002B01D1042353E02C4B03F5805388
:103CC000DB6C1B0EDBB203F00F03FB74FB7C0F2BD2
:103CD00003D14FF400237B6105E0FB7C244A32F8DA
:103CE00013309B027B617B6800221A607B687A69D3
:103CF0005A607B6801221A727B684FF48052DA6046
:103D00007B6800225A617B6800229A61786814F00F
:103D100052FB0346002B0ED0164B00221A60154BA7
:103D2000154A5A60134B154A9A607B68114ADA614A
:103D3000786814F0F9FA7B684FF0A0521A627B6839
:103D40004FF480525A627B684FF080529A627868D2
:103D500000F0FAF9F860FB68002B01D0FB6800E086
:103D6000002318461837BD4680BD00BF00700440D0
:103D7000F0CA01001409002094080020D408002093
:103D800080B590B000AFF860B9607A603B6007F131
:103D900010031A46B968F86814F06BFB3B6A7A683E
:103DA000B968F86814F024FBB863BB6B002B01D032
:103DB000BB6B48E0386800F0B3F9B863BB6B002B0D
:103DC00001D0BB6B3FE03B69BB607B697B63BA683A
:103DD0007B681344013BFB63FB6B7A6BB3FBF2F232
:103DE000796B01FB02F29B1A002B0BD0FA6B7B6BF9
:103DF000B2FBF3F301333B633B6B7A6B02FB03F3E0
:103E0000013BFB630021F86814F0BCFA11E0BB68C9
:103E100023F07F430E4A43F010631360F86800F00C
:103E200003F9B863BB6B002B08D1BA687B6B1344F2
:103E3000BB60BA68FB6B9A42E9D900E000BFF86842
:103E400014F094FABB6B18464037BD4680BD00BFE6
:103E50000400024080B58EB000AFF860B9607A60AF
:103E60003B607B68002B01D1042354E007F114036D
:103E70001A46B968F86814F0FCFA3B6A3A68B968FF
:103E8000F86814F0B5FA78637B6B002B01D07B6B7C
:103E900041E07B69BB600021F86814F073FA31E0FF
:103EA0007B681A1D7A601E4A04321B6813603B6AE5
:103EB000042B07D1BB6823F07F43194A43F0C0634A
:103EC000136010E03B6A082B0DD17B681A1D7A60E5
:103ED000134A08321B681360BB6823F07F43104A03
:103EE00043F0E0631360F86800F09EF878637B6B42
:103EF000002B0BD13B6ABA681344BB603B6A3A683B
:103F0000D31A3B603B68002BCAD100E000BFF868C1
:103F100014F02CFA7B6B18463837BD4680BD00BFC5
:103F20000400024080B58EB000AFF860B9607A60DE
:103F30003B60FB68002B02D07B68002B01D104237F
:103F400055E007F114031A46B968F86814F091FABD
:103F5000FA6A97F840303968B86800F00FFA786369
:103F60007B6B002B3DD07B6B41E0BB6823F07F4334
:103F7000214A43F040731360FB6A042B08D197F881
:103F800040301A061C4B083362F07F421A600AE088
:103F9000FB6A082B07D197F840301A06164B0433FA
:103FA00062F07F421A60F86800F03EF878637B6B3D
:103FB000002B1AD110497B681A1D7A604A681A6072
:103FC000FB6A082B05D10C497B681A1D7A608A6848
:103FD0001A60FB6ABA681344BB60FB6A3A68D31A7A
:103FE0003B603B68002BC0D100E000BF7B6B1846F4
:103FF0003837BD4680BD00BF0400024080B582B0A6
:1040000000AF78600C220649786818F04BF97B689D
:1040100001331A46034B1A6000BF0837BD4680BD06
:10402000C8CA01008C08002080B584B000AF786059
:10403000164B70221A70786814F0BDF9F860FB68AE
:10404000002B01D0FB681CE0114B1B680F48984700
:104050000E4B1B78FB72FB7A03F02003002B01D080
:1040600067230EE0FB7A03F01003002B01D06823D6
:1040700007E0FB7A03F00103002B01D0692300E085
:10408000002318461037BD4680BD00BF0000024027
:104090008C08002080B582B000AF78601C220649F1
:1040A000786818F0FFF87B6801331A46034B1A60F2
:1040B00000BF0837BD4680BDD4CA0100900800206B
:1040C00090B583B000AF00237B60074B7B60074B4C
:1040D0001C680F2314224FF470017868A04700BFBA
:1040E0000C37BD4690BD00BF04F001409008002091
:1040F00090B583B000AF00237B60074B7B60074B1C
:104100001C68012313224FF400217868A04700BFE8
:104110000C37BD4690BD00BF04F001409008002060
:1041200080B483B000AF78607B68064A934201D0C8
:104130006B2300E0002318460C37BD465DF8047B76
:10414000704700BF6B66656B80B588B002AF786062
:104150007B68002B01D104230AE107F10C02002344
:104160000093082384497868FFF7DCFE78617B6957
:10417000002B01D06E23FBE07B7C03F00F03DBB24E
:104180007B747B7C0F2B6FD801A252F823F000BF09
:10419000D1410000DB410000E5410000EF4100009B
:1041A000F9410000034200000D42000017420000E8
:1041B0001F420000274200002F4200003942000049
:1041C000434200004D42000057420000614200009F
:1041D0007B684FF6FF721A634BE07B684FF6FF7205
:1041E0001A6346E07B684FF480521A6341E07B68B3
:1041F0004FF400621A633CE07B684FF480621A63FC
:1042000037E07B684FF400721A6332E07B684FF44A
:1042100080721A632DE07B6880221A6329E07B6834
:1042200040221A6325E07B6820221A6321E07B6824
:104230004FF6FF721A631CE07B684FF6FF721A6339
:1042400017E07B684FF6FF721A6312E07B684FF647
:10425000FF721A630DE07B684FF6FF721A6308E085
:104260007B6800221A6304E07B684FF6FF721A63D2
:1042700000BF3B7C03F00F03DBB23B743B7C0F2B96
:1042800070D801A252F823F0C9420000D3420000C6
:10429000DD420000E7420000F1420000FB42000066
:1042A000034300000D430000174300001F430000BC
:1042B00029430000334300003D4300004743000012
:1042C000514300005B4300007B684FF40032DA6228
:1042D0004DE07B684FF0FF32DA6248E07B684FF4D4
:1042E000E032DA6243E07B684FF4C032DA623EE0EB
:1042F0007B684FF48032DA6239E07B680022DA6250
:1043000035E07B684FF0FF32DA6230E07B684FF0D7
:10431000FF32DA622BE07B680022DA6227E07B68FA
:104320004FF0FF32DA6222E07B684FF48042DA62BB
:104330001DE07B684FF40042DA6218E07B684FF4BE
:104340008032DA6213E07B684FF40032DA620EE00A
:104350007B684FF0FF32DA6209E07B684FF400328D
:10436000DA6204E07B684FF0FF32DA6200BF0023BC
:1043700018461837BD4680BDF803800080B487B06A
:1043800000AFF860B9607A60FB707B685A1EFB680A
:104390001340002B05D17B685A1EBB681340002BCD
:1043A00001D0652329E000237B61FA68BB681344D0
:1043B000013B3B61FB78012B0AD1FB68082B04D140
:1043C000FA68BB681344102B16D004237B6113E0FA
:1043D000FB78002B0ED13B69B3F5806F0CD3FB68E3
:1043E000B3F5000F03D33B69074A934204D9042372
:1043F0007B6101E004237B617B6918461C37BD4665
:104400005DF8047B704700BFFF03800080B584B077
:1044100000AF78600423BB600023FB6009E00F4A13
:10442000FB6852F823307A689A4207D0FB68013360
:10443000FB60FA68BB689A42F1D300E000BFFA68FB
:10444000BB689A4205D3064B064A6521064810F020
:10445000ABFCFB6818461037BD4680BD10CB010091
:1044600030CB010088CB01004CCB010080B487B079
:1044700000AF786039600023FB7500233B610023A7
:10448000FB607B689B6DFB60FB6843F00803FB608F
:104490007B685B6E3B610023FB750BE0FB7DDB0003
:1044A0000533012202FA03F33A6913433B61FB7DB2
:1044B0000133FB75FA7D7B682F498B4213D07B68F3
:1044C0002E498B420DD07B682D498B4207D07B68EB
:1044D0002C498B4201D1042306E0002304E0012390
:1044E00002E0012300E004239342D7DC7B683A69B1
:1044F0005A667B68D3F88C303B613B6943F0B40368
:104500003B613B6803F08003002B03D03B6943F41D
:10451000F8533B613B6803F07003002B1ED03B69EE
:1045200043F4F8133B613B6803F01003002B03D006
:10453000FB6843F01003FB603B6803F02003002B93
:1045400003D0FB6843F02003FB603B6803F04003AB
:10455000002B03D0FB6843F04003FB607B68FA68E4
:104560009A657B683A69C3F88C2000BF1C37BD464A
:104570005DF8047B704700BF00800340009003405B
:1045800000800B4000900B4080B485B000AF786095
:1045900039600023FB600023BB607B68D3F88C305C
:1045A00043F004027B68C3F88C207B685B6EBB60C1
:1045B0000023FB600BE0FB68DB000533012202FAFD
:1045C00003F3BA681343BB60FB680133FB607B688D
:1045D000464A934213D07B68454A93420DD07B688C
:1045E000444A934207D07B68434A934201D1042353
:1045F00006E0002304E0012302E0012300E004239D
:10460000FA689342D7D87B68BA685A667B68D3F851
:104610009830BB607B68354A934216D07B68344A39
:1046200093420FD07B68334A934208D07B68324A6A
:10463000934202D16FF0FF0309E0002307E06FF01F
:10464000030304E06FF0030301E06FF0FF03BA68B7
:104650001340BB607B68254A934214D07B68244A90
:1046600093420ED07B68234A934208D07B68224A4B
:10467000934201D1FF2307E04FF0FF3304E003230F
:1046800002E0032300E0FF233A681340BA681343B3
:10469000BB607B68BA68C3F898207B689B6DBB6081
:1046A0003B6803F48073002B04D0BB6843F0020323
:1046B000BB6003E0BB6823F00203BB603B6803F40C
:1046C0000073002B04D0BB6843F00103BB6003E020
:1046D000BB6823F00103BB607B68BA689A6500BFC2
:1046E0001437BD465DF8047B704700BF008003406F
:1046F0000090034000800B4000900B4080B584B0D8
:1047000000AF786039603B68002B05D1374B384AE1
:10471000E221384810F048FB3B685B6803F0F00387
:10472000002B01D101235DE07868FFF76FFE03469F
:10473000314A52F82330184613F001FF3B681B7BC7
:104740005B0103F0600343F005027B685A653B6838
:104750005B6819467868FFF789FE3B689B681946D5
:104760007868FFF711FF3B681B7803F007027B684E
:104770001A603B685B789B01DAB23B689B7E5B0208
:1047800003F400731A437B68C3F884203B681B7EE4
:104790001A467B68DA653B685B7E1A467B681A6757
:1047A0003B685A697B68DA663B689B7B9B01DAB29F
:1047B0003B681B6903F03F031A437B689A667B687A
:1047C000DB6FFB60FB6823F47063FB603B685B7B23
:1047D0001B0203F47063FA681343FB607B68FA689A
:1047E000DA67002318461037BD4680BDB0C8010007
:1047F00098CB01004CCB010020CB010080B582B0EA
:1048000000AF78607B68002B06D1174B174A40F247
:104810003311174810F0C8FA7B6800221A707B68C1
:1048200000225A707B6880225A607B6800229A605E
:104830007B6800221A737B6800225A737B6801220E
:104840009A737B6800221A617B6800225A617B6838
:1048500000221A767B6800225A767B6800229A76BC
:1048600000BF0837BD4680BDB0C80100A4CB010021
:104870004CCB010080B58AB000AFF860B96011463A
:104880001A460B46FB711346BB71BB68002B06D161
:10489000764B774A4FF4AB71764810F085FA7B6B14
:1048A000002B06D1744B724A40F25711714810F038
:1048B0007BFA3B6B002B06D1704B6D4A4FF4AC7109
:1048C0006C4810F071FAFB79002B06D16C4B684AEA
:1048D00040F25911674810F067FAFB681B6803F053
:1048E00007037A6B22FA03F3BB61BB79022B06D074
:1048F000022B1EDC002B02D0012B0DD019E0FB682F
:104900001B6823F02002FB681A60BA693B6BB2FB9C
:10491000F3F3013B7B620EE0FB681B6843F020026F
:10492000FB681A603B6B5B00BA69B2FBF3F37B6216
:1049300001E001232CE17B6AB3F5803F01D3012321
:1049400026E1FB687A6A9A600023FB771AE1BB686C
:104950009B78642B01D901231AE1BB79002B02D08B
:10496000BB79012B41D1BB681B78FA680133DB00AE
:1049700013445B687B617B6923F03C037B61BB680C
:104980005B789B001A467B6913437B617B6943F02C
:1049900020037B61BB681B78FA680133DB0013449A
:1049A0007A695A60BB689B78002B02D100237B8414
:1049B00012E0BB689B781A467B6A02FB03F3314A1C
:1049C000A2FB03235B097B847B8C7A6A9A4203D81F
:1049D0007B6A9BB201337B84BB681B787A8CF96855
:1049E0000133DB000B449A60C6E0BB681B781946B4
:1049F000FB68254A934213D0FB68244A93420DD0AA
:104A0000FB68234A934207D0FB68224A934201D1B4
:104A1000042306E0002304E0012302E0012300E078
:104A200004238B4201DC0123B2E0BB68DB78642BFA
:104A300001D90123ACE0BB68DB78002B02D1002355
:104A40003B840AE0BB68DB781A467B6A02FB03F30F
:104A50000C4AA2FB03235B093B84BB689B78002BB9
:104A60001AD100237B8400233B8428E058CB01002B
:104A7000BCCB01004CCB010064CB010070CB01002A
:104A80007CCB01001F85EB51008003400090034068
:104A900000800B4000900B40BB689B781A467B6AF5
:104AA00002FB03F33C4AA2FB03235B097B847B8C60
:104AB0007A6A9A4203D87B6A9BB201337B84BB68D3
:104AC0001B785B00FA680133DB0013445B687B6191
:104AD0007B6923F03C037B61BB685B789B001A46D3
:104AE0007B6913437B61BB681B785B00FA68013309
:104AF000DB0013447A695A60BB681B785B000133A2
:104B0000FA680133DB0013445B687B617B6923F047
:104B10003C037B61BB685B789B001A467B6913434F
:104B20007B61BB681B785B000133FA680133DB00F3
:104B300013447A695A60FB685A6EBB681B78DB00C5
:104B4000012101FA03F31A43FB685A66BB681B781C
:104B50005B003A8CF9680133DB000B449A603A8CB5
:104B60007B8C1A44BB681B785B0001331146FA68E2
:104B70000133DB0013449960BB680433BB60FB7FE7
:104B80000133FB77FA7FFB799A42FFF4E0AE002312
:104B900018462837BD4680BD1F85EB5180B485B0CF
:104BA00000AF7860084611461A460346FB700B4674
:104BB000BB7013467B700023BB817B689B687B8145
:104BC000BB78002B02D0BB78012B19D17B897A7876
:104BD00002FB03F32F4A82FB03125211DB17D31A95
:104BE000FB81FA897B899A4202D37B890133FB815D
:104BF000FB78FA8979680133DB000B449A6043E063
:104C0000FA787B6824498B4213D07B6823498B4216
:104C10000DD07B6822498B4207D07B6821498B42AB
:104C200001D1042306E0002304E0012302E0012374
:104C300000E00423934226DD7B897A7802FB03F3AC
:104C4000144A82FB03125211DB17D31AFB81FB7843
:104C50005B007A680133DB0013449B68BB81FA89EF
:104C60007B899A4202D37B890133FB81BA89FB8914
:104C70001A44FB785B00013311467A680133DB008C
:104C80001344996000E000BF1437BD465DF8047B13
:104C9000704700BF1F85EB51008003400090034028
:104CA00000800B4000900B4080B584B000AF78606E
:104CB0000023FB6009E00E4AFB6852F823307A6853
:104CC0009A4206D0FB680133FB60FB68042BF2D9E3
:104CD00000E000BFFB68042B05D9064B064A5821AB
:104CE000064810F061F8FB6818461037BD4680BDD5
:104CF000E0CB0100F4CB010024CC010018CC010072
:104D000080B584B000AFF860B9607A607B68002B32
:104D100005D1144B144A5F21144810F045F87B6804
:104D20001B78002B0AD1FB685A690121BB6801FA84
:104D300003F3DB431A40FB685A610FE07B685B7842
:104D40001A46B968F86813F02FFCFB685A6901210C
:104D5000BB6801FA03F31A43FB685A6100BF1037BE
:104D6000BD4680BDB0C8010038CC010018CC0100A0
:104D700080B584B000AF78607868FFF795FF034690
:104D8000FB73FB7B054A52F82330BB60BB68D3F84A
:104D9000A03018461037BD4680BD00BFCCCB010007
:104DA00080B584B000AF786039607868FFF77CFF29
:104DB0000346FB73FB7B064A52F82330BB60BB689B
:104DC0003A68C3F8A02000BF1037BD4680BD00BFC1
:104DD000CCCB010080B582B000AF786039607B68D1
:104DE000DB78DBB203F01003002B06D17B689B78E5
:104DF000DBB203F02003002B05D0094B1B68396898
:104E00007868984704E0074B1B68396878689847CA
:104E1000BFF34F8F00BF00BF0837BD4680BD00BF46
:104E20002C0900203009002080B500AF034B1B681F
:104E300019460348FFF7CEFF00BF80BD20090020C0
:104E40000060064080B500AF034B5B68194603481D
:104E5000FFF7C0FF00BF80BD2009002000700640A2
:104E600080B500AF034B9B6819460348FFF7B2FFBC
:104E700000BF80BD2009002000600E4080B584B0D6
:104E800000AF78600023FB6006E00D4A7B68934228
:104E900006D0FB680133FB60FB68002BF5D000E017
:104EA00000BFFB68002B05D0064B074A4C21074882
:104EB0000FF07AFFFB6818461037BD4680BD00BF73
:104EC0000070034048CC010078CC01006CCC01009C
:104ED00080B582B000AF786039603B68002B05D1A7
:104EE000134B144A532114480FF05EFF7868FFF704
:104EF000C5FF124B184613F068FB7B681B6823F054
:104F000002027B681A603B681B78002B06D07B6826
:104F10001B6823F001027B681A6005E07B681B6850
:104F200043F001027B681A6000BF0837BD4680BDB0
:104F3000B0C8010088CC01006CCC010017003C1007
:104F400080B483B000AF78600E4B03F580535A6D88
:104F50007B681A600B4B03F580539A6D7B685A602F
:104F6000084B03F58053DA6D7B689A60054B03F5B7
:104F700080531A6E7B68DA6000BF0C37BD465DF85F
:104F8000047B70470070044080B584B000AF786047
:104F90000623BB600023FB6009E00F4AFB6852F860
:104FA00023307A689A4207D0FB680133FB60FA68C5
:104FB000BB689A42F1D300E000BFFA68BB689A422E
:104FC00005D3064B064AA52106480FF0EDFEFB6807
:104FD00018461037BD4680BD94CC0100C4CC0100FA
:104FE00084CD0100E0CC010080B588B000AFF8604E
:104FF000B9607A60BB68002B05D19E4B9E4AD021D8
:105000009E480FF0D1FEBB681B68002B05D19C4B5E
:10501000994AD12199480FF0C7FEFB68994A9342FB
:1050200014D0FB68984A93420ED0FB68974A93428B
:1050300008D0FB68964A934201D1012307E04FF064
:10504000FF3304E0012302E0082300E00823BA68EC
:105050005279934205DA8F4B874AD32187480FF064
:10506000A3FEFB68874A934214D0FB68864A9342AA
:105070000ED0FB68854A934208D0FB68844A93426D
:1050800001D1012307E04FF0FF3304E0012302E0E8
:10509000082300E00823BA689279934205DA7E4B30
:1050A000754AD42175480FF07FFE0023FB8300234F
:1050B0007B770023BB61BB681B681B017A68B2FB6E
:1050C000F3F3FB83FB8B002B01D10123FB83002334
:1050D0007B617B685A00BB681B68B2FBF3F39AB232
:1050E000FB8B5B019BB2D31A7B827B685B00FA8BE4
:1050F00051017A8A0A44B3FBF2F37B61BB681B68F7
:105100007A699A4204D9BB681B687A69D31A03E0AA
:10511000BB681A687B69D31ABB61BB681B685F4AAE
:10512000A2FB03235A0913465B001344BA699A424F
:1051300002D940F2F53398E0F868FFF725FF0346FF
:10514000574A52F82330184613F059FAFB68DB78B7
:10515000DBB223F00C03DAB2FB68DA70FB681B7871
:10516000DBB223F01F03DAB2FB8B1B0A9BB2DBB26C
:105170001343DAB2FB681A70FB8BDAB2FB685A7021
:10518000FB689B7ADBB223F01F03DAB27B8ADBB2C7
:1051900003F01F03DBB21343DAB2FB689A72FB68B9
:1051A0009B78DBB223F017037B77BB685B7A9B00AD
:1051B000DBB203F00403DAB27B7F13437B77BB6877
:1051C0001B79002B07D0BB681A797B7F1343DBB2B6
:1051D00043F010037B77FB687A7F9A70BB685A793B
:1051E000FB68DA74BB689A79FB685A75FB681B7CAC
:1051F000DBB263F07703DAB2FB681A74FB685B7C9E
:10520000DBB263F03F03DAB2FB685A74BB68DB7948
:10521000002B07D0FB685B7BDBB243F00803DAB2FC
:10522000FB685A73BB681B7A002B07D0FB685B7B5B
:10523000DBB243F00103DAB2FB685A73FB68DB7838
:105240007B77BB689B7A002B03D07B7F43F00803FE
:105250007B77BB68DB7A002B03D07B7F43F00403B2
:105260007B77FB687A7FDA70002318462037BD46CB
:1052700080BD00BFB0C8010098CD0100E0CC0100A6
:10528000ECCC010000A0064000B0064000C0064083
:1052900000D0064004CD010044CD01001F85EB5134
:1052A000ACCC010080B582B000AF78607B68002B89
:1052B00006D1134B134A40F26F1113480FF074FDDF
:1052C0007B684FF4E1321A607B6800221A717B68B8
:1052D00000225A717B6801229A717B680022DA7180
:1052E0007B6800221A727B6800225A727B68002257
:1052F0009A727B680022DA7200BF0837BD4680BD13
:10530000B0C80100A4CD0100E0CC010080B483B09E
:1053100000AF786039603A68174B13403B607B6898
:105320001B78DAB23B68DBB21343DAB27B681A70DF
:105330007B68DB78DAB23B681B0ADBB21343DAB274
:105340007B68DA707B689B79DAB23B681B0CDBB256
:105350001343DAB27B689A717B685B7CDAB23B6894
:105360001B0EDBB21343DAB27B685A7400BF0C37F2
:10537000BD465DF8047B7047C0F00F0780B500AFF5
:10538000054B1B68054A9268114605489847BFF3CC
:105390004F8F00BF00BF80BD4C09002034090020A2
:1053A00000C0064080B500AF054B1B68054AD268B7
:1053B000114605489847BFF34F8F00BF00BF80BD1F
:1053C0004C0900203409002000D0064080B500AF11
:1053D000054B1B68054A1269114605489847BFF3FB
:1053E0004F8F00BF00BF80BD4C0900203409002052
:1053F00000A00E4080B500AF054B1B68054A5269FE
:10540000114605489847BFF34F8F00BF00BF80BDCE
:105410004C0900203409002000B00E4080B400AFD9
:10542000054B03F580531A46044B536400BFBD4639
:105430005DF8047B704700BF007004400000071354
:1054400080B483B000AF7860044A7B68136000BF0B
:105450000C37BD465DF8047B704700BF7008002024
:1054600080B483B000AF7860044A7B68136000BFEB
:105470000C37BD465DF8047B704700BF7408002000
:1054800080B582B000AF78600B46FB701B4813F00C
:105490007DF91B4B1B6903F48073002B09D17968DC
:1054A000174813F0A9F9164B1B69154A43F480738A
:1054B0001361FB78002B06D0114B1B69104A23F4B3
:1054C0000073136105E00E4B1B690D4A43F4007332
:1054D00013614FF40040FFF7C3FF094B5B6903F012
:1054E0000103002B03D0064B054A1B6813600348D9
:1054F00013F066F900BF0837BD4680BD1D003C10A3
:1055000000D0034080B483B000AF0346FB710B4B67
:105510001B78DBB223F03803DAB2FB79DB00DBB2B5
:1055200003F03803DBB205491343DBB20B7000BF55
:105530000C37BD465DF8047B704700BF0040064055
:1055400080B500AFFFF76AFF01210020FFF798FF49
:105550000E48FEF74BFA0E4B1846FFF771FF00237B
:105560001846FFF7CFFF00230A4A00211846FEF72E
:10557000DFFA0948FEF770F8084B094A1A60084933
:105580004FF4A020FEF782F800BF80BDD0CD01000F
:1055900000127A00C4CD0100C8CD0100E001002056
:1055A000000E270780B500AF314813F04BF93148A2
:1055B00013F048F9304813F045F9022201212F4831
:1055C00013F05AF9022202212C4813F055F9042253
:1055D00004212B4813F050F907220521284813F025
:1055E0004BF903220021274813F046F9254B1B688D
:1055F00023F0807323F00303224A43F00303136074
:10560000032201211F4813F037F91E4B5B6823F07A
:10561000807323F003031B4A43F00303536001220A
:105620000421184813F028F9164B1B6923F08073E6
:1056300023F00303134A43F00303136101220521FE
:10564000104813F019F90F4B5B690E4A23F0807371
:1056500023F0030353610C4B03F580531B690A4A83
:1056600023F0330302F58052136100BF80BD00BFF9
:10567000090038100B0038100D003810009004405D
:1056800000B0044000D004400070044080B485B0F5
:1056900000AF0346FB710023FB6015E00F49FA6879
:1056A00013465B0013445B000B441B78FA799A4263
:1056B00007D1FA6813465B0013445B00074A1344A2
:1056C00006E0FB680133FB60FB68242BE6D900236E
:1056D00018461437BD465DF8047B7047D8CD0100ED
:1056E00080B483B000AF0346FB71FB79042B17D85D
:1056F00001A252F823F000BF0D570000115700001F
:1057000015570000195700001D570000084B09E00D
:10571000084B07E0084B05E0084B03E0084B01E0AD
:1057200000BF084B18460C37BD465DF8047B704738
:10573000B8CE0100C0CE0100C8CE0100D4CE010019
:10574000E0CE0100E8CE0100B0B590B000AF034656
:10575000FB718E4B1B78062B00F20B8101A252F8D5
:1057600023F000BF815700008F570000C157000091
:1057700001580000F3570000295800006B58000042
:10578000012000F0CBFC814B01221A70FAE0804B23
:105790001B68184608F070F87E4B1B68184608F026
:1057A00093F804F0B9FC0346002B02D0774B042297
:1057B0001A70FB79002B00F0DE8000F0FBF8DAE0D5
:1057C000754B1B780133DAB2734B1A70724B1B782E
:1057D000322B07D9704B00221A706D4B1B6818468C
:1057E00008F09AF8FB79002B00F0C78000F0EEF883
:1057F000C3E0FB79002B00F0C28001F0D7FDBEE0D2
:10580000634B1B68184608F05FF8624B1B6818462C
:1058100008F05AF8FB79002B00F0B38001F076FC19
:105820005A4B04221A70ACE0022004F0E1FB03465C
:10583000012B16D102F0F0F8584B00221A7002F03A
:105840001DFC01F051FC002000F068FC07F0CCF8D2
:1058500003465B681946524814F06CF84B4B06221D
:105860001A700A200DF042F88CE001F09FFD03460B
:1058700083F00103DBB2002B13D002F0F3F90346EF
:10588000002B0ED04748FDF75BF807F0ADF8034654
:105890005B681946444814F04DF83C4B04221A70DA
:1058A0001AE001F083FD034683F00103DBB2002B15
:1058B00012D002F0D7F9034683F00103DBB2002BCC
:1058C0000AD002F0DBFB0021002000F05DFE022088
:1058D00000F03AFE01F008FC02F0AAF803461A466E
:1058E0002E4B1B789A4240D002F0A2F803461A468B
:1058F0002A4B1A704FF47A714FF47A7000F05AFB09
:105900002A4B07F108041D460FCD0FC40FCD0FC45D
:1059100095E8070003C4227007F1310300221A60E2
:105920005A601A720023FB631C4B1A7807F13C0380
:105930000421184614F0BCFB07F13C0207F10803F0
:105940003221184614F058FB07F10803184A322197
:10595000184614F051FB07F047F803465A6807F160
:1059600008031146184613F0E5FF0A200CF0BEFFAD
:1059700008E000BF06E000BF04E000BF02E000BF97
:1059800000E000BF00BF4037BD46B0BDD2350020AB
:10599000680800206C080020D3350020D435002092
:1059A000F4CE010024CF010040CF010074CF0100EC
:1059B00070CF010080B500AF04F08AFB024B0222D9
:1059C0001A7000BF80BD00BFD235002080B500AF87
:1059D000034B04221A7004F07BFB00BF80BD00BFA4
:1059E000D235002080B500AF1848FCF7A9FFFFF7BB
:1059F000E1FF0021012005F02BFF4FF4FA700CF0BD
:105A000075FF0021032005F023FF4FF4FA700CF01E
:105A10006DFF0021032005F01BFF4FF4FA700CF01E
:105A200065FF0021012005F013FF4FF4FA700CF020
:105A30005DFF0021112005F00BFFFFF7C7FF0448B1
:105A4000FCF77EFF0023184680BD00BFA8CF0100F1
:105A5000C4CF010080B500AF064B05221A7006F0D6
:105A6000C3FF03465B681946034813F063FF002336
:105A7000184680BDD2350020E4CF010080B582B049
:105A800000AF0346FB71FB79184612F05CFFFB790F
:105A9000072B49D801A252F823F000BFBD5A0000DD
:105AA000C95A0000D55A0000EB5A0000F35A000012
:105AB000055B0000295B0000175B00001D4B1B68A5
:105AC000184607F0D9FE30E01A4B1B68184607F05D
:105AD00023FF2AE001F02CFB174B1B68184607F048
:105AE0001BFF1648FCF72CFF1FE01548FCF728FFAA
:105AF0001BE0114B1B68184607F00EFF1148FCF71E
:105B00001FFF12E00C4B1B68184607F005FF0E48FC
:105B1000FCF716FF09E0084B1B68184607F0FCFE6F
:105B20000A48FCF70DFF00E000BF00BF0837BD4684
:105B300080BD00BF680800206C08002014D0010060
:105B400024D0010034D0010044D0010058D001001D
:105B500080B582B000AF786064200CF0C7FE0121F0
:105B6000044801F045F90020FFF7EEFD0A200CF093
:105B7000BDFEF4E77D5A000080B582B000AF7860CA
:105B80007B685B681A460F490F4814F007F97B6879
:105B90005B681A460D490E4814F000F97B685B6893
:105BA0001A460C490C4814F0F9F87B685B681A46F1
:105BB0000A490B4814F0F2F8002318460837BD468E
:105BC00080BD00BF6CD0010084D0010088D00100EE
:105BD000A4D00100B4D00100DCD00100E8D0010065
:105BE00008D1010080B582B000AF78607B685B6847
:105BF0001A461149114814F0E3F87B685B681A46AD
:105C00000F49104814F0DCF80F4B1B781846FFF7CB
:105C100067FD01467B685B681A460C4814F0D0F8B3
:105C20007B685B6819460A4813F084FE0023184617
:105C30000837BD4680BD00BF18D1010084D00100E7
:105C400030D101003CD10100D235002044D1010007
:105C5000D4DE010080B586B000AFF860B9607A602C
:105C60000023FB752649F86816F00BFC0346002B51
:105C700006D02449F86816F004FC0346002B07D12F
:105C8000BB6801221A707868FFF776FF034632E09E
:105C90001D49F86816F0F5FB0346002B06D01B499A
:105CA000F86816F0EEFB0346002B07D1BB68012213
:105CB0001A707868FFF796FF03461CE01449F868ED
:105CC00016F0DFFB0346002B06D1BB6801221A70D9
:105CD000FFF7C0FE03460EE00E49F86816F0D1FB50
:105CE0000346002B06D1BB6801221A70FFF77AFE2B
:105CF000034600E0FB7D18461837BD4680BD00BF57
:105D000060FC010050D1010070FC01005CD1010079
:105D100068D1010078D1010080B582B002AF0D4892
:105D20000CF072FAFDF798F80B4B00221A70002362
:105D3000019301230093002396220849084816F096
:105D400083F80346012B00D0FEE70CF065FE00BF90
:105D5000BD4680BD88D10100D2350020A0D1010010
:105D6000515B000080B582B000AF786039603B685D
:105D7000012B06D9074B084A4FF4FD7107480FF075
:105D800013F87B683A68043253F822301846083713
:105D9000BD4680BDA8D1010098D20100C4D1010048
:105DA00080B584B000AF7860164A00211648FDF730
:105DB000A5F902E001200CF099FD00211248FDF741
:105DC000DDF9034603F08003002BF3D000210E48D9
:105DD000FFF7C8FF0346FB81FB894FF47D7202FB8E
:105DE00003F30A4A82FB03121A44D213DB17D31AB5
:105DF000BB60BB689AB27B681A80002318461037D4
:105E0000BD4680BD5009002000B00B4001800080DD
:105E100080B58CB000AF78607B685B681A46194922
:105E2000194813F0CDFF00233B7407F10E03184609
:105E3000FFF7B6FF0346002B0FD1FB891A4607F187
:105E400010032021184609F0FFFB07F110030F4A49
:105E50002021184614F0D0F806E007F110030C4A90
:105E60002021184614F0C8F87B685A6807F110031F
:105E70001946084813F0A4FF002318463037BD46E2
:105E800080BD00BF00D2010014D201001CD201006D
:105E900024D201002CD2010080B582B000AF78601E
:105EA0007B685B681A460849084813F077FF7B68EF
:105EB0005B681A460649074813F070FF002318462E
:105EC0000837BD4680BD00BF38D2010014D20100A2
:105ED00054D20100A4D0010080B586B000AFF860B4
:105EE000B9607A600023FB751849F86816F0C9FAA2
:105EF0000346002B06D01649F86816F0C2FA03468E
:105F0000002B07D1BB6801221A707868FFF7C4FF25
:105F1000034616E00F49F86816F0B3FA0346002B63
:105F200006D00D49F86816F0ACFA0346002B07D1ED
:105F3000BB6801221A707868FFF76AFF034600E029
:105F4000FB7D18461837BD4680BD00BF60FC0100D0
:105F500078D2010070FC010088D2010080B584B0C5
:105F600000AF3B1D1846FDF797F800237B72032313
:105F70003B723B1D19460D48FDF700F800210B4808
:105F800012F0ECFC094812F093F80346002B00D005
:105F9000FEE7074B13221A60054B00221A71044BCF
:105FA00000225A7100BF1037BD4680BD00B00B40C3
:105FB0005009002090B587B002AF03460A46FB8027
:105FC0001346BB80FB88B3F57A7F01D91B236DE0B4
:105FD000FB88002B12D1374B1868BB884FF47A72BC
:105FE00002FB03F3344AA2FB03239A0964230093C0
:105FF000002304210DF0DAFDF86016E02D4B18683F
:10600000FB884FF47A7292FBF3F31A464FF47A73DB
:1060100002FB03F3284AA2FB03239A09642300939B
:10602000002304210DF0C2FDF860FB68012B01D0B4
:106030001B233BE0214B1868BB884FF47A7202FBAC
:1060400003F31D4AA2FB03239A0964230093002350
:1060500004210DF0ABFDF860FB68012B01D01B2380
:1060600024E0144B1C680CF0CBFD02466423009323
:106070000023012120460DF099FDF860FB68012BFB
:1060800001D01B2312E00D4B1C680CF0B9FD024639
:10609000642300930023012120460DF087FDF86062
:1060A000FB68012B01D01B2300E0002318461437A6
:1060B000BD4690BD58090020D34D62105C090020F8
:1060C00080B584B000AF78607B68FB60FB689A683D
:1060D000FB681B68DB0013441B6898B2FB689A6876
:1060E000FB681B68DB0013445B689BB21946FFF733
:1060F00061FFFB681B685A1CFB681A60FB681A6822
:10610000FB685B689A4202DB034B00221A6000BF07
:106110001037BD4680BD00BF6409002080B582B045
:1061200000AF0346FB71FB79042B01D9042317E070
:10613000FA790D4913465B0013449B000B4400227F
:106140001A60FA7913465B0013449B00064A134415
:10615000064A1360054B1B681846FFF7B1FF002382
:1061600018460837BD4680BD940100206409002010
:1061700080B582B000AF7860044B1B68184607F00A
:10618000A1F900BF0837BD4680BD00BF60090020EF
:1061900080B584B002AF78600A4B1868642300931E
:1061A0000023002203210DF001FD074B1B68002B8B
:1061B00004D0054B1B681846FFF782FF00BF083765
:1061C000BD4680BD580900206409002080B582B01A
:1061D00000AF78607B685B681A460F490F4813F080
:1061E000DDFD7B685B681A460D490E4813F0D6FD4D
:1061F0007B685B681A460C490C4813F0CFFD7B683E
:106200005B681A460A490B4813F0C8FD002318467C
:106210000837BD4680BD00BFC8D40100E4D40100EA
:10622000ECD40100A4D001000CD5010034D501004C
:1062300048D5010064D5010080B586B000AF786014
:106240007B685B681A461349134813F0B9FD07F1E0
:106250000803124A1021184613F0A9FE07F108039B
:1062600004221021184614F007F907F108030C4A1C
:106270001021184613F0C0FE7B685A6807F1080326
:106280001946084813F09CFD002318461837BD46F0
:1062900080BD00BF78D50100E4D4010088D501009D
:1062A000D4DE010090D5010080B588B000AFF86061
:1062B000B9607A604B49F86816F0E3F80346002BA2
:1062C00006D04949F86816F0DCF80346002B07D1E0
:1062D000BB6801221A707868FFF778FF03467DE0FB
:1062E0004249F86816F0CDF80346002B06D0404925
:1062F000F86816F0C6F80346002B07D1BB680122E8
:106300001A707868FFF798FF034667E00B22394957
:10631000F86816F0D0F80346002B2ED1BB68012296
:106320001A70FB680B33FB6107F11A0207F11C03BB
:106330001146184614F0B2F90346002B4DD107F16F
:10634000180207F11C031146184614F0A7F903467A
:10635000002B42D17B8B3A8B11461846FFF72AFE61
:106360000346002B07D07B689B681946224813F030
:10637000E1FA1B2332E0002330E011221F49F868C4
:1063800016F099F80346002B18D1BB6801221A7049
:10639000FB681133FB6107F1170207F11C0311467B
:1063A000184614F031F9FB7D042B05D8FB7D184607
:1063B000FFF7B4FE034611E01B230FE01049F86815
:1063C00016F05FF80346002B07D1BB6801221A7054
:1063D0000020FFF7A3FE034600E000231846203705
:1063E000BD4680BD60FC010098D5010070FC010035
:1063F000A4D50100B4D50100C0D50100DCD5010051
:10640000F0D5010080B588B002AF3B1D184606F0FC
:1064100057FF1A4BBB601A4BFB6003233B61002301
:106420003B7101237B713B1D184606F0ADFF03460F
:10643000144A1360144B00930023012201211348D6
:1064400015F05BFE0346124A1360114B1B68002BCC
:1064500000D1FEE70F4B00930023002201210E48DC
:1064600015F04BFE03460D4A13600C4B1B68002BC6
:1064700000D1FEE700BF1837BD4680BD80F00F4059
:1064800000B00440600900207161000004D60100E2
:10649000580900209161000010D601005C0900201D
:1064A00080B584B000AF264B1B68184615F0E9FA9A
:1064B0000346002B01D000233EE0224B1B78032B28
:1064C00039D1012004F0CEFCF860002004F0CAFCB1
:1064D000B860FB6813F1310F2BDBFB68312B28DC34
:1064E000BB6813F1310F24DBBB68312B21DC03F0D7
:1064F00023F80346FB80134BDB681AB2B7F906306A
:106500001146184612F046FA0346002B11D003F04C
:106510001FF80346FB800B4B1B691AB2B7F9063014
:106520001146184612F036FA0346002B01D001231B
:1065300002E0002300E0012318461037BD4680BD6D
:106540007C0900206809002080B586B000AF0346B2
:10655000FB7100233B73FB793B740A4B186807F10E
:106560000C0100234FF0FF3214F0C7FE0346012B4D
:1065700001D01B2302E00BF0EBFF00231846183775
:10658000BD4680BD7C09002080B586B000AF786034
:10659000396001233B737B683B613B687B610A4B3D
:1065A000186807F10C0100234FF0FF3214F0A5FE2C
:1065B0000346012B01D01B2302E00BF0C9FF00238F
:1065C00018461837BD4680BD7C09002080B586B0CE
:1065D00000AF7860396002233B737B683B613B68A6
:1065E0007B610A4B186807F10C0100234FF0FF3262
:1065F00014F083FE0346012B01D01B2302E00BF0B5
:10660000A7FF002318461837BD4680BD7C0900202F
:1066100080B483B000AF0346FB71FB79032B13D822
:1066200001A252F823F000BF396600003D66000069
:106630004166000045660000074B06E0074B04E09A
:10664000074B02E0074B00E0074B18460C37BD46EE
:106650005DF8047B704700BF1CD6010024D6010002
:106660002CD6010034D6010038D6010080B582B0A6
:1066700000AF78607B685B681A461949194813F0C7
:106680008DFB7B685B681A461749184813F086FB38
:106690007B685B681A461649164813F07FFB7B68D7
:1066A0005B681A461449154813F078FB7B685B68F1
:1066B0001A461349134813F071FB7B685B681A464E
:1066C0001149124813F06AFB7B685B681A4610494F
:1066D000104813F063FB00BF0837BD4680BD00BF04
:1066E00040D6010010D101005CD60100A4D0010009
:1066F0007CD60100A8D60100B8D60100E8D601007A
:1067000000D7010034D7010050D7010080D7010025
:1067100098D70100BCD7010080B588B000AF786081
:106720007B685B681A464C494C4813F049FB4C4B5C
:106730001B781846FFF76CFF01467B685B681A46BA
:10674000484813F03DFB7B685B681946464813F0E8
:10675000F1F8434B5A6807F108031821184608F06E
:1067600067FE07F10803414A1821184613F044FC5C
:106770007B685A6807F1080319463D4813F020FB6F
:10678000374B9A6807F108031821184608F050FEA5
:1067900007F10803354A1821184613F02DFC7B68D1
:1067A0005A6807F108031946324813F009FB2C4BCD
:1067B000DA6807F108031821184608F039FE07F1D6
:1067C00008032D4A1821184613F016FC02F0B4FEF7
:1067D00003461A4607F108031821184613F034FE41
:1067E00007F10803254A1821184613F005FC7B68B9
:1067F0005A6807F108031946214813F0E1FA184BCB
:106800001A6907F108031821184608F011FE07F16C
:106810000803194A1821184613F0EEFB02F098FEFF
:1068200003461A4607F108031821184613F00CFE18
:1068300007F10803114A1821184613F0DDFB7B68A5
:106840005A6807F1080319460E4813F0B9FA00BF59
:106850002037BD4680BD00BFC8D7010010D1010060
:10686000680900203CD10100D4DE0100D8D7010026
:10687000E8D70100F8D7010008D8010068D8010066
:1068800014D8010020D8010080B58AB000AFF860AC
:10689000B9607A60002387F82730B049F86815F0AE
:1068A000F0FD0346002B06D0AD49F86815F0E9FD70
:1068B0000346002B06D17868FFF7D8FEBB6801229B
:1068C0001A708BE1A749F86815F0DBFD0346002B31
:1068D00006D0A549F86815F0D4FD0346002B06D173
:1068E0007868FFF719FFBB6801221A7076E10C2265
:1068F0009E49F86815F0DFFD0346002B3CD1FB688C
:106900000C33BB6107F1140207F118031146184656
:1069100013F0CAFD0346002B24D107F1100207F142
:1069200018031146184613F0BFFD0346002B12D181
:106930007B693A6911461846FFF726FE0346002B8D
:1069400005D07B689B681946894812F0F3FFBB6845
:1069500001221A7042E17B689B681946844812F054
:10696000E9FF3BE17B689B681946824812F0E2FF31
:106970001B2387F8273031E10F227F49F86815F093
:106980009AFD0346002B44D1FB680F33BB6107F12E
:10699000140207F118031146184613F085FD03464B
:1069A000002B2CD107F1100207F1180311461846ED
:1069B00013F07AFD0346002B1AD1704B5A687B699D
:1069C00013443B626D4B9A683B691344FB61F96960
:1069D000386AFFF7D9FD0346002B05D07B689B681A
:1069E0001946634812F0A6FFBB6801221A70F5E051
:1069F0007B689B6819465E4812F09CFFEEE07B685E
:106A00009B6819465B4812F095FF1B2387F82730D7
:106A1000E4E00F225A49F86815F04DFD0346002BBB
:106A200016D1002002F068FD002002F075FD002163
:106A30000020FFF7CBFD0346002B05D07B689B6849
:106A400019464B4812F076FFBB6801221A70C5E068
:106A50000A224C49F86815F02EFD0346002B3CD164
:106A6000FB680A33BB6107F1140207F118031146F2
:106A7000184613F019FD0346002B24D107F110022C
:106A800007F118031146184613F00EFD0346002BBC
:106A900012D17B693A6911461846FFF797FD034604
:106AA000002B05D07B689B681946314812F042FFE5
:106AB000BB6801221A7091E07B689B6819462C48DC
:106AC00012F038FF8AE07B689B681946294812F06B
:106AD00031FF1B2387F8273080E00B222A49F86812
:106AE00015F0E9FC0346002B78D1FB680B33BB6142
:106AF000BB692649184615F0C4FC0346002B09D192
:106B00000020FFF721FD0346002B5AD01B2387F8F6
:106B1000273056E0BB691E49184615F0B2FC034603
:106B2000002B09D10120FFF70FFD0346002B48D0B1
:106B30001B2387F8273044E0BB691649184615F037
:106B4000A0FC0346002B27D10220FFF7FDFC0346E3
:106B5000002B36D01B2387F8273032E060FC010081
:106B60002CD8010070FC010038D8010048D8010081
:106B7000D0D5010058D801006CD801006809002068
:106B80007CD801008CD8010098D80100A4D801005D
:106B9000DCDF010090EC0100BB691349184615F0D9
:106BA00070FC0346002B09D10320FFF7CDFC034600
:106BB000002B06D01B2387F8273002E01B2387F821
:106BC000273097F82730002B05D07B689B68194643
:106BD000064812F0AFFEBB6801221A7097F8273002
:106BE00018462837BD4680BD70F00100D0D50100A1
:106BF00080B584B000AF194B1B6839460022184697
:106C000014F03AFDF860FB68002B01D10A2320E064
:106C10000BF062FC3B78002B05D102F095FB3A7932
:106C20000F4B1A7012E03B78012B06D17B680C4A9F
:106C30005360BB680A4A936008E03B78022B05D199
:106C40007B68074AD360BB68054A13610BF06AFC96
:106C5000002318461037BD4680BD00BF7C090020C8
:106C60006809002080B584B000AF78600BF0C8FFE1
:106C70000346FB6000BFFFF7BBFF0346002BFAD0C3
:106C800004F008F9264B1B78022B12D1012004F0E6
:106C9000E9F8234B5B680122194601F0EFFF002061
:106CA00004F0E0F81E4B9B680022194601F0E6FF55
:106CB0002EE01B4B1B78012B12D1012004F0D2F8DF
:106CC000034601220021184601F0D8FF002004F0FD
:106CD000C9F8034600220021184601F0CFFF17E053
:106CE0000F4B1B78032B13D102F026FC03461846EA
:106CF0000B4BDB680122194601F0A0FF02F028FCD3
:106D000003461846064B1B690022194601F096FF00
:106D100007F10C03052118460BF082FDAAE700BF1E
:106D20006809002080B582B002AF194B02221A70A8
:106D3000174B00225A60164B00229A60144B002217
:106D4000DA60134B00221A6100220C21042014F097
:106D500064FA03460F4A13600E4B1B68002B00D1E8
:106D6000FEE70C4B1B680C4918460BF0A1FC0023F6
:106D700001930323009300237D220749074815F060
:106D800063F80346012B00D0FEE700BFBD4680BD7F
:106D9000680900207C090020ACD80100656C000067
:106DA00080B485B000AF0346FB71EFF3108072B67C
:106DB000F873FB795B09D8B202460C4B53F82220DA
:106DC000FB7903F01F034FF0004121FA03F3014662
:106DD0001343064A42F82130F87B80F3108800BF45
:106DE0001437BD465DF8047B704700BF8009002062
:106DF00080B584B000AF78600B46FB70EFF3108075
:106E000072B6B8730023FB732BE0FB7B5B09DBB22C
:106E10001A461D4B53F82220FB7B03F01F034FF053
:106E2000004121FA03F31340002B17D0FB78002B0D
:106E30001BD0FB7B5B09D8B20246134B53F82220D0
:106E4000FB7B03F01F034FF0004121FA03F3DB4308
:106E5000014613400C4A42F8213006E0FB7B013327
:106E6000FB73FB7B082BD0D900E000BFB87B80F31D
:106E70001088FB7B092B03D0FA7B7B681046984770
:106E800000BF1037BD4680BD8009002080B483B0AC
:106E900000AF0023FB71FB79084A002142F8231060
:106EA000FB790133FB71FB79002BF4D000BF00BFED
:106EB0000C37BD465DF8047B704700BF8009002099
:106EC00080B586B000AF3B46184612F0BCFA0346C8
:106ED000FB74FB7C002B21D100237B611BE07A69D2
:106EE00013465B001344DB0008330F4A1A443B4649
:106EF0001146184612F0DEFA0346002B08D00A4964
:106F00007A6913465B001344DB000B441B7806E0F0
:106F10007B6901337B617B69242BE0D926231846EA
:106F20001837BD4680BD00BF64DA010080B485B06B
:106F300000AF0346FB710023FB6015E00F49FA68C0
:106F400013465B001344DB000B441B78FA799A422A
:106F500007D1FA6813465B001344DB00074A134469
:106F600006E0FB680133FB60FB68242BE6D90023B5
:106F700018461437BD465DF8047B704764DA01009B
:106F800080B500AF064B1B78272B05D1FFF798FF84
:106F900003461A46024B1A70014B1B78184680BDF7
:106FA0004802002080B58CB000AF78607B685B68D9
:106FB0001A461949194812F003FFFFF7E1FF03468B
:106FC0001846FFF7B3FFF862FB6A002B17D0FB6A85
:106FD0005A6807F10C032021184612F0E8FF07F168
:106FE0000C030F4A2021184613F006F87B685A68F4
:106FF00007F10C0319460B4812F0E2FE06E07B682D
:107000005B681A460849074812F0DAFE0023184662
:107010003037BD4680BD00BFDCDD0100F0DD010082
:10702000D4DE0100F4DD010000DE010080B584B093
:1070300000AFF860B9607A601D49F86815F021FA70
:107040000346002B06D01B49F86815F01AFA0346D0
:10705000002B12D17B685B681A461749174812F05B
:107060009DFE7B685B681A461549164812F096FE2D
:10707000BB6801221A70002316E01349F86815F066
:1070800000FA0346002B06D01049F86815F0F9F90C
:107090000346002B07D1BB6801221A707868FFF7FE
:1070A00081FF034600E0002318461037BD4680BD2F
:1070B00060FC01000CDE010014DE0100F0DD0100C7
:1070C00054D20100A4D0010070FC01002CDE0100AC
:1070D00080B400AF034B27221A7000BFBD465DF895
:1070E000047B70474802002080B582B002AF064B97
:1070F0001868002300930123012200210CF078FB83
:1071000000BFBD4680BD00BF8409002080B582B0AD
:1071100002AF064B186800230093012302220021CE
:107120000CF066FB00BFBD4680BD00BF8409002097
:1071300080B582B002AF00F039F90346002B09D0C8
:107140000A4B1868002300930123022200210CF04F
:107150004FFB08E0054B1868002300930123012230
:1071600000210CF045FB00BFBD4680BD8409002016
:1071700080B584B000AF03460A46FB711346BB716D
:1071800007F10B03184602F0D9FFFB79184602F00D
:107190002FFF0346FB73FB7B012B0DD02448FBF72D
:1071A000CFFBFB7B184602F0E9FE03461846FBF7CF
:1071B000C7FB2048FBF7C4FBFB7B012B12D107F177
:1071C0000B03184602F0BAFF0346BB8102F044FFEE
:1071D00003461A46BB79B88940F6AC5101F0B6FCBB
:1071E000012321E01448FBF7ABFBFB7B184602F0C0
:1071F000C5FE03461846FBF7A3FB0E48FBF7A0FBB2
:10720000002000F04DFF03460021184600F0DCFF8F
:10721000012000F045FF03460021184600F0D4FF8E
:1072200014200BF063FB002318461037BD4680BDC9
:1072300038DE0100D4DE01004CDE010080B582B0F2
:1072400000AF544B1B78DBB2042B00F29F8001A2ED
:1072500052F823F083730000697200008F720000FF
:10726000537300006773000001210220FFF780FFC5
:10727000034683F00103DBB2002B00F08480002181
:10728000112004F0E5FA434B02221A707DE000F071
:10729000E9FC0346002B35D03F4800F0CFFE034603
:1072A000FB71FB79112B1DD1FB790021184604F0ED
:1072B000CFFA0020FFF748F9364B04221A703748FE
:1072C000FBF73EFB0120FEF729FF00F0D7FE00216F
:1072D000112004F0BDFA0020FFF736F93048FBF723
:1072E0002FFB51E00021082004F0B2FAFB790021C5
:1072F000184604F0ADFA0020FFF726F9254B0122CD
:107300001A7042E00023BB7100237B71BA1D7B1D04
:107310001146184600F0D0FB0346002B15D1002083
:10732000FFF712F97B79002B0BD01A4B03221A704E
:1073300000F08AFC184B00221A700020FFF704F9B5
:1073400022E0144B01221A701EE0124B04221A7024
:107350001AE01448FBF7F4FA0320FEF7DFFE0D4BAA
:1073600004221A7010E01048FBF7EAFA0020FFF739
:10737000EBF80021112004F06BFA064B00221A7082
:1073800002E000BF02E000BF00E05AE700BF08379C
:10739000BD4680BDD6350020D735002064DE010013
:1073A0008CDE0100ACDE0100CCDE010080B400AF59
:1073B000064B1B78DBB2002B14BF01230023DBB28A
:1073C0001846BD465DF8047B704700BFD6350020E7
:1073D00080B483B000AF0346FB71FB79022B0AD067
:1073E000022B0ADC002B02D0012B02D005E0064B59
:1073F00004E0064B02E0064B00E0064B18460C3753
:10740000BD465DF8047B7047D8DE0100DCDE01007C
:10741000E4DE010038D6010080B586B000AF034637
:10742000FB7107F110031946002001F0B5FA03467D
:10743000FB75FB7D002B02D13B69002B01D11B2387
:1074400094E007F10C031946022001F0A5FA034667
:10745000FB75FB7D002B02D1FB68002B01D11B23A8
:1074600084E007F108031946032001F095FA03466A
:10747000FB75FB7D002B02D1BB68002B01D11B23C8
:1074800074E0FB79022B47D0022B66DC002B02D084
:10749000012B21D061E03B690F221A743B694FF444
:1074A0007A621A603B694FF4FA729A60B422AA2198
:1074B0004FF42A7004F0F8F8FB681E221A74FB6877
:1074C0004FF4FA621A60FA68BB6812681A60FA68C8
:1074D000BB68127C1A7442E03B691E221A743B6935
:1074E00041F27C521A603B69224ADA606422BE2172
:1074F0004FF42F7004F0D8F8FB6850221A74FB6820
:107500004FF4FA621A60FA68BB6812681A60FA6887
:10751000BB68127C1A7422E03B6928221A743B690A
:107520004FF4FA621A603B6947F23052DA60502237
:1075300096214FF42F7004F0B7F8FB6864221A7498
:10754000FB684FF4FA621A60FA68BB6812681A6046
:10755000FA68BB68127C1A7401E01B2306E0064A35
:10756000FB7913700548FBF7EBF900231846183731
:10757000BD4680BDA0860100D5350020ECDE0100AF
:1075800080B586B002AF78600020FFF745FF07F1B5
:107590000803012200920322002100200CF0AEF823
:1075A000F860FB68012B23D1BB6803F00103002BBB
:1075B00016D002F0B1FD0346002B08D001F0C4FE46
:1075C000134B01221A700020FEF7BEFF08E011489D
:1075D000FBF7B6F94FF4FA714FF4FA70FEF7EAFCD4
:1075E000BB6803F00203002B02D0094B04221A707F
:1075F000FFF724FEFFF7DAFE0346002B03D0052039
:107600000BF074F9C3E764200BF070F9BFE700BF1B
:10761000D63500200CDF010080B582B000AF786065
:107620007B685B681A460E490E4812F0B7FB7B6810
:107630005B681A460C490D4812F0B0FB7B685B682A
:107640001A460B490B4812F0A9FB7B685B681A4687
:1076500009490A4812F0A2FB00BF0837BD4680BDA9
:1076600024DF010048DF010050DF0100A4D0010049
:107670006CDF0100A0DF0100B0DF0100D4DF0100FA
:1076800080B58AB000AF78607B685B681A46334982
:10769000334812F095FB334B1B78DBB2042B35D803
:1076A00001A252F823F000BFBD760000CD760000A5
:1076B000ED760000FD760000DD7600007B685B68FB
:1076C0001A462949294812F07BFB27E07B685B6852
:1076D0001A462749254812F073FB1FE07B685B6858
:1076E0001A462449214812F06BFB17E07B685B685F
:1076F0001A4621491D4812F063FB0FE07B685B6866
:107700001A461E49194812F05BFB07E07B685B686C
:107710001A461B49154812F053FB00BF194B1B7842
:107720001846FFF755FE024607F1080320211846C8
:1077300012F03DFC07F10803134A2021184612F00D
:107740005BFC7B685A6807F1080319460F4812F082
:1077500037FB00BF2837BD4680BD00BFE4DF010016
:10776000FCDF0100D635002008E0010010E0010038
:1077700018E001002CE0010034E001003CE00100D1
:1077800000DE0100D5350020D4DE010048E0010014
:1077900080B586B000AFF860B9607A600023FB75F1
:1077A0003849F86814F06DFE0346002B06D03649C0
:1077B000F86814F066FE0346002B06D17868FFF7E0
:1077C0002BFFBB6801221A7057E03049F86814F0AB
:1077D00058FE0346002B06D02D49F86814F051FEE0
:1077E0000346002B06D17868FFF74AFFBB680122E9
:1077F0001A7042E02749F86814F043FE0346002B54
:1078000005D1FFF771FCBB6801221A7035E02249EF
:10781000F86814F036FE0346002B05D1FFF776FC1E
:10782000BB6801221A7028E01C49F86814F029FE90
:107830000346002B06D10020FFF7EEFDBB680122B6
:107840001A701AE01649F86814F01BFE0346002B64
:1078500006D10120FFF7E0FDBB6801221A700CE0A1
:107860001049F86814F00DFE0346002B05D10220E4
:10787000FFF7D2FDBB6801221A70FB7D184618374E
:10788000BD4680BD60FC010050E0010070FC0100BD
:107890005CE0010068E0010074E0010080E00100AC
:1078A00090E00100A4E0010080B582B002AF0A4B75
:1078B00000221A70094B01930223009300239622A1
:1078C0000749084814F0C0FA0346012B00D0FEE730
:1078D00000BFBD4680BD00BFD63500208409002012
:1078E000B4E001008175000080B584B000AF3B4674
:1078F0000621184602F040F90023FB7320E0FB7BD1
:107900005B0010333B4433F8103CFF2B15D9FB7B55
:107910005B0010333B4433F8102CFB7B0C4931F8EF
:1079200013309A4209D9FB7BFA7B5B0010333B444E
:1079300033F8101C064B23F81210FB7B0133FB734A
:10794000FB7B052BDBD900BF00BF1037BD4680BDD8
:107950008809002080B485B000AF00233B603B68FD
:107960007B607B68BB600023FB6015E01C4AFB6802
:1079700032F81330FF2B0CD9BB680133BB60FB68B6
:10798000022B03DC7B6801337B6002E03B68013340
:107990003B60FB680133FB60FB68052BE6DDBB68E1
:1079A000002B01D1002315E0BB68062B01D1042375
:1079B00010E00B4B1B88FF2B05D8094B5B89FF2B75
:1079C00001D8012306E0064B1B88FF2B01D90223B7
:1079D00000E0032318461437BD465DF8047B70476A
:1079E0008809002080B483B000AF00237B6007E0EB
:1079F000084A7B68002122F813107B6801337B6002
:107A00007B68052BF4DD00BF00BF0C37BD465DF879
:107A1000047B70478809002080B400AF034B00222C
:107A20001A7000BFBD465DF8047B7047DA35002050
:107A300080B400AF034B1B781846BD465DF8047B4D
:107A4000704700BFDA35002080B400AF034B1B78CD
:107A50001846BD465DF8047B704700BF4902002010
:107A600080B586B000AF0346FB710023FB75114A59
:107A7000FB79137000F06AFF38613B69002B13D06B
:107A80003B695A780B4B1B789A420DD000F05EFF91
:107A9000024607F10C0312881A8007F10C031846FE
:107AA00000F044FF0346FB75FB7D18461837BD46C2
:107AB00080BD00BF4902002080B584B000AF78606F
:107AC00039607B6800221A703B6800221A7002201D
:107AD00002F08EFA0346BB73BB7B002B02D104235A
:107AE000FB7318E0FFF77EFFFFF7FEFE304908202A
:107AF00003F0AEFEFFF72EFF03467B73022002F079
:107B000077FA0346BB73BA7B7B7B1146184610F0AD
:107B100081FF0346FB73FB7B0E2B0AD17B6801229E
:107B20001A702448FAF70CFF0320FEF7F7FA002337
:107B30003AE0FB7B062B0DD13B681B78002B09D06C
:107B4000042000F09BF800F0B9F81B48FAF7F8FEA3
:107B5000002329E0FB7B062B0AD1FB7B184600F0B3
:107B60008DF800F0ABF81548FAF7EAFE00231BE0A9
:107B7000FB7B112B06D1FFF7C9FA1148FAF7E0FE9B
:107B80001B2311E0FB7B0021184603F061FE0D4B27
:107B90001B780133DAB20B4B1A70FB7B184600F0EE
:107BA0006DF800F08BF8002318461037BD4680BDF5
:107BB000D9890100BCE00100D4E00100ECE0010043
:107BC00004E10100DA35002080B584B000AF1C4B21
:107BD0001B78002B2FD01A4B1B78013BBB60002376
:107BE000FB6023E0174AFB6813441B78FB71154ABE
:107BF000BB6813441B78184610F0F5FE034619467F
:107C0000104AFB6813440A461A70FB79184610F0B4
:107C1000EAFE034619460B4ABB6813440A461A702B
:107C2000FB680133FB60BB68013BBB60FA68BB6863
:107C30009A42D7DD00E000BF1037BD4680BD00BFCF
:107C4000D83500209409002080B500AF044B0122F4
:107C50001A70FFF7B9FF112000F010F800BF80BDC7
:107C6000D935002080B400AF034B1B781846BD46C1
:107C70005DF8047B704700BFD935002080B483B025
:107C800000AF0346FB710B4B1B783F2B0BD8094B06
:107C90001B781946084AFB795354064B1B7801336D
:107CA000DAB2044B1A7000BF0C37BD465DF8047B96
:107CB000704700BFD83500209409002080B483B0FD
:107CC00000AF474B1B78022B40F28180444B1B785E
:107CD000023B444AD35C052B06D0414B1B78023B48
:107CE000404AD35C042B74D10023FB800123BB806A
:107CF0002BE03B4B1B781A46BB88D31A394AD35C1E
:107D0000013B042B1DD801A252F823F0217D000075
:107D1000437D00002B7D0000337D00003B7D000093
:107D2000FB8803F58773FB800CE0FB885A33FB80EC
:107D300008E0FB88B433FB8004E0FB88B433FB80AD
:107D400000E000BFBB880133BB80BB88032BD0D9C8
:107D5000FB88DA082449A1FB021292084FF4B4719F
:107D600001FB02F29B1AFB80FB88B3F5877F20D0D2
:107D7000B3F5877F24DCB42B14D0B42B20DC002B8C
:107D800002D05A2B07D01BE0154B1B78033B154A3A
:107D90000621D15414E0124B1B78033B114A0321F6
:107DA000D1540DE00E4B1B78033B0E4A0421D154F5
:107DB00006E00B4B1B78033B0A4A0121D15400BF5C
:107DC000074B1B78023BDAB2054B1A7002E000BF8A
:107DD00000E000BF0C37BD465DF8047B704700BF74
:107DE000D835002094090020176CC11680B582B0E8
:107DF00000AF78607B685B681A460E490E4811F048
:107E0000CDFF7B685B681A460C490D4811F0C6FF30
:107E10007B685B681A460B490B4811F0BFFF7B6813
:107E20005B681A4609490A4811F0B8FF00BF0837D5
:107E3000BD4680BD20E1010044E101004CE10100AC
:107E4000A4D0010068E1010084E101008CE101009F
:107E5000B4E1010080B584B000AF78607B685B68F6
:107E60001A462F492F4811F0ABFFFFF7EDFD0346EF
:107E7000002B01D02C4900E02C497B685B681A4636
:107E80002B4811F09DFFFFF7EDFE0346002B01D0BC
:107E9000284900E028497B685B681A46274811F0AA
:107EA0008FFF7B685B681A462549264811F088FFDA
:107EB000254B1A787B685B681946104611F069FDFE
:107EC0007B685B681946214811F034FD0023FB6094
:107ED00016E01F4AFB6813441B78184603F000FCA9
:107EE00002467B685B681946104611F023FD7B68EB
:107EF0005B681946174811F01DFDFB680133FB60F4
:107F0000114B1B781A46FB689342E2DB7B685B6887
:107F10001946114811F00EFD00BF1037BD4680BD57
:107F2000C8E1010044E10100E0E10100F8E10100E5
:107F300014E201001CE2010024E201002CE2010035
:107F400038E201003CE20100D835002044E20100A3
:107F500094090020F8FB0100D4DE010080B586B052
:107F600000AFF860B9607A600023FB752B49F868B0
:107F700014F087FA0346002B06D02949F86814F05C
:107F800080FA0346002B06D17868FFF72FFFBB6805
:107F900001221A703CE02349F86814F072FA034693
:107FA000002B06D02049F86814F06BFA0346002B2A
:107FB00006D17868FFF74EFFBB6801221A7027E0F0
:107FC0001A49F86814F05DFA0346002B05D100F059
:107FD00055F8BB6801221A701AE01549F86814F0C8
:107FE00050FA0346002B06D1124B01221A70BB68CF
:107FF00001221A700CE01049F86814F042FA0346A6
:10800000002B05D10B4B00221A70BB6801221A709D
:10801000FB7D18461837BD4680BD00BF60FC0100DF
:1080200048E2010070FC010054E2010060E201003E
:108030006CE20100490200207CE2010080B483B0C0
:1080400000AF78607B681A780A4B1B789A4209D295
:108050007B681B785A1CD1B27A6811701A46064B9D
:108060009B5C00E0112318460C37BD465DF8047B8D
:10807000704700BFD83500209409002080B400AFBD
:10808000054B00221A70054B00221A7000BFBD4636
:108090005DF8047B704700BFD9350020D83500203B
:1080A00080B483B000AF0346FB71FB79002B01D194
:1080B000044B00E0044B18460C37BD465DF8047BCA
:1080C000704700BFD4090020E009002080B582B0CD
:1080D00000AF0346FB80FB88DB43FB80FA88084B3C
:1080E000A3FB0213D21A520813445B0AFB80FB88DD
:1080F000DBB2184603F020F900BF0837BD4680BD4B
:10810000EB47389080B582B000AF0346FB80FB8818
:10811000DB43FB80FA88084BA3FB0213D21A5208F8
:1081200013445B0AFB80FB88DBB2184603F01CF9A2
:1081300000BF0837BD4680BDEB47389080B582B0A0
:1081400000AF0346FB71054B1B68FA7911461846D0
:1081500005F0DEF900BF0837BD4680BDEC09002000
:1081600080B582B000AF0346FB71054B1B68FA79FE
:108170001146184605F0CCF900BF0837BD4680BD52
:10818000F009002080B582B000AF78600B467B809C
:108190000C4B1B78002B08D07B687A885A807B6850
:1081A0005B687A881046984708E07B684FF6FF7254
:1081B0005A807B685B684FF6FF70984700BF0837AE
:1081C000BD4680BD4A02002080B584B000AF786013
:1081D0000B46FB7097F90330642B02DD6423FB70C0
:1081E00006E097F9033013F1640F01DA9C23FB706A
:1081F0007B68FA785A7097F90330002B08DA01216E
:10820000786810F0A6FCFB785B42DBB2FB7003E001
:108210000021786810F09DFC97F90330C3F16402E7
:1082200013461B049B1A084A82FB03125211DB17E8
:10823000D31AFB60FB689BB219467868FFF7A2FF70
:1082400000BF1037BD4680BD1F85EB5180B483B0A1
:1082500000AF78600B46FB707B685B88C3F57F439B
:10826000FF33642202FB03F30D4A82FB03121A441C
:10827000D213DB17D31A5AB27B685A70FB78012BE2
:1082800008D17B6893F90130DBB25B42DBB25AB2B2
:108290007B685A7000BF0C37BD465DF8047B7047A1
:1082A0000180008080B582B000AF78607B685B6839
:1082B0001A461249124811F071FD7B685B681A4634
:1082C0001049114811F06AFD7B685B681A460F4936
:1082D0000F4811F063FD7B685B681A460D490E4834
:1082E00011F05CFD7B685B681A460C490C4811F084
:1082F00055FD00BF0837BD4680BD00BF8CE20100C0
:10830000A8E20100B0E20100A4D00100D0E2010027
:10831000ECE20100F8E2010014E3010030E30100A7
:1083200054E3010080B58CB002AF78607B685B6875
:108330001A465E495E4811F043FD0020FFF7B0FE8B
:1083400003461B78002B01D05A4900E05A497B684C
:108350005B681A46594811F033FD0120FFF7A0FE73
:1083600003461B78002B01D0524900E052497B683C
:108370005B681A46524811F023FD524B1B78002BC4
:1083800001D0514900E051497B685B681A4650486A
:1083900011F016FD7B685B681A464E494E4811F095
:1083A0000FFD00233B724D4B93F901301AB207F1D8
:1083B0000800042300932023202111F0E3FE07F19D
:1083C0000803474A2021184611F016FE434810F0D2
:1083D000A5FB03461A4607F108032021184611F0B1
:1083E000C6FF3E4810F0F1FB0346002B01D13D4A89
:1083F00000E03D4A07F108032021184611F0FCFD7A
:108400007B685A6807F108031146184611F092FA82
:108410007B685B681946354811F08CFA7B685B68AD
:108420001A462C49324811F0CBFC00233B72314BE9
:1084300093F901301AB207F10800042300932023B6
:10844000202111F09FFE07F10803254A202118463C
:1084500011F0D2FD274810F061FB03461A4607F1E0
:1084600008032021184611F082FF224810F0ADFBCE
:108470000346002B01D11B4A00E01B4A07F1080309
:108480002021184611F0B8FD7B685A6807F10803EF
:108490001146184611F04EFA7B685B68194613487E
:1084A00011F048FA00BF2837BD4680BD6CE30100DB
:1084B0007CE301001CE2010024E2010084E30100EE
:1084C00094E301004A0200200CE3010040FD01009A
:1084D000A4E301003CCF0100B0E30100D409002077
:1084E000BCE30100C4E30100CCE30100D4DE0100E1
:1084F000D4E30100E009002080B588B000AFF86047
:10850000B9607A600023FB778749F86813F0B9FFF8
:108510000346002B06D08549F86813F0B2FF0346E6
:10852000002B06D17868FFF7BDFEBB6801221A70E8
:10853000F5E07F49F86813F0A4FF0346002B06D04E
:108540007C49F86813F09DFF0346002B06D178683C
:10855000FFF7E8FEBB6801221A70E0E07649F86890
:1085600013F08FFF0346002B07D10021734810F052
:10857000F0FABB6801221A70D1E07149F86813F073
:1085800080FF0346002B07D100216E4810F0E1FA6E
:10859000BB6801221A70C2E06B49F86813F071FFE2
:1085A0000346002B07D10121644810F0D2FABB68C2
:1085B00001221A70B3E06549F86813F062FF0346C0
:1085C000002B07D101215F4810F0C3FABB680122DC
:1085D0001A70A4E00D225E49F86813F06CFF0346A0
:1085E000002B37D15B4B1B7883F00103DBB2002BF0
:1085F00008D07B689B681946574811F09BF91B23EC
:10860000FB778CE0FB680D337B6107F1180207F103
:1086100014031146184611F047FF0346002B10D1F2
:10862000BB6913F1640F0CDBBB69642B09DCBB690C
:108630005BB219464148FFF7C7FDBB6801221A70BB
:108640006DE07B689B681946444811F073F91B2361
:10865000FB7764E00D224249F86813F02CFF0346D3
:10866000002B37D13B4B1B7883F00103DBB2002B8F
:1086700008D07B689B681946374811F05BF91B23CB
:10868000FB774CE0FB680D337B6107F1180207F1C3
:1086900014031146184611F007FF0346002B10D1B2
:1086A000BB6913F1640F0CDBBB69642B09DCBB698C
:1086B0005BB219462348FFF787FDBB6801221A7099
:1086C0002DE07B689B681946244811F033F91B2381
:1086D000FB7724E008222349F86813F0ECFE0346F8
:1086E000002B06D11B4B01221A70BB6801221A70A5
:1086F00015E009221C49F86813F0DDFE0346002B43
:108700000DD100210D48FFF75FFD00210D48FFF757
:108710005BFD104B00221A70BB6801221A70FB7FB0
:1087200018462037BD4680BD60FC0100E0E3010033
:1087300070FC0100ECE30100FCE30100D40900201F
:108740000CE40100E00900201CE4010030E4010019
:1087500044E401004A02002054E4010078E40100EE
:10876000ACE40100BCE40100C8E4010080B586B0BF
:1087700000AF3B1D184604F0A3FD0F4BBB600F4B31
:10878000FB6009233B6100233B7101237B713B1D8F
:10879000184604F0F9FD0346094A136008233B61BB
:1087A0003B1D184604F0F0FD0346064A136000BF67
:1087B0001837BD4680BD00BF80F00F4000B00440B8
:1087C000EC090020F009002080B500AFFFF7CEFFD4
:1087D0000E4B00221A700E4B00221A700B4B0D4AE2
:1087E0009A600B4B0C4A9A60084B0C4A5A60084B33
:1087F0000B4A5A6000210548FFF7E6FC00210448B7
:10880000FFF7E2FC02F0C8FD00BF80BDD4090020E4
:10881000E00900203D81000061810000CD80000062
:108820000581000080B588B000AFF860B9607A605B
:108830000023FB610BE0FB699B0003F180531A6886
:108840002349FB6941F82320FB690133FB61FB6984
:10885000B3F5806FEFD31F4BDA681F4B4FF0805199
:108860001C48FBF78DFA38613B69002B01D01B23B4
:108870002AE0FB6803F17043154A1344BB61BB68EF
:108880007B610023FB610CE07B691A78BB691A707D
:10889000BB690133BB617B6901337B61FB690133D8
:1088A000FB61FA697B689A42EED34FF48053084A21
:1088B0004FF080510748FBF7CDFA38613B69002B38
:1088C00001D01B2300E0002318462037BD4680BDA1
:1088D000280A0020F40900206B66656B80B582B021
:1088E00000AF78600B467B807B88202B01D9042366
:1088F00006E07B881A4679680348FFF793FF034632
:1089000018460837BD4680BD0200001080B500AF94
:108910002021054810F06BF90346002B01D00023FD
:1089200000E0014B184680BD0200001080B582B007
:1089300000AF7860022279680348FFF773FF0346AF
:1089400018460837BD4680BD2600001080B500AF30
:108950000221054810F04BF90346002B01D00023FB
:1089600000E0014B184680BD2600001080B582B0A3
:1089700000AF34220021074813F0A2FC0548FBF7A2
:1089800093F978607B68002B00D0FEE700BF0837C2
:10899000BD4680BDF409002080B483B000AF03461B
:1089A0003960FB71FB79052B22D801A252F823F024
:1089B000C9890000F1890000D1890000D98900002F
:1089C000E1890000E98900003B680F4A1A6014E061
:1089D0003B680E4A1A6010E03B680D4A1A600CE0D2
:1089E0003B680C4A1A6008E03B680B4A1A6004E0D6
:1089F0003B6800221A601B2300E0002318460C3756
:108A0000BD465DF8047B7047281A0020441A0020F8
:108A1000601A00207C1A0020981A002080B489B0C7
:108A200000AFF860B9607A60BA68FB68D31AFB617E
:108A30007B681B68FA6902FB03F3324A82FB03126C
:108A40005211DB17D31ABB617B689A69FB691A4420
:108A50007B689A617B689A697B68DB689A4204DD6F
:108A60007B68DA687B689A610BE07B689A697B684F
:108A7000DB685B429A4204DA7B68DB685A427B68B7
:108A80009A614FF6FF737B617B689B697A699A42B2
:108A900003DA7B687A699A6109E07B689A697B6985
:108AA0005B429A4203DA7B695A427B689A617B682F
:108AB0009B697A68526802FB03F3124A82FB031235
:108AC0005211DB17D31ABA691344BB617B685B6927
:108AD000FA69D31A7A68926802FB03F3094A82FBA7
:108AE00003125211DB17D31ABA691344BB617B68B6
:108AF000FA695A61BB6918462437BD465DF8047BA4
:108B0000704700BF1F85EB5180B483B000AF786021
:108B10007B68002B02DA7B685B427B607B680A4AD9
:108B200082FB03121A445211DB17D31A7B607B6855
:108B3000642B01DD64237B607B68DBB218460C3755
:108B4000BD465DF8047B7047EBA00EEA90B585B09A
:108B500002AF0446084611461A462346FB800346E8
:108B6000BB800B467B8013467B707B787A88B98804
:108B7000F888044C009410F085F800BF0C37BD460F
:108B800090BD00BF281A002080B588B000AFF86003
:108B9000B9603B601346FB710023FB763A68B96805
:108BA000F868FFF73BFFF861FB694FF47A7202FB4C
:108BB00003F3FB61FB69002B02DB0023FB7604E07F
:108BC000FB695B42FB610123FB76FB69B3F5803FE8
:108BD00002DB4FF6FF73FB613B681B7C1A46FB69A7
:108BE00002FB03F3144A82FB03125211DB17D31A60
:108BF000FB61FB79002B04D00020FFF751FA78616C
:108C000003E00120FFF74CFA7861FB699BB2DB437C
:108C10009BB219467869FFF7B5FAFB7E1946786969
:108C20000FF097FFFB7E19467869FFF70FFB00BF37
:108C30002037BD4680BD00BF1F85EB5180B584B095
:108C400000AFF860B9601346FB71FB79002B06D0CA
:108C5000FA79084BB968F868FFF796FF05E0FA79EA
:108C6000054BB968F868FFF78FFF00BF1037BD46A6
:108C700080BD00BF441A0020601A002080B584B077
:108C800000AFF860B9601346FB71FB79002B06D08A
:108C9000FA79084BB968F86810F024F905E0FA7918
:108CA000054BB968F86810F01DF900BF1037BD46D4
:108CB00080BD00BF7C1A0020981A002080B582B0C9
:108CC00000AF78607B685B681A461C491C4811F04D
:108CD00065F87B685B681A461A491B4811F05EF814
:108CE0007B685B681A461949194811F057F87B6888
:108CF0005B681A461749184811F050F87B685B68A2
:108D00001A461249154811F049F87B685B681A4603
:108D10001049134811F042F87B685B681A46114904
:108D2000114811F03BF87B685B681A4609490F4807
:108D300011F034F800BF0837BD4680BDD4E401000F
:108D4000ECE40100F0E40100A4D001000CE5010016
:108D50003CE5010054E501006CE5010080E50100FF
:108D6000A0E50100BCE50100E8E5010000E6010026
:108D700080B594B000AFF860B9607A6007F1100375
:108D8000834A3021184611F012F907F11003BA682E
:108D90003021184611F030F907F110037D4A3021D7
:108DA000184611F029F907F120037B4A30211846B3
:108DB00011F0FDF8FB681A6807F12003302118460E
:108DC00011F042FB07F12003744A3021184611F0DC
:108DD00013F9FB685A6807F120033021184611F097
:108DE00033FB07F120036E4A3021184611F004F9D5
:108DF000FB689A6807F120033021184611F024FB24
:108E000007F12003674A3021184611F0F5F87B6816
:108E10005A6807F1200107F11003184610F0D0FF3F
:108E200007F110035A4A3021184611F0C0F807F133
:108E30001003BA683021184611F0DEF807F110036C
:108E4000594A3021184611F0D7F8FB68DA6807F163
:108E500020033021184606F0EBFA07F12003514AAF
:108E60003021184611F0C8F87B685A6807F12001D4
:108E700007F11003184610F0A3FF07F11003444A4E
:108E80003021184611F093F807F11003BA68302129
:108E9000184611F0B1F807F11003444A3021184682
:108EA00011F0AAF8FB685A6907F12003302118462F
:108EB00006F0BEFA07F120033A4A3021184611F0B5
:108EC0009BF87B685A6807F1200107F110031846E8
:108ED00010F076FF07F110032D4A3021184611F0EB
:108EE00066F807F11003BA683021184611F084F8CB
:108EF00007F110032E4A3021184611F07DF8FB6867
:108F00009A6907F120033021184606F091FA07F11B
:108F10002003244A3021184611F06EF87B685A6805
:108F200007F1200107F11003184610F049FF07F17F
:108F30001003174A3021184611F039F807F11003D1
:108F4000BA683021184611F057F807F11003194A92
:108F50003021184611F050F8FB681A7C07F1200305
:108F60003021184611F0A4F807F12003124A3021ED
:108F7000184611F041F87B685A6807F1200107F1A3
:108F80001003184610F01CFF00BF5037BD4680BDCF
:108F900014E6010018E6010060DE010020E6010091
:108FA00028E60100D4DE010030E6010038E60100C9
:108FB00040E601004CE6010054E6010080B582B0B5
:108FC00000AF78607B685B681A461049104810F063
:108FD000F7FE7A680F491048FFF7CAFE7A680F4912
:108FE0000F48FFF7C5FE7A680E490F48FFF7C0FE2D
:108FF0007A680E490E48FFF7BBFE7A680D490E48A5
:10900000FFF7B6FE00BF0837BD4680BD58E6010039
:10901000ECE4010074E60100281A002078E6010063
:10902000441A002080E60100601A002088E6010052
:109030007C1A002090E60100981A002080B588B0C4
:1090400000AFF860B9607A603B600023FB770222D2
:109050006349B86813F02FFA0346002B1ED1BB6892
:109060000233BB6107F1140207F1180311461846D9
:1090700011F05FFB0346002B07D17B691A46FB68A2
:109080001A607B6801221A70A5E03B689B6819464C
:10909000544810F04FFC1B23FB779CE002225249FE
:1090A000B86813F008FA0346002B1ED1BB680233E0
:1090B000BB6107F1140207F118031146184611F0BD
:1090C00038FB0346002B07D17B691A46FB685A60C0
:1090D0007B6801221A707EE03B689B681946414814
:1090E00010F028FC1B23FB7775E002223F49B8688B
:1090F00013F0E1F90346002B1ED1BB680233BB61BC
:1091000007F1140207F118031146184611F011FB7C
:109110000346002B07D17B691A46FB689A607B687F
:1091200001221A7057E03B689B6819462D4810F0E1
:1091300001FC1B23FB774EE002222D49B86813F097
:10914000BAF90346002B1ED1BB680233BB6107F19D
:10915000140207F118031146184611F0EAFA034603
:10916000002B07D17B691A46FB68DA607B68012215
:109170001A7030E03B689B6819461A4810F0DAFB19
:109180001B23FB7727E006221A49B86813F093F9EE
:109190000346002B1FD1BB680633BB6107F11302E6
:1091A00007F118031146184611F02EFA0346002B5A
:1091B00009D1FB7C642B06D8FA7CFB681A747B68A7
:1091C00001221A7007E03B689B681946054810F0B9
:1091D000B1FB1B23FB77FB7F18462037BD4680BDC4
:1091E00098E601009CE60100B0E60100BCE6010043
:1091F000B4E60100B8E6010080B586B000AFF860C3
:10920000B9607A600023FB754249F86813F039F9B8
:109210000346002B06D04049F86813F032F90346A4
:10922000002B06D17868FFF749FDBB6801221A7050
:109230006BE03A49F86813F024F90346002B06D096
:109240003749F86813F01DF90346002B06D17868FA
:10925000FFF7B4FEBB6801221A7056E007223149BD
:10926000F86813F028F90346002B09D1FB68D91DD3
:109270007B68BA682C48FFF7E1FE0346FB7544E0C3
:1092800008222A49F86813F016F90346002B17D173
:10929000FB6803F108017B68BA682548FFF7CEFE3A
:1092A0000346FB75FB7D002B2FD1FB6803F1080102
:1092B0007B68BA681F48FFF7C1FE0346FB7524E0D0
:1092C0000C221D49F86813F0F6F80346002B0AD16A
:1092D000FB6803F10C017B68BA681848FFF7AEFE23
:1092E0000346FB7511E00C221549F86813F0E3F80A
:1092F0000346002B09D1FB6803F10C017B68BA68B7
:109300001048FFF79BFE0346FB75FB7D1846183798
:10931000BD4680BD60FC0100C0E6010070FC01009C
:10932000CCE60100D8E60100281A0020E0E60100A2
:10933000441A0020601A0020ECE601007C1A00208C
:10934000FCE60100981A002080B400AF114B002207
:109350005A61104B00229A610F4B00225A610E4B4A
:1093600000229A610D4B00225A610C4B00229A6137
:109370000B4B00225A610A4B00229A61094B0022D2
:109380005A61084B00229A6100BFBD465DF8047B1C
:10939000704700BF281A0020441A0020601A0020DD
:1093A0007C1A0020981A002080B400AF3F4B4FF485
:1093B0007A621A603D4B0F225A603C4B4FF4FA72AE
:1093C0009A603A4B3A4ADA60384B19221A74374B92
:1093D00000225A61354B00229A61364B4FF4FA62F3
:1093E0001A60344B02225A60324B32229A60314B5F
:1093F000C822DA602F4B23221A742E4B00225A61A6
:109400002C4B00229A612B4B1B682B4A1360294B73
:109410005B68294A5360274B9B68274A9360254B1A
:10942000DB68254AD360234B1A7C234B1A74214BEB
:109430005B69214A53611F4B9B691F4A93611F4B14
:109440004FF4FA621A601D4B50225A601B4B0022E7
:109450009A601A4B1A4ADA60184B32221A74174B68
:1094600000225A61154B00229A61144B1B68154A61
:109470001360124B5B68134A5360104B9B68114A90
:1094800093600E4BDB680F4AD3600C4B1A7C0D4B7C
:109490001A740A4B5B690B4A5361084B9B69094A72
:1094A000936100BFBD465DF8047B7047281A002019
:1094B000A0860100441A0020601A00207C1A0020B7
:1094C000C0D40100981A002080B400AF034B1B6881
:1094D0001846BD465DF8047B704700BFCC1A0020DB
:1094E00080B400AF034B1B681846BD465DF8047B93
:1094F000704700BFD01A002080B483B000AF7860FE
:10950000044A7B68136000BF0C37BD465DF8047BDE
:10951000704700BFC41A002080B483B000AF7860E9
:10952000044A7B68136000BF0C37BD465DF8047BBE
:10953000704700BFC81A002080B400AF034B1B68FF
:109540001846BD465DF8047B704700BFC41A002072
:1095500080B400AF034B1B681846BD465DF8047B22
:10956000704700BFC81A002080B483B000AF034624
:10957000FB71044AFB79137000BF0C37BD465DF8E0
:10958000047B7047DB35002080B483B000AF034616
:10959000FB71044AFB79137000BF0C37BD465DF8C0
:1095A000047B7047DC35002098B500AF184B1B7862
:1095B000002B15D0174B1B68184610F0A0F8034677
:1095C000002B01D0022400E00024134B1B68184636
:1095D00010F095F803465BB223435BB2DBB214E0B4
:1095E0000D4B1B68184610F08AF80346002B01D07B
:1095F000022400E00024074B1B68184610F07FF897
:1096000003465BB223435BB2DBB2184698BD00BF92
:10961000DB350020B81A0020B41A002098B500AF3E
:10962000184B1B78002B15D0174B1B68184610F0F1
:1096300066F80346002B01D0022400E00024134BFF
:109640001B68184610F05BF803465BB223435BB21D
:10965000DBB214E00D4B1B68184610F050F80346BF
:10966000002B01D0022400E00024074B1B681846A1
:1096700010F045F803465BB223435BB2DBB21846F9
:1096800098BD00BFDC350020C01A0020BC1A0020A5
:1096900080B582B000AFFFF787FF0346FB71264B12
:1096A0001B781A46FB79254992000A4413441B781B
:1096B000BB71214AFB79137097F90630032B05D152
:1096C0001F4B1B6801331E4A13600AE097F90630EE
:1096D000002B06D097F906201A4B1B681344194A31
:1096E0001360FFF79BFF0346FB71174B1B781A466D
:1096F000FB79124992000A4413441B78BB71124A49
:10970000FB79137097F90630032B05D10F4B1B68BB
:1097100001330E4A13600AE097F90630002B06D099
:1097200097F906200A4B1B681344094A136000BFCF
:109730000837BD4680BD00BFDD3500200CE70100C5
:10974000CC1A0020C41A0020DE350020D01A0020D8
:10975000C81A002080B586B000AFF860B9607A60A2
:109760000023FB758749F86812F08BFE0346002B37
:1097700006D08549F86812F084FE0346002B18D104
:109780007B685B681A468149814810F007FB7B685B
:109790005B681A467F49804810F000FB7B685B6875
:1097A0001A467E497E4810F0F9FABB6801221A7009
:1097B000E3E07C49F86812F064FE0346002B07D012
:1097C0007949F86812F05DFE0346002B40F0C58031
:1097D0007B685B681A4675496D4810F0F1FA7B6842
:1097E0005B681A467249734810F0EAFA724B1B68BC
:1097F0001A467B685B681946104610F0B4F87B681F
:109800005B6819466D4810F095F87B685B681A46EE
:1098100067496B4810F0D4FA6A4B1B681A467B689C
:109820005B681946104610F09EF87B685B68194625
:10983000624810F07FF87B685B681A465C496248B2
:1098400010F0BEFA614B1B6818460FF058FF034634
:10985000002B06D07B685B6819465D4810F06AF8FB
:1098600005E07B685B6819465A4810F063F85A4B6C
:109870001B6818460FF043FF0346002B06D07B6899
:109880005B681946554810F055F805E07B685B6841
:109890001946534810F04EF87B685B681A464449F5
:1098A000504810F08DFA504B1B681A467B685B6875
:1098B0001946104610F057F87B685B6819463F4818
:1098C00010F038F87B685B681A463949474810F051
:1098D00077FA474B1B681A467B685B681946104647
:1098E00010F041F87B685B681946344810F022F8A4
:1098F0007B685B681A462E493E4810F061FA3E4B81
:109900001B6818460FF0FBFE0346002B06D07B6851
:109910005B6819462E4810F00DF805E07B685B681F
:1099200019462C4810F006F8344B1B6818460FF007
:10993000E6FE0346002B06D07B685B681946274885
:109940000FF0F8FF05E07B685B68194624480FF0CC
:10995000F1FFBB6801221A700FE02949F86812F084
:1099600090FD0346002B08D10020FFF7C5FD002025
:10997000FFF7D2FDBB6801221A70FB7D184618372D
:10998000BD4680BD60FC01001CE7010030E701001E
:109990004CE7010054D20100A4D0010058E70100B7
:1099A00080E7010070FC010088E701009CE70100EE
:1099B0003CCF010014D80100C41A0020D4DE0100FD
:1099C000B8E70100CC1A0020C8E70100B41A002053
:1099D000D8E70100DCE70100B81A0020E0E7010049
:1099E00060D5010020D80100C81A0020E4E701007A
:1099F000D01A0020F4E70100BC1A0020C01A002091
:109A000004E8010080B500AF0C4B1B68012118462B
:109A10000FF098FE0A4B1B68012118460FF092FECA
:109A2000084B1B68012118460FF08CFE064B1B6883
:109A3000012118460FF086FE00BF80BDB41A002039
:109A4000BC1A0020B81A0020C01A002080B586B0C9
:109A500000AF3B1D184603F033FC174BBB60174BA0
:109A6000FB6010233B6101233B713B1D184603F053
:109A70008BFC0346124A136011233B613B1D1846C1
:109A800003F082FC03460F4A13600A233B613B1D2F
:109A9000184603F079FC03460B4A13600B233B6125
:109AA0003B1D184603F070FC0346084A136000BFD4
:109AB0001837BD4680BD00BF80F00F4000B00440A5
:109AC000B41A0020B81A0020BC1A0020C01A0020C6
:109AD00098B500AFFFF7BAFF1D4B00221A601D4B6F
:109AE00000221A601C4B1B6818460FF008FE034644
:109AF000002B01D0022400E00024184B1B681846FC
:109B00000FF0FDFD03465BB223435BB2DAB2144BA8
:109B10001A70144B1B6818460FF0F1FD0346002B1A
:109B200001D0022400E000240F4B1B6818460FF000
:109B3000E6FD03465BB223435BB2DAB20B4B1A700D
:109B40000B4B00221A700B4B00221A7000BF98BDFD
:109B5000C41A0020C81A0020B41A0020B81A002025
:109B6000DD350020BC1A0020C01A0020DE350020A0
:109B7000DB350020DC35002080B485B000AF786094
:109B800039600023FB600BE0FB685B007A681344DC
:109B90000A49FA6831F812201A80FB680133FB6029
:109BA000FA683B689A4202DAFB68052BECDD00BFDD
:109BB0001437BD465DF8047B704700BF0C1B0020C6
:109BC00080B584B000AF786039606E4B1B7883F04D
:109BD0000103DBB2002B01D00123CEE0694B5B789F
:109BE000002B29D0674B5B68184603F045FC664B99
:109BF0001B68664AA2FB03239B0CC82202FB03F3EB
:109C0000002B19D0604B1B68604AA2FB03239B0CFE
:109C1000C82202FB03F30A2B02D810F082FE0BE0ED
:109C2000594B1B68594AA2FB03239B0CC82202FB19
:109C300003F3184605F048FD0023BB731AE0BB7B15
:109C4000504A023352F823300121184603F078FBC2
:109C5000BB7B4C4A023352F82330184603F00CFC0D
:109C6000BB7B5B007A6813444FF6FF721A80BB7BA4
:109C70000133BB73BB7B052BE1D9434B1B68434AC4
:109C8000A2FB03239B0C322202FB03F3002B19D00F
:109C90003D4B1B683D4AA2FB03239B0C322202FB77
:109CA00003F30A2B02D810F03CFE0BE0364B1B6886
:109CB000364AA2FB03239B0C322202FB03F3184615
:109CC00005F002FD08F008FC0023BB730AE0BB7B33
:109CD0002C4A023352F82330184603F00FFBBB7BAB
:109CE0000133BB73BB7B052BF1D901F0F1FA01F015
:109CF000DBFA0023FB7301F0F7FAB860BA683B683F
:109D00009A422BD80023BB7321E0BB7B5B007A68AF
:109D100013441B884FF6FF72934212D1BB7B194A42
:109D2000023352F8233018460FF0F5FC0346002B9F
:109D30000AD0BB7B5B007A681344BA6892B21A807F
:109D400002E0FB7B0133FB73BB7B0133BB73BB7B4B
:109D5000052BDAD9FB7B062BCBD100E000BF08F046
:109D6000E1FB01F0ABFA074B5B78002B04D0054B0D
:109D70005B68184603F05AFB002318461037BD46AF
:109D800080BD00BFD41A0020E001002083DE1B4309
:109D900080B586B000AFF860B9607A600FF0FEFA67
:109DA0000346274AA2FB03239B094FF4C87202FB18
:109DB00003F3234AA2FB03239B0919467868FFF7A4
:109DC000FFFE034683F00103DBB2002B34D00023F7
:109DD0007B612EE07B695B007A6813441A887B699B
:109DE0005B00F9680B441B889A4209D27B695B00CF
:109DF0007A681A447B695B00F9680B4412881A8000
:109E00007B695B007A6813441A887B695B00B968D8
:109E10000B441B889A4209D97B695B007A681A4413
:109E20007B695B00B9680B4412881A807B69013337
:109E30007B617B69052BCDDD00BF1837BD4680BD3A
:109E4000D34D621080B586B000AF786039600023D2
:109E5000FB6000237B6115E0464B1A687B69043385
:109E60005B0013449B881A46FB68934207D2414B20
:109E70001A687B6904335B0013449B88FB607B6931
:109E800001337B617B69052BE6DD0FF087FA034622
:109E9000394AA2FB03239B094FF4C87202FB03F368
:109EA000354AA2FB03239B09FA689A420FD90FF0A7
:109EB00075FA0346304AA2FB03239B094FF4C8728C
:109EC00002FB03F32C4AA2FB03239B09FB60F96806
:109ED0003868FFF775FE274B1B68002B45D0002321
:109EE0007B613EE000233B61224B1A687B690433AF
:109EF0005B0013449B8819461E4B1B687A6933F834
:109F00001230CB1ABB60BB68002B13D07B695B009F
:109F10003A6813441B881946164B1B687A6933F854
:109F20001230CB1A4FF47A7203FB02F2BB6892FB39
:109F3000F3F33B613B69002B02DA00233B6106E04F
:109F40003B69B3F57A7F02DD4FF47A733B617B693D
:109F50005B007A6813443A6992B21A807B690133D4
:109F60007B617B69052BBDDD00E000BF1837BD4676
:109F700080BD00BFF81A0020D34D621080B483B0BA
:109F800000AF0346FB71FB79052B1BD801A252F8E9
:109F900023F000BFAD9F0000B19F0000B59F0000FF
:109FA000B99F0000BD9F0000C19F0000094B0AE05F
:109FB000094B08E0094B06E0094B04E0094B02E0BD
:109FC000094B00E0094B18460C37BD465DF8047B91
:109FD000704700BF1CD6010018E8010024E801000A
:109FE0002CE8010034E801003CE8010040E80100F1
:109FF00080B483B000AF0346FB71FB79012B05D021
:10A00000FB79022B02D0FB79032B02D1114B1B7879
:10A010001AE0FB79002B15D10E4B1B78052B0FDCBA
:10A02000042B0BDA002B05D0002B09DB013B022BA4
:10A0300006D801E0002307E0012305E0002303E048
:10A04000002301E0034B1B7818460C37BD465DF832
:10A05000047B7047E035002080B400AF034B1B88C1
:10A060001846BD465DF8047B704700BFCE35002022
:10A0700080B500AF10491148FFF7E4FE00220E49F9
:10A080000E480EF07FFF03461AB20D4B1A800B48A4
:10A090000FF074F803461A460A4B1A800A4B1B78D5
:10A0A000DBB2062B06D105480EF0B9FF03461A466F
:10A0B000064B1A7000BF80BD001B00200C1B002047
:10A0C000CC350020CE350020DF350020E0350020E3
:10A0D00080B500AF0D4B01221A700D4B1B78DBB21F
:10A0E000012B09D00A4B1B78DBB2032B04D0084BA1
:10A0F0001B78DBB2062B06D1064B18680023002222
:10A10000002111F0FAF800BF80BD00BFD41A002072
:10A11000DF350020F41A002080B400AF064B1B7816
:10A12000DBB2062B0CBF01230023DBB21846BD4671
:10A130005DF8047B704700BFDF35002080B483B03A
:10A1400000AF78600E4BB3F90030002B08DD0C4BEC
:10A15000B3F9003041F65732934201DC012300E0AD
:10A16000002303F00103DAB27B681A70044BB3F9E1
:10A1700000309BB218460C37BD465DF8047B704733
:10A18000CC35002080B582B000AF78607B685B681A
:10A190001A46124912480FF001FE7B685B681A46A6
:10A1A000104911480FF0FAFD7B685B681A460F49A9
:10A1B0000F480FF0F3FD7B685B681A460D490E48A7
:10A1C0000FF0ECFD7B685B681A460C490C480FF0F9
:10A1D000E5FD002318460837BD4680BD48E801006C
:10A1E00068E8010054D20100A4D001006CE801002D
:10A1F000A0E80100B4E80100ECE8010004E9010076
:10A200003CE9010080B400AF154B1B78DBB2062B94
:10A210001ED801A252F823F035A2000039A2000096
:10A220003DA2000041A2000045A2000049A200009A
:10A230004DA200000B4B0DE00B4B0BE00B4B09E06C
:10A240000B4B07E00B4B05E00B4B03E00B4B01E026
:10A2500000BF0B4B1846BD465DF8047B704700BF3E
:10A26000DF350020C0CE010054E9010064E901009F
:10A2700078E9010084E9010098E90100ACE90100F6
:10A2800038D6010080B58CB000AF78607B685B6821
:10A290001A469A499A480FF093FD9A4B1B78002B67
:10A2A00001D0994900E099497B685B681A46984853
:10A2B0000FF086FD7B685B681A46964996480FF05A
:10A2C0007FFDFFF79FFF01467B685B681A46934856
:10A2D0000FF076FD7B685B68194691480FF02AFB0A
:10A2E000884B5B78002B01D0874900E087497B6869
:10A2F0005B681A468B480FF063FD07F10C038A4A2E
:10A30000202118460FF053FE07F10C0340222021B4
:10A31000184610F02CF807F10C03814A202118464A
:10A320000FF06AFE7B685A6807F10C0319467F48F4
:10A330000FF046FD07F10C037B4A202118460FF071
:10A3400036FE07F10C034FF480722021184610F0FE
:10A350000EF807F10C03724A202118460FF04CFE4C
:10A360007B685A6807F10C03194671480FF028FD05
:10A3700007F10C034FF4C8722021184604F042FF85
:10A3800007F10C036B4A202118460FF035FE0FF041
:10A3900005F80346684AA2FB03239B094FF4C872E1
:10A3A00002FB03F3644AA2FB03239B099AB207F161
:10A3B0000C03202118460FF0DAFF07F10C035F4A67
:10A3C000202118460FF018FE7B685A6807F10C032D
:10A3D00019465B480FF0F4FC7B685B681A465949E4
:10A3E00059480FF0EDFC0023FB6226E0FB6A002BCE
:10A3F00006D17B685B6819464B480FF09BFA05E075
:10A400007B685B68194651480FF094FA00233B7350
:10A410004F4AFB6A32F8132007F10C03202118463B
:10A420000FF0A5FF7B685A6807F10C031146184628
:10A430000FF080FAFB6A0133FB62FB6A052BD5DD66
:10A440007B685B68194636480FF074FA414B1B680D
:10A45000002B3AD07B685B681A463A493E480FF0B9
:10A46000AFFC0023FB6227E0FB6A002B06D17B6870
:10A470005B6819462C480FF05DFA05E07B685B6865
:10A48000194632480FF056FA00233B73314B1B68D4
:10A49000FA6A33F8122007F10C03202118460FF056
:10A4A00066FF7B685A6807F10C03114618460FF0E7
:10A4B00041FAFB6A0133FB62FB6A052BD4DD7B6842
:10A4C0005B68194616480FF035FA224B1B68002BC3
:10A4D0006FD07B685B681A461A4920480FF070FC01
:10A4E0000023FB625CE0FB6A002B39D17B685B6870
:10A4F00019460D480FF01EFA38E000BFB4E901001C
:10A50000CCE90100D41A00201CE2010024E2010081
:10A51000D8E90100E4E90100ECE9010010E00100E4
:10A52000D4DE0100F4E9010004EA010008EA0100B8
:10A5300014EA010020EA0100D34D621028EA01006C
:10A5400034EA01003CCF010040EA010024EA0100A6
:10A55000001B0020F81A00204CEA010058EA010014
:10A560007B685B6819465D480FF0E4F900233B7394
:10A570005B4B1A68FB6A04335B0013449A8807F14B
:10A580000C03202118460FF0F2FE7B685A6807F191
:10A590000C03114618460FF0CDF9FB6A0133FB623C
:10A5A000FB6A052B9FDD7B685B6819464D480FF001
:10A5B000C1F94B4B1B68002B39D07B685B681A468E
:10A5C00049494A480FF0FCFB0023FB6226E0FB6A86
:10A5D000002B06D17B685B68194645480FF0AAF945
:10A5E00005E07B685B6819463C480FF0A3F900233F
:10A5F0003B73404AFB6A32F8132007F10C03202119
:10A6000018460FF0B4FE7B685A6807F10C03114638
:10A6100018460FF08FF9FB6A0133FB62FB6A052BCA
:10A62000D5DD7B685B6819462E480FF083F97B689F
:10A630005B681A462C4930480FF0C2FB00233B737D
:10A640002E4BB3F9002007F10C03202118460FF020
:10A6500002FE7B685A6807F10C03114618460FF09A
:10A6600069F97B685B6819461E480FF063F97B68DF
:10A670005B681A461C4922480FF0A2FB00233B737B
:10A68000204B1B881AB207F10C03202118460FF04B
:10A69000E2FD7B685A6807F10C03114618460FF07B
:10A6A00049F97B685B6819460E480FF043F9164B71
:10A6B0001B781846FFF762FC01467B685B681A4608
:10A6C00012480FF07DFB7B685B68194605480FF068
:10A6D00031F9002318463037BD4680BD24EA010019
:10A6E000F81A0020D4DE01003CCF010064EA01002A
:10A6F00004EA01000C1B002070EA0100CC350020A8
:10A700007CEA0100CE350020E03500208CEA010013
:10A7100080B584B000AFF860B9607A605849F868D5
:10A7200011F0AFFE0346002B06D05649F86811F031
:10A73000A8FE0346002B07D1BB6801221A70786877
:10A74000FFF720FD034697E04F49F86811F099FEA6
:10A750000346002B06D04D49F86811F092FE0346DF
:10A76000002B07D1BB6801221A707868FFF78AFDB9
:10A77000034681E04649F86811F083FE0346002B4A
:10A7800007D1444B01221A70BB6801221A700023C2
:10A7900072E04149F86811F074FE0346002B07D1BE
:10A7A0003C4B00221A70BB6801221A70002363E040
:10A7B0003A49F86811F065FE0346002B18D1384B72
:10A7C0001B78DBB2012B04D0354B1B78DBB2062B98
:10A7D00006D1FBF7EFF8BB6801221A7000234BE0AB
:10A7E0007B689B6819462F480FF0A4F81B2343E0B1
:10A7F0002D49F86811F045FE0346002B13D1284B74
:10A800001B78DBB2032B06D1FBF7E0F8BB68012213
:10A810001A70002330E07B689B68194623480FF0CC
:10A8200089F81B2328E02249F86811F02AFE034624
:10A83000002B0CD1174B01225A70164B5B6818463F
:10A8400002F0F4FDBB6801221A70002314E01949DC
:10A85000F86811F016FE0346002B0CD10D4B0022B8
:10A860005A700C4B5B68184602F006FEBB6801226A
:10A870001A70002300E0002318461037BD4680BD43
:10A8800060FC010098EA010070FC0100A4EA0100EC
:10A89000B0EA0100D41A0020BCEA0100C8EA0100B5
:10A8A000DF350020D8EA010020EB010030EB010089
:10A8B00058EB01006CEB010080B582B000AF7C4B1F
:10A8C0001B78DBB2062B00F2EE8001A252F823F0D7
:10A8D000EDA8000015A900005DA90000D1A90000A5
:10A8E00021AA00002FAA00007FAA0000FEF70EF8A0
:10A8F0000346704A13606F4B1B68002B03D06C4BF0
:10A9000006221A70CFE06C48F8F71AF8684B01225B
:10A910001A70C8E0502007F0E9FF0EF03FFD034633
:10A92000664AA2FB03239B094FF4C87202FB03F3A0
:10A93000624AA2FB03239B0919466148FFF740F9CD
:10A94000604B1B680021184610F086FF0346012B60
:10A9500040F0A480564B02221A709FE05A48F7F745
:10A96000EFFF5A4B1B68002B03D0514B00221A708B
:10A9700099E0182007F0EAFA0346544A1360534B53
:10A980001B68002B20D000237B6016E04F4B1B6818
:10A990007A684FF6FF7123F812104C4B1A687B68E7
:10A9A00004335B00134400229A80494A7B680021EB
:10A9B00022F813107B6801337B607B68052BE5DD93
:10A9C0003B4B03221A706EE0394B00221A706AE08A
:10A9D000502007F08BFF3D4B1B68002B18D03B4BE2
:10A9E0001B681846394B1B680C33354A1946FFF76C
:10A9F000CFF932214FF49670FBF7DCFA314B1B682C
:10AA00000021184610F028FF0346012B48D103E02F
:10AA1000274B00221A7046E0254B04221A703FE0B3
:10AA20002C48F7F78DFF224B05221A703BE0274B8D
:10AA30001B6818211846FDF751FF0346002B02D072
:10AA40002548F7F77DFF214B1B68184607F020FBD0
:10AA50001E4B00221A60FDF759FF0346154A13608A
:10AA6000144B1B68002B06D01C48F7F769FF104BEE
:10AA700006221A7017E00E4B00221A7013E0FFF73F
:10AA8000F7FA104B1B680021184610F0E5FE03464C
:10AA9000012B07D1064B02221A7003E000BF02E02F
:10AAA00000BF00E000BF00BF0837BD4680BD00BF4B
:10AAB000DF350020F81A002080EB0100D34D621032
:10AAC000001B0020F41A0020A0EB0100FC1A00205B
:10AAD0000C1B0020B8EB0100D4EB0100F4EB0100EB
:10AAE00080B582B000AF7860064B1B78002B05D094
:10AAF000FFF7E2FE052007F0F9FEF5E7642007F016
:10AB0000F5FEF1E7D41A002090B5A1B002AF3B46A4
:10AB100060220021184611F0D3FB544B3B60544B8C
:10AB20007B600223BB60514B3B61514B7B61032334
:10AB3000BB614E4B3B624E4B7B620423BB624B4B73
:10AB40003B634B4B7B630523BB63484B3B64484BE8
:10AB50007B640623BB64454B3B65454B7B65072304
:10AB6000BB65444B01221A70424B00225A7007F118
:10AB70006003184602F0A4FB3C4B7B663C4BBB6673
:10AB80000123FB66002387F86030012387F86130DA
:10AB900007F16003184602F0F7FB0346354A53609D
:10ABA000354B00221A70012387F86030002387F8A4
:10ABB000613000237B6717E07B6F1B0178333B44D8
:10ABC000783B07F164040FCB84E80F0007F16003C2
:10ABD000184602F0D9FB024626497B6F023341F842
:10ABE00023207B6F01337B677B6F052BE4DD032222
:10ABF0000021012010F011FB0346204A13601F4B77
:10AC00001B68002B06D01D4B186800230022002172
:10AC100010F073FB194B1B68002B00D1FEE7174B9C
:10AC20001B680021184610F017FE144B1B681449CE
:10AC3000184607F03DFD134B00221A70124B0022FC
:10AC40001A70124B00221A800023019304230093F0
:10AC5000002389220E490F4811F0F6F80346012B14
:10AC600000D0FEE700BF7C37BD4690BDC0F00F406E
:10AC700000C00440D41A00204B020020F41A002027
:10AC800010EC0100DF350020E0350020CC3500203D
:10AC900020EC0100E1AA000080B582B000AF0346BD
:10ACA000FB71054B1868F91D00230A2210F025FBE3
:10ACB00000BF0837BD4680BD181B002080B5A6B078
:10ACC00000AF78600023BB6007F10C037C220021F9
:10ACD000184611F0F5FA002387F89730002387F81B
:10ACE0009630444B1B6807F18B010A22184610F07E
:10ACF000C3FCC7F89000D7F89030002B03D1002395
:10AD000087F88B30EDE7D7F89030012BE9D197F831
:10AD10008B30402B19D1012387F89730002387F817
:10AD20009630002387F895300BE097F895309833EC
:10AD30003B44002203F8902C97F89530013387F8B4
:10AD4000953097F99530002BEFDA97F88B30212B5F
:10AD500038D197F89730012B34D1002387F89730FA
:10AD600004F032F803465B68194623480EF0E2FD12
:10AD700004F02AF803465A6807F1080311461846FA
:10AD80000EF0D8FD04F020F803465B6819461B4816
:10AD90000EF0D0FD07F108030B221949184611F0F7
:10ADA0008AFB0346002B24D107F108030B33C7F8B5
:10ADB0008C3001F019FE03461946D7F88C00F7F7DE
:10ADC000ADFD16E097F89730012B8AD197F89630B1
:10ADD0005A1C87F8962097F88B2098333B4403F849
:10ADE000902C97F99630002BBFF67BAF002387F8A5
:10ADF000963076E7181B002028EC0100D4DE010015
:10AE000044EC010080B582B002AF0023019301231E
:10AE1000009300234FF480720E490F4811F014F88C
:10AE20000346012B00D0FEE700220121202010F074
:10AE3000F4F90346094A1360084B1B68002B00D144
:10AE4000FEE7064B1B680649184607F031FC00BFB9
:10AE5000BD4680BD50EC0100BDAC0000181B0020B9
:10AE600058EC010080B483B000AF0346FB71FB795E
:10AE7000002B02D0054B1B6801E0054B1B681846F0
:10AE80000C37BD465DF8047B704700BFA41B002053
:10AE9000A81B002080B48BB000AFEFF3108072B617
:10AEA000F8703D4B1B78DBB21A463C4B53F822300E
:10AEB000BB60394B1B78DBB21A46394B53F8223052
:10AEC0007B60354B1B78DBB2002B06D1334B1B6C00
:10AED000FB61334B1B6CBB610FE02F4B1B78DBB26C
:10AEE000013B2E4A52F82330FB612B4B1B78DBB21F
:10AEF000013B2B4A52F82330BB61F87880F310886D
:10AF0000BA68FB69D31A7B627B6A002B05DA7B6A1D
:10AF10005B427B620123FB7301E00023FB737A68D1
:10AF2000BB69D31A3B623B6A002B05DA3B6A5B4282
:10AF30003B620123BB7301E00023BB737B6A4FF4C8
:10AF40007A7202FB03F3174AA2FB03239B097B617E
:10AF5000FB7B002B02D07B695B427B613B6A4FF439
:10AF60007A7202FB03F30F4AA2FB03239B093B61A6
:10AF7000BB7B002B02D03B695B423B617B695B4240
:10AF8000094A13603B695B42084A136000BF2C37D3
:10AF9000BD465DF8047B7047E13500201C1B002096
:10AFA000601B0020CDCCCCCCA41B0020A81B002013
:10AFB00098B500AF194B1B6801331A46174B1A603E
:10AFC000164B1B68042B26DD144B00221A60144B11
:10AFD0001B78DBB21C46FEF7AFFA0346114A42F873
:10AFE00024300F4B1B78DBB21C46FEF7B1FA034648
:10AFF0000D4A42F824300A4B1B78DBB20133DAB237
:10B00000074B1A70064B1B78DBB2102B04D9044B8C
:10B0100000221A7000E000BF98BD00BFAC1B0020EA
:10B02000E13500201C1B0020601B002080B582B091
:10B0300000AF78607B685B681A461B491B480EF0BE
:10B04000BFFE7B685B681A4619491A480EF0B8FEC5
:10B050000120FFF707FF02467B685B681946104630
:10B060000EF081FC7B685B68194613480EF062FCA9
:10B070007B685B681A460E4910480EF0A1FE00205E
:10B08000FFF7F0FE02467B685B68194610460EF03B
:10B090006AFC7B685B68194607480EF04BFC00BFF2
:10B0A0000837BD4680BD00BF70EC010084EC010094
:10B0B0003CCF01008CEC0100D8D7010098EC0100D6
:10B0C00080B582B000AF78607B685B681A4607493C
:10B0D00007480EF063FE7B685B681A460549064820
:10B0E0000EF05CFE00BF0837BD4680BDA4EC010039
:10B0F000C0EC0100C8EC0100A4D0010080B584B010
:10B1000000AFF860B9607A601649F86811F0B9F9D3
:10B110000346002B06D01449F86811F0B2F9034633
:10B12000002B06D17868FFF7CBFFBB6801221A70AD
:10B1300013E00E49F86811F0A4F90346002B06D07D
:10B140000B49F86811F09DF90346002B05D178688A
:10B15000FFF76CFFBB6801221A70002318461037F6
:10B16000BD4680BD60FC0100E8EC010070FC010000
:10B17000F4EC010080B400AF064B00221A60064BCD
:10B1800000221A60054B00221A7000BFBD465DF810
:10B19000047B7047A41B0020A81B0020E135002081
:10B1A00080B483B000AF0346FB7197F90730002BE2
:10B1B0000BDBFB7903F01F02074997F907305B09A6
:10B1C000012000FA02F241F8232000BF0C37BD46EF
:10B1D0005DF8047B704700BF00E100E080B483B0FD
:10B1E00000AF03463960FB7197F90730002B0ADB8B
:10B1F0003B68DAB20C4997F907301201D2B20B441E
:10B2000083F800230AE03B68DAB20849FB7903F0CF
:10B210000F03043B1201D2B20B441A7600BF0C3765
:10B22000BD465DF8047B704700E100E000ED00E002
:10B2300080B582B000AF78607B68002B05D1064BEB
:10B24000064A8521064809F0AFFD7B6800221A7086
:10B2500000BF0837BD4680BDB0C8010040ED010009
:10B2600004ED010080B500AF0D4B1B6801330C4AA3
:10B2700013600B4B1A680B4BA3FB0213DB094FF453
:10B28000FA6101FB03F3D31A002B02D10120FBF773
:10B2900087FD00F099F9FFF78BFE00BF80BD00BF6E
:10B2A000B01B0020D34D621080B500AF01210248D1
:10B2B0000DF0C9FF00BF80BD0090034080B500AF16
:10B2C00002480DF0DDFF00BF80BD00BF00900340CD
:10B2D00080B400AF034B00225A6000BFBD465DF84A
:10B2E000047B70470090034080B500AF02480DF02A
:10B2F0009DFF0346184680BD0090034080B588B08E
:10B3000000AF3B1D1846F9F779FA00233B713B1D4E
:10B3100019460848F9F7F2F94FF6FF7105480DF0A4
:10B3200077FF012103480DF08EFF00BF2037BD4697
:10B3300080BD00BF0090034080B582B000AF0346DF
:10B34000FB71FB79C3F16403DBB2002202210548E3
:10B35000F9F724FC012103480DF0A2FF00BF0837D4
:10B36000BD4680BD0080034080B582B000AF03467B
:10B37000FB71FB79C3F16403DBB2002203210548B2
:10B38000F9F70CFC012103480DF08AFF00BF0837D4
:10B39000BD4680BD0080034080B500AF012102485A
:10B3A0000DF051FF00BF80BD0080034080B58CB020
:10B3B00002AF022387F82030012387F821300023D1
:10B3C00087F82230002387F82330032387F82430BE
:10B3D000012387F82530002387F82630002387F8DB
:10B3E00027303B1D1846F9F709FA3B1D19460E4850
:10B3F000F9F784F90220F8F795F8034607F12001E0
:10B40000019345F6C0530093002302220648F9F742
:10B4100031FA0020FFF790FF0020FFF7A5FF00BFE3
:10B420002837BD4680BD00BF0080034080B500AF17
:10B430000122002104480DF06CFFFEF729F9BFF34B
:10B440004F8F00BF00BF80BD007003402DE9B04F9B
:10B4500084B000AF07F10C031846FFF7E9FE0023A4
:10B460003B7307F10C0319462948F9F731FD022017
:10B47000F8F758F8034600229846914642464B4654
:10B48000911839605B417B60D7E9002312EB080417
:10B4900043EB09054FF000024FF00003EB0043EAD5
:10B4A0005473E20014461D4614EB080A45EB090BE1
:10B4B0004FF000024FF000034FEACB0343EA5A7308
:10B4C0004FEACA0292469B4650465946114A4FF0EF
:10B4D000000309F0E7FA02460B4613461A4600211C
:10B4E0000B480DF02BFF0222002109480DF0F4FE5D
:10B4F00000213020FFF772FE30200DF073FE002196
:10B5000003480DF02FFF00BF1037BD46BDE8B08FD8
:10B510000070034040420F0080B584B000AF0023AC
:10B52000BB730023FB7345E0EFF3108072B6F87035
:10B53000FA7B244913465B0013449B000B441B8891
:10B54000002B31D1FA7B1F4913465B0013449B004B
:10B550000B4404331B68002B26D0FA7B1949134691
:10B560005B0013449B000B4404331B68BB60FA7BF5
:10B57000144913465B0013449B000B4408331B68BB
:10B580007B60FA7B0F4913465B0013449B000B441E
:10B59000043300221A60F87880F31088BB6878685A
:10B5A00098470123BB7302E0F87880F31088FB7B97
:10B5B0000133FB73FB7B022BB6D9BB7B18461037DC
:10B5C000BD4680BDB41B002080B582B000AFEFF354
:10B5D000108072B678710023FB711EE0FA79184969
:10B5E00013465B0013449B000B441B88002B11D0B7
:10B5F000FA79134913465B0013449B000B441B88E4
:10B60000013B98B20E4913465B0013449B000B4468
:10B6100002461A80FB790133FB71FB79022BDDD9DD
:10B62000787980F31088FFF777FF0346BB71BB7909
:10B63000002BF8D100BF00BF0837BD4680BD00BF5A
:10B64000B41B002080B483B000AF0023FB711FE067
:10B65000FA79144913465B0013449B000B44002203
:10B660001A80FA790F4913465B0013449B000B4480
:10B67000043300221A60FA790A4913465B00134426
:10B680009B000B44083300221A60FB790133FB71E5
:10B69000FB79022BDCD900BF00BF0C37BD465DF83B
:10B6A000047B7047B41B002080B485B000AFF86005
:10B6B000B9607A60074ABB681360074A7B68136009
:10B6C000064AFB68136000BF1437BD465DF8047B73
:10B6D000704700BFD4010020D8010020D001002015
:10B6E00080B483B000AF0346FB71FB79112B45D8C2
:10B6F00001A252F823F000BF41B7000045B7000097
:10B7000049B700004DB7000051B7000055B7000021
:10B7100059B700005DB700006DB7000071B70000B9
:10B7200061B700007DB7000065B7000069B7000091
:10B7300079B700007DB700007DB7000075B7000045
:10B74000124B1CE0124B1AE0124B18E0124B16E0A1
:10B75000124B14E0124B12E0124B10E0124B0EE0B1
:10B76000124B0CE0124B0AE0124B08E0124B06E0C1
:10B77000124B04E0124B02E0124B00E0124B184651
:10B780000C37BD465DF8047B704700BF58ED0100E3
:10B7900060ED010068ED010070ED010078ED010041
:10B7A00080ED010018E801008CED01009CED010026
:10B7B000ACED0100C0ED0100D4ED0100ECED0100A5
:10B7C00024D6010004EE01000CEE010080B584B027
:10B7D00000AFF860B9603B601346FB71B968F86868
:10B7E000FAF7F4FE0320FAF7AFFE3B68002B04D013
:10B7F0003B6898470346002B17D1012007F076F8E5
:10B80000BB69013BBB61BB69002B10DDFB79002BE1
:10B8100004D0FAF745FE0346002B0AD1FB7983F0EA
:10B820000103DBB2002B06D1DFE700BF04E000BF5D
:10B8300002E000BF00E000BFBB69002B02DC034850
:10B84000F7F77EF800BF1037BD4680BD1CEE010043
:10B8500080B582B000AF03463960FB71FB79112BD4
:10B8600000F2008101A252F823F000BFB5B8000039
:10B8700001B90000DBB8000017B900002DB90000C5
:10B880004DB9000065BA00008BB90000DBB90000BB
:10B89000FBB900009DB900006DB90000B3B900000C
:10B8A000C5B9000065BA00001FBA000031BA000037
:10B8B00043BA00006F4B1B685B42DA0F13445B1006
:10B8C00018466C4B1B68DA0F13445B1019464FF493
:10B8D000FA733A680DF074FDC5E0664B1B68DA0F29
:10B8E00013445B101846634B1B685B42DA0F13442A
:10B8F0005B1019464FF4FA733A680DF061FDB2E03F
:10B900005C4B1B6858425B4B19684FF47A733A687A
:10B910000DF056FDA7E0574B1868564B1B6859426F
:10B920004FF47A733A680DF04BFD9CE0514B1A6866
:10B930001346DB079B1A5B0018464E4B1B685900E9
:10B940004FF4FA633A680DF03BFD8CE0494B1B68FD
:10B950005800484B1A681346DB079B1A5B001946D0
:10B960004FF4FA633A680DF02BFD7CE0424B1B6804
:10B970001A469B00D01A404B1B681A469B00D11AEE
:10B98000C8233A680DF01CFD6DE03B4B18683A4B3C
:10B990001968C8233A680DF013FD64E0364B1B6844
:10B9A0005842354B1B685942C8233A680DF008FDD0
:10B9B00059E0324B1868314B1968C8233A680DF0CA
:10B9C000FFFC50E02D4B1B6858422C4B1B68594222
:10B9D000C8233A680DF0F4FC45E0274B1A68274B62
:10B9E0001B68D018244B1A68244B1B68D1184FF4DD
:10B9F000C8733A680DF0E4FC35E01F4B1B685A42EF
:10BA00001E4B1B68D01A1C4B1B685A421B4B1B68F1
:10BA1000D11A4FF4C8733A680DF0D2FC23E000202D
:10BA2000FCF73EFB034600211846FCF7CDFB1AE06D
:10BA30000120FCF735FB034600211846FCF7C4FB48
:10BA400011E00020FCF72CFB034600211846FCF710
:10BA5000BBFB0120FCF724FB034600211846FCF742
:10BA6000B3FB00E000BF0DF0CEFC00BF0837BD46C1
:10BA700080BD00BFD0010020D4010020D8010020EB
:10BA800080B584B000AF03463960FB80FB88DB0BD8
:10BA9000FB73FB7B002B03D0FB885B429BB2FB80DC
:10BAA000B7F90630274A82FB03121A441112DA173B
:10BAB0008A1A4FF4B47101FB02F29B1AFB80B7F9AA
:10BAC0000630214A126802FB03F31E4A82FB03126E
:10BAD0001A449211DB17D31ABB60FB7B002B15D0E5
:10BAE000BB685842B7F90630164A82FB03121A4463
:10BAF0009211DB17D31A1BB201334FF47A7202FB97
:10BB000003F33A68B9680DF05BFC14E0BB68594276
:10BB1000B7F906300B4A82FB03021A449211DB1775
:10BB2000D31A1BB201334FF47A7202FB03F33A6863
:10BB3000B8680DF045FC0DF066FC00BF1037BD463F
:10BB400080BD00BFB7600BB6D001002080B582B0C9
:10BB500000AF78607B685B681A46204920480EF089
:10BB60001DF97B685B681A461E491F480EF016F9DE
:10BB70007B685B681A461D491D480EF00FF97B680B
:10BB80005B681A461B491C480EF008F97B685B6825
:10BB90001A461A491A480EF001F97B685B681A4682
:10BBA000184919480EF0FAF87B685B681A4617497D
:10BBB00017480EF0F3F87B685B681A46154916487B
:10BBC0000EF0ECF87B685B681A46144914480EF0D6
:10BBD000E5F800BF0837BD4680BD00BF34EE010068
:10BBE00050EE010058EE0100A4D0010074EE0100F7
:10BBF000C0EE0100CCEE0100E4EE0100F0EE010029
:10BC000018EF01002CEF010048EF010054EF010094
:10BC10007CEF010090EF0100BCEF0100D0EF0100CC
:10BC2000FCEF010080B58AB000AF78607B685B688C
:10BC30001A46504950480EF0C3F8504B1A6807F1A5
:10BC400008032021184603F0F3FB07F108034C4AD0
:10BC5000202118460EF0D0F97B685A6807F10803D6
:10BC6000194648480EF0ACF8474B1A6807F108032C
:10BC70002021184603F0DCFB07F10803404A20218D
:10BC800018460EF0B9F97B685A6807F1080319469F
:10BC90003E480EF095F83E4B1A6807F10803202144
:10BCA000184603F0C5FB07F10803354A2021184662
:10BCB0000EF0A2F97B685A6807F108031946354867
:10BCC0000EF07EF8FDF738FC03461A4607F108032C
:10BCD0002021184603F0ACFB07F108032E4A20216F
:10BCE00018460EF089F9FDF7EFFB03469AB207F10B
:10BCF0000803202118460EF095FA07F10803274A99
:10BD0000202118460EF078F97B685A6807F108037D
:10BD1000194623480EF054F8FDF71AFC03461A465C
:10BD200007F108032021184603F082FB07F10803FE
:10BD3000194A202118460EF05FF9FDF7D1FB0346A2
:10BD40009AB207F10803202118460EF06BFA07F1AA
:10BD50000803124A202118460EF04EF97B685A68F3
:10BD600007F1080319460F480EF02AF800BF2837DC
:10BD7000BD4680BD14F0010050EE0100D00100204E
:10BD800028F0010034F00100D4010020ECE90100AA
:10BD9000D801002040F001004CF0010050F00100FB
:10BDA0005CF0010068F0010080B588B000AFF86079
:10BDB000B9607A600023FB778D49F86810F061FB69
:10BDC0000346002B06D08B49F86810F05AFB034657
:10BDD000002B06D17868FFF7B9FEBB6801221A7004
:10BDE00000E18549F86810F04CFB0346002B06D0B3
:10BDF0008249F86810F045FB0346002B06D17868AD
:10BE0000FFF710FFBB6801221A70EBE005227C49A6
:10BE1000F86810F050FB0346002B36D1FB68053361
:10BE20001B7818460DF0F6FA0346002B2DD0FB6860
:10BE30000533BB6107F1100207F1180311461846DC
:10BE40000EF032FB0346002B16D13B691BB20021DA
:10BE50001846FFF715FE00211120FFF7F9FC4FF4FB
:10BE6000C8714FF4C870FAF78FFB0220FAF76CFB29
:10BE7000BB6801221A70B5E07B689B68194661486F
:10BE80000DF058FD1B23FB77ACE05F49F86810F01C
:10BE9000F8FA0346002B0BD100210820FFF7D8FC4D
:10BEA00000211120FFF7D4FCBB6801221A7099E031
:10BEB0005649F86810F0E5FA0346002B0BD1002133
:10BEC0000720FFF7C5FC00211120FFF7C1FCBB686C
:10BED00001221A7086E04E49F86810F0D2FA034643
:10BEE000002B0BD100210A20FFF7B2FC002111200A
:10BEF000FFF7AEFCBB6801221A7073E00D224549C2
:10BF0000F86810F0D8FA0346002B1ED1FB680D33F9
:10BF1000BB6107F1160207F11803114618460EF02F
:10BF2000BDFB0346002B07D1FB8A1A463A4B1A6029
:10BF3000BB6801221A7055E07B689B68194631483E
:10BF40000DF0F8FC1B23FB774CE013223349F86813
:10BF500010F0B1FA0346002B1ED1FB681333BB610E
:10BF600007F1160207F11803114618460EF096FB6A
:10BF70000346002B07D1FB8A1A46294B1A60BB687F
:10BF800001221A702EE07B689B6819461D480DF04F
:10BF9000D1FC1B23FB7725E00F222249F86810F023
:10BFA0008AFA0346002B1DD1FB680F33BB6107F1F2
:10BFB000160207F11803114618460EF06FFB0346F0
:10BFC000002B07D1FB8A1A46174B1A60BB68012267
:10BFD0001A7007E07B689B6819460A480DF0AAFCB6
:10BFE0001B23FB77FB7F18462037BD4680BD00BF73
:10BFF00060FC010074F0010070FC010080F00100A1
:10C000008CF001009CE6010094F00100ACF001000E
:10C01000BCF00100CCF00100D0010020DCF00100F8
:10C02000D8010020F0F00100D401002080B400AF5E
:10C03000074B4FF434721A60064B96221A60064B77
:10C0400064221A6000BFBD465DF8047B704700BFE4
:10C05000D0010020D8010020D401002080B59CB080
:10C0600000AF78607B685B681A46244924480DF06D
:10C07000A7FE07F10C0318460DF0E5F9034687F813
:10C080006F3097F86F30002B0AD107F11C0107F1D0
:10C090000C035322184600F071F8034687F86F30FE
:10C0A00097F86F30002B06D007F11C03154A532177
:10C0B00018460DF07CFF7B685A6807F11C0319468F
:10C0C00011480DF07DFE7B685B6819460F480DF046
:10C0D00031FC00F0DFF801467B685B681A460C48CB
:10C0E0000DF06EFE7B685B68194608480DF022FC77
:10C0F000002318467037BD4680BD00BFA0F1010087
:10C10000B4F10100C0F10100C8F10100D4DE01006A
:10C11000D0F1010080B582B000AF78607B685B68C9
:10C120001A460B490B480DF039FE7B685B681A46CE
:10C1300009490A480DF032FE7B685B681A460849D7
:10C1400008480DF02BFE002318460837BD4680BD79
:10C15000DCF10100B4F10100FCF1010080E7010015
:10C1600054D20100A4D0010080B400AF014B024AB8
:10C17000DA60FEE700ED00E00400FA0580B586B065
:10C1800000AFF860B9607A60164A7968B8680DF057
:10C190000EFF00237B6118E0134A7968B8680DF040
:10C1A0002BFFFA687B6913441B781A467968B868D4
:10C1B0000EF0AEF87B690E2B04D80C4A7968B8688B
:10C1C0000DF01AFF7B6901337B617B690F2BE3D98B
:10C1D000074A7968B8680DF00FFF00231846183732
:10C1E000BD4680BD18F2010004EA01001CF2010006
:10C1F00020F2010080B586B000AFF860B9607A60C7
:10C200000023FB751E49F86810F03BF90346002B2C
:10C2100006D01C49F86810F034F90346002B07D10A
:10C22000BB6801221A707868FFF774FF034623E0A9
:10C230001549F86810F025F90346002B06D013497C
:10C24000F86810F01EF90346002B08D1BB680122E4
:10C250001A707868FFF702FF0346FB750BE00C4984
:10C26000F86810F00EF90346002B04D1BB680122D8
:10C270001A70FFF779FFFB7D18461837BD4680BD61
:10C2800060FC010024F2010070FC010038F20100A2
:10C290004CF2010080B483B000AF0D4B03F5805326
:10C2A0005B6A1B0903F003037B607B68002B07DBE1
:10C2B0007B68082B04DC074A7B6852F8233000E0D7
:10C2C000054B18460C37BD465DF8047B704700BF30
:10C2D0000070044080F1010060F2010080B582B07E
:10C2E00000AF78607B68002B05D1074B074A2E21F1
:10C2F000074808F059FD1422064978680FF0D2FF6C
:10C3000000BF0837BD4680BD90F20100C8F20100B1
:10C31000A0F201007CF2010080B584B000AF78602B
:10C320007B68002B05D10E4B0E4A47210E4808F0C2
:10C330003BFD7B68FB60FB681B78002B06D0FB682D
:10C340005B6818460DF0E7F9034605E0FB685B689B
:10C35000184601F013F9034618461037BD4680BD54
:10C36000ACF20100E0F20100A0F2010080B588B05B
:10C3700000AF78607B68002B05D11E4B1E4A53210D
:10C380001E4808F011FD082005F0E0FDF861FB698A
:10C39000002B05D11A4B184A5A21184808F004FD01
:10C3A000FB69002B20D008220021F8690FF088FFDC
:10C3B0007B681A78FB691A7007F10803184600F0C9
:10C3C0007FFF01233B727B68191D07F108030433CB
:10C3D000102218460FF066FF07F10803184600F018
:10C3E000D3FF0246FB695A60FB6918462037BD46F9
:10C3F00080BD00BF90F20100ECF20100A0F201004C
:10C40000B8F2010080B586B000AF78607B681B7819
:10C41000072B00F2308101A252F823F07BC6000006
:10C420003DC4000065C400007BC400009FC4000040
:10C4300073C500001BC6000055C600007B68DB68A2
:10C44000002B05D17B685B6A984702467B68DA60FF
:10C450007B6800221A617B6800225A617B68022295
:10C460001A7011E17B689B6A7A68D26811460020D5
:10C4700098477B6803221A7006E17B681A697B681B
:10C480005B681A447B681A617B681A697B689B69E0
:10C490009A42C0F0F4807B6804221A70ECE07B685A
:10C4A0001A697B685B681A447B681A617B685B6AFF
:10C4B000984778617B69002B03D17B6806221A704C
:10C4C000DAE07B68DB687A699A422AD17B681A696C
:10C4D0007B681B6A9A420ED37B689B6A7A68D26833
:10C4E0001146022098477B681A697B685A617B680D
:10C4F00005221A70C8E07B681A697B685B69D21AEA
:10C500007B68DB699A4240F2BC807B689B6A7A68F0
:10C51000D2681146012098477B681A697B685A6186
:10C52000AFE07B68DB68DB437A691340FB60FB6844
:10C53000002B08D07B689B6AF968002098477B68CD
:10C540001A697B685A617B68DA687B69DB43134050
:10C55000FB60FB68002B08D07B689B6AF9680420AD
:10C5600098477B681A697B685A617B687A69DA60E8
:10C570008AE07B681A697B685B681A447B681A6189
:10C580007B685B6A984778617B69002B03D17B6885
:10C5900006221A7070E07B68DB687A699A4214D1CF
:10C5A0007B681A697B685B69D21A7B68DB699A428F
:10C5B00069D97B689B6A7A68D268114603209847DC
:10C5C0007B681A697B685A615DE07B68DB68DB43E6
:10C5D0007A6913403B613B69002B08D07B689B6AFA
:10C5E0003969002098477B681A697B685A617B68C3
:10C5F000DA687B69DB4313403B613B69002B08D061
:10C600007B689B6A3969052098477B681A697B6853
:10C610005A617B687A69DA6036E07B681A697B6800
:10C620001B6A9A4207D37B689B6A7A68D268114674
:10C630000520984706E07B689B6A7A68D2681146B5
:10C64000042098477B681A697B685A617B680722D7
:10C650001A7011E07B689B6A7A68D26811460620DE
:10C6600098477B680022DA607B6800221A617B6849
:10C6700000221A7008E000BFC8E600BF04E000BF57
:10C6800002E000BF00E000BF1837BD4680BD00BF1C
:10C6900080B483B000AF0346FB7197F90730002BDD
:10C6A0000BDBFB7903F01F02074997F907305B09A1
:10C6B000012000FA02F241F8232000BF0C37BD46EA
:10C6C0005DF8047B704700BF00E100E080B483B0F8
:10C6D00000AF03463960FB7197F90730002B0ADB86
:10C6E0003B68DAB20C4997F907301201D2B20B4419
:10C6F00083F800230AE03B68DAB20849FB7903F0CB
:10C700000F03043B1201D2B20B441A7600BF0C3760
:10C71000BD465DF8047B704700E100E000ED00E0FD
:10C7200080B483B000AF7860044A7B68136000BFB8
:10C730000C37BD465DF8047B704700BFE81B002046
:10C7400080B400AF034B1B681846BD465DF8047B00
:10C75000704700BFE81B002080B500AF034B1B688B
:10C760000021184600F0ECFD00BF80BDD81B002062
:10C7700080B500AF034B1B68184600F0BFFD00BF3B
:10C7800080BD00BFD81B002080B500AF034B1B68E5
:10C790000021184600F0D4FD00BF80BDDC1B002046
:10C7A00080B500AF034B1B68184600F0A7FD00BF23
:10C7B00080BD00BFDC1B002080B588B004AF0346FD
:10C7C000FB71FB79704A12781146704A1278029216
:10C7D000019100936E4B71226E49002001F0BCF96B
:10C7E000694B1B78FA799A4200F0CA806A4B1B7831
:10C7F000002B04D0684B1B78012B40F0BA8000233B
:10C80000FB73FB7903F00103002B03D0FB7B43F0A8
:10C810000203FB73FB7903F00203002B03D0FB7BC5
:10C8200043F00103FB73FB79FA7B019200935B4BAE
:10C8300084225849002001F08FF9FB7B032B7DD027
:10C84000032B03DC012B2BD0022B2CD0FFF790FF06
:10C85000534B1B68534AA2FB03239B0C642202FB2D
:10C8600003F3002B19D04E4B1B684E4AA2FB032347
:10C870009B0C642202FB03F30A2B02D80EF051F842
:10C880000BE0474B1B68474AA2FB03239B0C642227
:10C8900002FB03F3184602F017FFFFF781FF51E098
:10C8A000FFF772FF4EE0404B1B6818460CF033FF59
:10C8B0000346002B1AD03D4B1B6818460CF02BFF8B
:10C8C0000346002B09D03A4B01221A70394B9622AD
:10C8D0003049002001F040F908E0354B00221A7081
:10C8E000354B99222B49002001F036F9FFF740FF24
:10C8F0002B4B1B682B4AA2FB03239B0C642202FBDD
:10C9000003F3002B1DD0264B1B68264AA2FB0323F2
:10C910009B0C642202FB03F30A2B02D80EF001F8F1
:10C920000FE01F4B1B681F4AA2FB03239B0C6422D2
:10C9300002FB03F3184602F0C7FE02E0FFF70CFF0C
:10C9400000E000BFFB79002B13D10F4B1B78022BAB
:10C950000FD10E4B1B78002B0BD1184BAA220D497F
:10C96000022001F0F9F8164B01221A70104B002238
:10C970001A70054B1A78054B1A70034AFB7913702D
:10C9800000BF1037BD4680BD4E0200204F02002080
:10C9900000F3010024F30100E235002030F3010030
:10C9A000E001002083DE1B43D81B0020DC1B00209D
:10C9B000E335002048F3010068F3010060F3010053
:10C9C0004C02002080B582B000AF0346FB71054BDE
:10C9D0001868F91D002300220EF08FFC00BF0837F5
:10C9E000BD4680BDE41B002080B400AF024B18465A
:10C9F000BD465DF8047B704770F3010080B584B0DC
:10CA000000AF0023FB6012480BF013FEF860FB68D8
:10CA100003F02803002B14D00D480CF0ABFD0346A7
:10CA2000FB720C4B18683A1D07F10B0100230EF046
:10CA300072FD7B68002B04D0BFF34F8F00BF05F061
:10CA400087FDBFF34F8F00BF00BF1037BD4680BDCD
:10CA500000B00640E01B002080B582B000AF7860D7
:10CA60007B685B681A46204920480DF097F97B687F
:10CA70005B681A461E491F480DF090F97B685B6899
:10CA80001A461D491D480DF089F97B685B681A46F6
:10CA90001B491C480DF082F97B685B681A461A49ED
:10CAA0001A480DF07BF97B685B681A4618491948EB
:10CAB0000DF074F97B685B681A46174917480DF04A
:10CAC0006DF97B685B681A46154916480DF066F9E2
:10CAD0007B685B681A46144914480DF05FF900231F
:10CAE00018460837BD4680BD84F30100ACF3010051
:10CAF000B4F30100A4D00100D4F3010080E70100E9
:10CB0000F0F3010010F4010028F401004CF40100DE
:10CB100064F401008CF40100A0F40100B8F40100F9
:10CB2000D0F40100F8F4010010F5010038F501001F
:10CB300080B592B000AF78607B685B681A464B495D
:10CB40004B480DF03DF94B4B1B6807F108014022A3
:10CB5000184600F03BFD07F10803474A40211846FC
:10CB60000DF04AFA7B685A6807F1080319464348F2
:10CB70000DF026F9424B1B6807F1080140221846C8
:10CB800000F024FD07F108033B4A402118460DF050
:10CB900033FA7B685A6807F10803194639480DF0E3
:10CBA0000FF9394B1B78012B1AD107F10803374ACB
:10CBB000402118460DF0FBF9354B1B78002B07D0B0
:10CBC00007F10803334A402118460DF015FA26E014
:10CBD00007F10803284A402118460DF00DFA1EE01F
:10CBE000294B1B78002B07D107F108032A4A402163
:10CBF00018460DF0DCF912E0234B1B78022B07D10D
:10CC000007F10803254A402118460DF0D0F906E047
:10CC100007F10803224A402118460DF0C8F97B6845
:10CC20005A6807F1080319461E480DF0C9F81E4B53
:10CC30001B78002B01D01D4900E01D497B685B6813
:10CC40001A461C480DF0BCF8114B1B78002B01D084
:10CC5000194900E011497B685B681A4617480DF0D6
:10CC6000AFF8002318464837BD4680BD48F501009F
:10CC7000ACF30100D81B0020D4DE010058F5010000
:10CC8000DC1B002060F50100E235002068F50100A2
:10CC90004D0200206CF5010094F5010040FD0100FB
:10CCA00024D201009CF50100E33500201CE20100C4
:10CCB00024E20100A8F501000CE30100B8F5010031
:10CCC00090B5A7B000AFF860B9607A609749F8688E
:10CCD0000FF0D7FB0346002B06D09549F8680FF0FC
:10CCE000D0FB0346002B07D1BB6801221A7078687D
:10CCF000FFF7B2FE034614E18E49F8680FF0C1FB5E
:10CD00000346002B06D08C49F8680FF0BAFB0346A7
:10CD1000002B07D1BB6801221A707868FFF708FF63
:10CD20000346FEE08549F8680FF0ABFB0346002B95
:10CD300006D1BB6801221A700CF029FC0023F0E038
:10CD40007F49F8680FF09DFB0346002B10D1BB68AC
:10CD500001221A70FFF718FD012005F0C7FD0CF045
:10CD600016FC012005F0C2FDFFF71AFD0023D8E0F4
:10CD70007449F8680FF085FB0346002B0BD1BB68A4
:10CD800001221A70FFF70CFD012005F0AFFD0CF039
:10CD9000FEFB0023C5E06C49F8680FF072FB034608
:10CDA000002B06D1BB6801221A70FFF7EDFC0023AF
:10CDB000B7E06649F8680FF064FB0346002B06D124
:10CDC000BB6801221A70FFF7EBFC0023A9E0604961
:10CDD000F8680FF056FB0346002B06D1BB68012212
:10CDE0001A70FFF7B9FC00239BE05A49F8680FF06E
:10CDF00048FB0346002B06D1BB6801221A70FFF7DF
:10CE0000B7FC00238DE05449F8680FF03AFB034665
:10CE1000002B07D1BB6801221A70504B01221A70F7
:10CE200000237EE04E49F8680FF02BFB0346002BF1
:10CE300007D1BB6801221A70484B00221A700023E8
:10CE40006FE04849F8680FF01CFB0346002B0AD13D
:10CE5000BB6801221A70444B00221A70434B002217
:10CE60001A7000235DE04249F8680FF00AFB0346A0
:10CE7000002B0AD1BB6801221A703B4B01221A70A9
:10CE80003A4B01221A7000234BE03A49F8680FF040
:10CE9000F8FA0346002B0AD1BB6801221A70324B04
:10CEA00002221A70314B00221A70002339E00B2243
:10CEB0003149F8680FF0FFFA0346002B30D1BB6808
:10CEC00001221A70FB680B33C7F89430D7F89430FE
:10CED0001B78222B10D107F1140107F19403802253
:10CEE00018460DF06FFC0346002B01D01B2318E001
:10CEF00007F11403C7F89430D7F89440FFF774FD96
:10CF000003465B68194620460CF014FDFFF76CFDE4
:10CF100003465B68194619480CF00CFD002300E03D
:10CF2000002318469C37BD4690BD00BF60FC010041
:10CF3000C8F5010070FC0100D4F50100E4F5010022
:10CF4000F0F5010000F6010010F6010020F60100E6
:10CF500034F6010048F6010060F601004D020020A1
:10CF600078F6010090F60100E2350020E33500205C
:10CF7000A4F60100B4F60100C8F60100D4DE0100F9
:10CF800080B586B000AF78601B4B1B6807F10F01BE
:10CF90004FF0FF3218460EF06FFB78617B69012B72
:10CFA00022D1F5F75DFC0346002B04D0134B5B68E0
:10CFB000FA7B10469847124B1B78002BE4D0114B9C
:10CFC0001B7883F00103DBB2002BDDD0FFF7B8FB49
:10CFD00038613B69002BD7D0FA7B3B695B68194607
:10CFE00010460CF095FCCFE7074B40F28F12074933
:10CFF000052000F0B1FDC7E7E01B002068C6010076
:10D000004D020020E3350020D4F6010024F3010096
:10D0100080B586B000AF7860304B1B78002B0BD00A
:10D020002E4B00221A702E4B4FF4CF722D49022046
:10D0300000F092FD0CF0ABFA0023FB752A4B1B6845
:10D0400007F10B01002218460EF016FB38613B6910
:10D05000012B08D10123FB7507F10B0301221946AF
:10D0600022480BF04FFB3B69012BE7D026E0012360
:10D07000FB751F4B1B6807F10B021046984707F121
:10D080000B030122194619480BF03CFB194B1B7886
:10D09000002B13D0184B1B7883F00103DBB2002B5D
:10D0A0000CD0FFF74DFBF860FB68002B06D0FA7A36
:10D0B000FB685B68194610460CF02AFC0C4BDB68D9
:10D0C00098470346002BD2D1FB7D83F00103DBB2EE
:10D0D000002BA1D0052005F009FC9DE74C020020A3
:10D0E000F4F6010024F30100E41B002000B0064028
:10D0F00068C601004D020020E335002080B584B0F1
:10D1000000AF3B1D1846F8F7CDF84FF4E1337B60D4
:10D110000123FB730123BB730020F6F703FA0246D9
:10D120003B1D19462548F7F75FFF4FF402212348BE
:10D13000F8F7ECF821200CF007FA05212120FFF781
:10D14000C5FA032001F018FF002201214FF480509E
:10D150000EF063F803461A4A1360194B1B68002B44
:10D1600007D1184B40F2D1121749052000F0F4FC0A
:10D17000FEE7134B1B681549184605F099FA002283
:10D1800001214FF480500EF048F80346104A136016
:10D190000F4B1B68002B07D10E4B4FF4EC720A4962
:10D1A000052000F0D9FCFEE7094B1B680A49184628
:10D1B00005F07EFA00BF1037BD4680BD00B00640C6
:10D1C000E01B002008F7010024F3010024F7010010
:10D1D000E41B002038F7010054F7010080B586B049
:10D1E00000AF3B1D184600F06BF801233B710F4B5D
:10D1F000BB600F4BFB600C233B613B1D184600F0EE
:10D20000C3F803460B4A1360084BBB60084BFB6036
:10D2100005233B613B1D184600F0B6F80346064A5D
:10D22000136000BF1837BD4680BD00BF00F00F403F
:10D2300000900440D81B0020DC1B002080B582B089
:10D2400002AFFFF7CBFFFFF759FF00230193032342
:10D25000009300237D22134913480EF0F5FD034689
:10D26000012B07D0114B40F205221149052000F097
:10D2700073FCFEE7002301930323009300237D2228
:10D280000C490D480EF0E0FD0346012B07D00B4B77
:10D2900040F211220649052000F05EFCFEE700BFC7
:10D2A000BD4680BD68F7010081CF000074F7010022
:10D2B00024F3010094F7010011D00000A0F7010051
:10D2C00080B582B000AF78607B68002B05D1074B3A
:10D2D000074A6721074807F067FD14220649786866
:10D2E0000EF0E0FF00BF0837BD4680BD90F20100A0
:10D2F0002CF80100D4F70100C0F7010080B584B01C
:10D3000000AF78607B68FB607B68002B05D1094B20
:10D31000094ABC21094807F047FD00220121F868AD
:10D320000CF0AEF9FB6801221A7000BF1037BD4641
:10D3300080BD00BFE0F7010048F80100D4F701000C
:10D3400080B584B000AF78600B46FB707B68FB60F3
:10D350007B68002B05D1094B094AC421094807F015
:10D3600023FDFB781A460021F8680CF089F9FB6868
:10D3700000221A7000BF1037BD4680BDE0F70100E3
:10D380005CF80100D4F7010080B584B000AF78608C
:10D390007B68002B05D1214B214AE021214807F071
:10D3A00003FD142004F0D2FDF860FB68002B05D1CA
:10D3B0001D4B1B4AE7211B4807F0F6FCFB68002BBE
:10D3C00010D014220021F8680EF07AFF7B681A78DA
:10D3D000FB681A70FB68181D7B680433102219461D
:10D3E0000EF060FF7B6819787B685B781A46F868F6
:10D3F0000CF046F97B681B7C1946F8680CF0A2F922
:10D400007B6898687B68DB68012219460CF01BF981
:10D41000FB6818461037BD4680BD00BF90F2010082
:10D4200070F80100D4F70100B8F2010080B584B0B3
:10D4300000AF78607B68002B06D10C4B0C4A4FF490
:10D44000A2710C4807F0B0FC7B68FB60FB685A686F
:10D45000FB68DB68012101FA03F3194610460CF062
:10D46000C4F800BF1037BD4680BD00BFE0F7010023
:10D4700084F80100D4F7010080B584B000AF786073
:10D480007B68002B06D10C4B0C4A4FF4AF710C4853
:10D4900007F08AFC7B68FB60FB685A68FB68DB6806
:10D4A000012101FA03F3194610460CF090F800BF71
:10D4B0001037BD4680BD00BFE0F7010094F80100C1
:10D4C000D4F7010080B584B000AF78607B68002B92
:10D4D00006D10C4B0C4A4FF4BC710C4807F064FCAD
:10D4E0007B68FB60FB685A68FB68DB68012101FA16
:10D4F00003F3194610460CF086F800BF1037BD46FE
:10D5000080BD00BFE0F70100A4F80100D4F70100DE
:10D5100080B584B000AF78600B46FB707B68002B51
:10D5200006D1134B134A40F29711134807F03CFC05
:10D530007B68FB60FB78002B0BD0FB685A68FB68AC
:10D54000DB68012101FA03F3194610460CF03FF89D
:10D550000AE0FB685A68FB68DB68012101FA03F303
:10D56000194610460CF041F800BF1037BD4680BD8B
:10D57000E0F70100B4F80100D4F7010080B584B0F1
:10D5800000AF78607B68002B06D10D4B0D4A4FF43D
:10D59000E5710D4807F008FC7B68FB60FB685A6882
:10D5A000FB68DB68194610460CF03BF80346002B7D
:10D5B00014BF01230023DBB218461037BD4680BDDF
:10D5C000E0F70100C8F80100D4F7010080B586B08B
:10D5D00000AFF860B9607A60FB687B61BB680022CD
:10D5E0001A70F8680CF072F80346002B05D0224A36
:10D5F0007968B8680CF000FD04E0204A7968B868E2
:10D600000CF0FAFCF868FFF7B9FF0346002B05D0D1
:10D610001B4A7968B8680CF0EFFC04E0194A796895
:10D62000B8680CF0E9FC184A7968B8680CF0E4FCBA
:10D630007B695B681A467968B8680CF0CFFE134ABC
:10D640007968B8680CF0D8FC7B699B681A467968E1
:10D65000B8680CF0C3FE0E4A7968B8680CF0CCFCD0
:10D660007B69DB681A467968B8680CF005FF00BF73
:10D670001837BD4680BD00BFECF70100F4F701008C
:10D68000FCF7010004F801000CF8010018F8010093
:10D6900024F8010080B483B000AF78607B681B6819
:10D6A000214A13607B6804331B68204A13607B683F
:10D6B00008331B681E4A13607B680C331B681D4AC5
:10D6C00013607B6810331B681B4A13607B6814333C
:10D6D0001B681A4A13607B6818331B68184A13606A
:10D6E0007B681C331B68174A1360174B1B68174A6B
:10D6F0001360174B1B68174A1360174B1B68174AB8
:10D700001360174B1B68174A1360174B1B68174AA7
:10D710001360174B1B68174A136000BE00BF0C371D
:10D72000BD465DF8047B7047EC1B0020F01B002019
:10D73000F41B0020F81B0020FC1B0020001C002014
:10D74000041C0020081C002028ED00E00C1C002018
:10D750002CED00E0101C002030ED00E0141C002037
:10D760003CED00E0181C002034ED00E01C1C002003
:10D7700038ED00E0201C002080B582B000AF78605A
:10D780007B68002B05D1074B074A3E21074807F06D
:10D790000BFB1422064978680EF084FD00BF0837A1
:10D7A000BD4680BD90F2010004F90100ECF80100D3
:10D7B000D8F8010080B58AB000AF78607B68002B94
:10D7C00005D1294B294A4721294807F0EDFA07F1ED
:10D7D0000C031846FFF774FD00233B737B68191D8B
:10D7E00007F10C030433102218460EF05BFD7B6832
:10D7F0001B78002B0ED07B685B78002B14BF0123B5
:10D800000023DBB283F00103DBB203F00103DBB2E0
:10D810007B7302E07B685B787B7307F10C0318462F
:10D82000FFF7B2FD7862082004F090FB38623B6A93
:10D83000002B05D10F4B0D4A56210D4807F0B4FAC5
:10D840003B6A002B0BD008220021386A0EF038FD0D
:10D850003B6A7A6A1A607B681A783B6A1A713B6A7B
:10D8600018462837BD4680BD90F201001CF9010022
:10D87000ECF80100B8F2010080B584B000AF786028
:10D880007B68002B05D10D4B0D4A6B210D4807F02D
:10D890008BFA7B68FB60FB681B79002B05D0FB686B
:10D8A0001B681846FFF7C2FD04E0FB681B681846BA
:10D8B000FFF7E2FD00BF1037BD4680BDF8F801005C
:10D8C0002CF90100ECF8010080B584B000AF78605D
:10D8D0007B68002B05D10D4B0D4A76210D4807F0D2
:10D8E00063FA7B68FB60FB681B79002B05D0FB6843
:10D8F0001B681846FFF7C0FD04E0FB681B6818466C
:10D90000FFF794FD00BF1037BD4680BDF8F8010059
:10D9100038F90100ECF8010080B584B000AF786000
:10D920007B68002B05D1084B084A8121084807F085
:10D930003BFA7B68FB60FB681B681846FFF7C2FD7B
:10D9400000BF1037BD4680BDF8F8010044F9010062
:10D95000ECF8010080B500AF064B9B68002B06D0A9
:10D96000044B9B68034AD26801211046984700BFC8
:10D9700080BD00BF241C002080B500AF064B9B6813
:10D98000002B06D0044B9B68034AD2680021104646
:10D99000984700BF80BD00BF241C002080B590B018
:10D9A00002AFF860B96011461A460B46FB71134688
:10D9B000BB7100233B7407F11000604BFA68202113
:10D9C0000CF081FA07F110032022202118460CF0F8
:10D9D00046FB07F110005A4BBA6820210CF0A4FA5C
:10D9E00007F110032022202118460CF038FB07F124
:10D9F0001003FA6CB96C18460BF032FF00233B742D
:10DA0000BB79002B0DD04F4B5B7D002B09D0FB79F0
:10DA10004D4A52F8232007F11003202118460CF03C
:10DA2000EBFAFB79494A52F8232007F1100006234C
:10DA30000093202320210CF012FFBB79002B0AD089
:10DA4000404B5B7D002B06D007F11003404A20219C
:10DA500018460CF0D1FA07F11003FA6CB96C1846AD
:10DA60000BF0FEFE3B6C7B637B6B1B782E2B0CD18B
:10DA700002E07B6B01337B637B6B1B78202BF8D040
:10DA80007B6B1B782E2BF4D031E0386C0EF00BFD45
:10DA90000346013B3B6302E03B6B013B3B633B6B5B
:10DAA000012B0DD93B6B013B3A6C13441B782F2B98
:10DAB00006D03B6B013B3A6C13441B785C2BEBD1DB
:10DAC0003B6B012B0FD13B6B013B3A6C13441B7832
:10DAD0002F2B08D03B6B013B3A6C13441B785C2B1B
:10DAE00001D000233B633A6C3B6B13447B63FA6CBD
:10DAF000B96C786B0BF0B4FE00233B7407F1100394
:10DB00003A22202118460CF0AAFA7A6C07F1100389
:10DB1000202118460CF0B0FC07F110030D4A20211B
:10DB200018460CF069FA07F11003FA6CB96C184644
:10DB30000BF096FE00BF3837BD4680BDDCF9010012
:10DB4000E8F90100241C0020C4F90100ACF901002F
:10DB5000F4F9010048DE010008B480B58DB004AFCF
:10DB60000346B9607A60FB732E4B1B78FA7B9A42AE
:10DB700051D3FFF7EFFE07F1180207F11403114626
:10DB800018460CF090F9274B1B7D83F00103DBB2A4
:10DB9000002B3DD00023FB6137E0224AFB690433B0
:10DBA00052F82330002B2DD01E4AFB69043352F863
:10DBB00023309B68FA7B07F1140107F118000393E7
:10DBC000194B02937B680193BB6800930123FFF715
:10DBD000E5FE07F130033B61124AFB69043352F85A
:10DBE000233099683B69FA6A0F4801F013FE0D4A29
:10DBF000FB69043352F823309B681A460A490B48E4
:10DC00000BF02EFEFB690133FB61FB69002BC4DDC9
:10DC1000FFF7B2FE00E000BF2437BD46BDE88040FC
:10DC200001B07047241C002041980100A8DE0100CB
:10DC300080B584B000AF78607B68002B05D10B4BBA
:10DC40000B4A23210B4807F0AFF8EFF3108072B6B0
:10DC5000F8730822084978680EF024FBF87B80F3FB
:10DC6000108800BF1037BD4680BD00BF90F2010094
:10DC700044FA010004FA0100FCF9010080B584B007
:10DC800000AF78607B68002B05D11F4B1F4A2E2107
:10DC90001F4807F089F8182004F058F9F860FB686D
:10DCA000002B05D11B4B194A3421194807F07CF889
:10DCB000FB68002B22D018220021F8680EF000FB30
:10DCC0007B685A68FB685A607B681A68FB681A6050
:10DCD000FB681B68FA68526802FB03F3184604F0FD
:10DCE00035F90246FB685A61FB685B69002B05D178
:10DCF000094B064A3E21064807F056F8FB681846CD
:10DD00001037BD4680BD00BF90F201005CFA0100F3
:10DD100004FA0100B8F201000CFA010080B584B0E9
:10DD200000AF78607B68FB607B68002B05D1064BF9
:10DD3000064A5821064807F037F8FB689B681846E2
:10DD40001037BD4680BD00BF20FA01006CFA01000B
:10DD500004FA010080B586B000AF786039607B6856
:10DD60003B6100237B617B68002B02D03B68002B6A
:10DD700005D11F4B1F4A74211F4807F015F8EFF318
:10DD8000108072B6F8733B699A683B691B689A42C7
:10DD900002D104237B6121E03B695A693B69DB685E
:10DDA0003969496801FB03F3D0183B695B681A467F
:10DDB00039680EF077FA3B69DB685A1C3B69DA6018
:10DDC0003B69DA683B691B689A4202D13B690022D1
:10DDD000DA603B699B685A1C3B699A60F87B80F368
:10DDE00010887B69DBB218461837BD4680BD00BF7E
:10DDF0002CFA010080FA010004FA010080B586B017
:10DE000000AF786039607B683B6100237B617B6891
:10DE1000002B02D03B68002B05D11E4B1E4A9921D6
:10DE20001E4806F0C1FF3B699B68002B02D1092305
:10DE30007B6128E03B695A693B691B69396949681C
:10DE400001FB03F3D1183B695B681A4638680EF092
:10DE500029FAEFF3108072B6F8733B699B685A1E7B
:10DE60003B699A603B691B695A1C3B691A613B69B3
:10DE70001A693B691B689A4202D13B6900221A6108
:10DE8000F87B80F310887B69DBB218461837BD46F3
:10DE900080BD00BF2CFA01008CFA010004FA0100D9
:10DEA00090B5B9B002AF7860002387F8D330002373
:10DEB0003B7307F10C00042300932023B54A202173
:10DEC0000CF0CDFC7B685A6807F10C03114618462C
:10DED0000BF030FD00233B7307F10C000723009388
:10DEE0002023AD4A20210CF0BAFC7B685A6807F168
:10DEF0000C03114618460BF01DFD00233B7307F180
:10DF00000C000B2300932023A44A20210CF0A7FC33
:10DF10007B685A6807F10C03114618460BF00AFD9E
:10DF200000233B7307F10C000D23009320239C4A30
:10DF300020210CF094FC7B685A6807F10C03114611
:10DF400018460BF0F7FC00233B7307F10C00092384
:10DF500000932023934A20210CF081FC7B685A68AF
:10DF600007F10C03114618460BF0E4FC00233B7349
:10DF700007F10C000823009320238B4A20210CF08A
:10DF80006EFC7B685A6807F10C03114618460BF0CB
:10DF9000D1FC00233B7307F10C000B2300932023DB
:10DFA000824A20210CF05BFC7B685A6807F10C0365
:10DFB000114618460BF0BEFC00233B7307F10C0022
:10DFC0000B23009320237A4A20210CF048FC7B6825
:10DFD0005A6807F10C03114618460BF0ABFC0023FE
:10DFE0003B7307F10C00082300932023714A202182
:10DFF0000CF035FC7B685A6807F10C031146184693
:10E000000BF098FC00233B7307F10C0015230093E1
:10E010002023694A20210CF022FC7B685A6807F112
:10E020000C03114618460BF085FC00233B7307F1E7
:10E030000C00082300932023604A20210CF00FFCE1
:10E040007B685A6807F10C03114618460BF072FC06
:10E0500000233B7307F10C00112300932023584A3F
:10E0600020210CF0FCFB7B685A6807F10C03114679
:10E0700018460BF05FFC7B685B68194651480BF053
:10E0800059FC04F0CDFDC7F8CC00D7F8CC304E4A8F
:10E09000A2FB03235B09C7F8CC3004F0D3FDC7F81B
:10E0A000C800D7F8C830102B11D907F10C03474A24
:10E0B000202118460BF07BFF7B689A6807F10C0360
:10E0C000114618460BF036FC1023C7F8C83007F18C
:10E0D00080031021184605F0C7FCC7F8C8000023CC
:10E0E000C7F8D430CFE2D7F8D4309B00D8333B44C4
:10E0F00053F8583C002B00F0C182D7F8D4309B0075
:10E10000D8333B4453F8580C07F12C010523012266
:10E1100005F0CAF8D7F8D4309B00D8333B4453F805
:10E12000580C07F1740407F1780207F17C0107F13C
:10E1300073030093234605F0E5FC002387F8503075
:10E140007A6B07F15003202118460CF095F9002353
:10E150003B7307F1500207F10C00042300932023C6
:10E1600020210CF07CFB7B685A6807F10C031146F8
:10E1700018460BF0DFFB002387F8503097F8733018
:10E18000002B27D107F15003114A202118460BF02C
:10E190000EFF35E09CFA0100A0FA0100A8FA010088
:10E1A000B0FA0100B8FA0100C0FA0100C8FA010093
:10E1B000D4FA0100E0FA0100E8FA0100F4FA0100E3
:10E1C000FCFA0100D4DE01001F85EB5104FB0100C5
:10E1D00040FB010007F15003584A202118460BF07C
:10E1E000E6FE97F8732007F15003202118460CF043
:10E1F00000F807F15003524A202118460BF0FCFEAC
:10E2000000233B7307F1500207F10C000723009332
:10E21000202320210CF023FB7B685A6807F10C03B4
:10E22000114618460BF086FB07F15003454A2021A2
:10E2300018460BF0BCFED7F8D4309B00D8333B44D3
:10E2400053F8583C1A4607F15003202118460CF0A9
:10E25000C5F800233B7307F1500207F10C000B23B4
:10E260000093202320210CF0FAFA7B685A6807F10A
:10E270000C03114618460BF05DFB00233B73D7F8E7
:10E28000D4309B00D8333B4453F8583C184604F034
:10E29000E5FC024607F10C000D230093202320210A
:10E2A0000CF0DDFA7B685A6807F10C03114618463A
:10E2B0000BF040FB97F83830052B51D801A252F8EB
:10E2C00023F000BFDDE20000EDE200000DE30000FE
:10E2D000FDE200001DE300002DE3000007F1500304
:10E2E000194A202118460BF062FE41E007F1500365
:10E2F000164A202118460BF05AFE39E007F1500368
:10E30000134A202118460BF052FE31E007F150036A
:10E31000104A202118460BF04AFE29E007F150036D
:10E320000D4A202118460BF042FE21E007F1500370
:10E330000A4A202118460BF03AFE19E048FB01007A
:10E3400050E9010004EA010050FB010058FB010004
:10E3500060FB01006CFB010074FB01007CFB010011
:10E3600007F15003CE4A202118460BF020FE00BFD3
:10E3700000233B7307F1500207F10C0009230093BF
:10E38000202320210CF06BFA7B685A6807F10C03FC
:10E39000114618460BF0CEFA002387F8503007F1EB
:10E3A00050032822202118460BF059FE3A6C07F141
:10E3B0005003202118460CF05FF807F150032C227F
:10E3C000202118460BF04BFEFA6B07F15003202179
:10E3D00018460CF051F807F1500329222021184665
:10E3E0000BF03DFE00233B7307F1500207F10C00D8
:10E3F00008230093202320210CF031FA7B685A680F
:10E4000007F10C03114618460BF094FA07F150037C
:10E41000A44A202118460BF0CAFDFB6F1A4607F1EB
:10E420005003202118460BF0D9FF00233B7307F15E
:10E43000500207F10C000B230093202320210CF045
:10E440000EFA7B685A6807F10C03114618460BF068
:10E4500071FA07F15003934A202118460BF0A7FDEB
:10E46000BB6F1A4607F15003202118460BF0B6FF88
:10E4700000233B7307F1500207F10C000B230093BC
:10E48000202320210CF0EBF97B685A6807F10C037C
:10E49000114618460BF04EFAFB6F1A46BB6FD31AA3
:10E4A0009BB20833A7F8C630002387F85030B7F87E
:10E4B000C62007F1500005230093202320210BF0F4
:10E4C000E4FE07F15003784A202118460BF094FD32
:10E4D00000233B7307F1500207F10C00082300935F
:10E4E000202320210CF0BBF97B685A6807F10C034C
:10E4F000114618460BF01EFA07F15003694A202115
:10E5000018460BF054FD7B6F1A4607F1500320218B
:10E5100018460BF063FF07F15003644A20211846A8
:10E520000BF06AFDFB6F1A467B6FD31A9BB2043364
:10E530009AB207F1500005230093202320210BF00D
:10E54000A4FE07F150035A4A202118460BF054FD4F
:10E5500000233B7307F1500207F10C0015230093D1
:10E56000202320210CF07BF97B685A6807F10C030B
:10E57000114618460BF0DEF9002387F85030B7F843
:10E580004C309B009AB207F15000052300932023E2
:10E5900020210BF07AFE07F15003434A2021184650
:10E5A0000BF02AFD00233B7307F1500207F10C002A
:10E5B00008230093202320210CF051F97B685A682E
:10E5C00007F10C03114618460BF0B4F907F150039C
:10E5D000344A202118460BF0EAFC7A6C07F150030C
:10E5E000202118460BF0FAFED7F8CC30002B2BD0A8
:10E5F0007A6CD7F8CC30B2FBF3F3C7F8C030D7F859
:10E60000C030002B19D007F15003284A20211846AA
:10E610000BF0F2FCD7F8C0309AB207F15000032398
:10E620000093202320210BF030FE07F15003214AF4
:10E63000202118460BF0E0FC06E007F150031E4ACB
:10E64000202118460BF0D8FC00233B7307F1500241
:10E6500007F10C0011230093202320210CF0FFF878
:10E660007B685A6807F10C03114618460BF062F9F3
:10E670007B685B68194611480BF05CF9D7F8D43019
:10E680000133C7F8D430D7F8D420D7F8C8309A422D
:10E69000FFF429AD97F8D3301846DC37BD4690BD5E
:10E6A00084FB010004EA010090FB010094FB0100DF
:10E6B00098FB01009CFB0100A0FB0100D4DE0100DF
:10E6C00080B586B000AF78607B685B681A463349D6
:10E6D00033480BF075FB7B685B681A46314932485A
:10E6E0000BF06EFB7B685B68194630480BF022F933
:10E6F0007B685B681A462E492E480BF061FB07F1D8
:10E7000008034FF47A721021184600F0F1FD7B687F
:10E710005A6807F10803114618460BF00BF97B689D
:10E720005B68194624480BF005F907F1080301223C
:10E730001021184600F0DCFD7B685A6807F10803D9
:10E74000114618460BF0F6F87B685B6819461B48C3
:10E750000BF0F0F87B685B681A46154918480BF017
:10E760002FFB03F0EBFC024607F1080310211846CB
:10E7700000F0F6FE7B685A6807F108031146184658
:10E780000BF0D8F87B685B6819460E480BF0D2F89E
:10E79000002318461837BD4680BD00BFA8FB010006
:10E7A000C8FB0100D0FB0100D8FB0100D4DE010052
:10E7B0003CCF0100E4FB0100F4FB0100FCFB010085
:10E7C00004FC010010FC010080B582B000AF78604D
:10E7D0007B685B681A460B490B480BF0DFFA7B68D5
:10E7E0005B681A4609490A480BF0D8FA7B685B68EF
:10E7F0001A46084908480BF0D1FA00231846083792
:10E80000BD4680BD1CFC0100C8FB010054D20100C4
:10E81000A4D0010038FC01004CFC010080B584B09C
:10E8200000AFF860B9607A601F49F8680DF029FE02
:10E830000346002B06D01D49F8680DF022FE034662
:10E84000002B07D1BB6801221A707868FFF7BCFF64
:10E85000034625E01649F8680DF013FE0346002B29
:10E8600006D01449F8680DF00CFE0346002B07D1C2
:10E87000BB6801221A707868FFF722FF03460FE099
:10E880000D49F8680DF0FDFD0346002B07D1BB686C
:10E8900001221A707868FFF703FB034600E00023AB
:10E8A00018461037BD4680BD60FC010058FC0100D1
:10E8B00070FC010068FC010078FC010080B400AF2E
:10E8C000024B1846BD465DF8047B70478CFC010086
:10E8D00080B584B000AFF860B9607A604549F868E7
:10E8E0000DF0CFFD0346002B06D04349F8680DF02C
:10E8F000C8FD0346002B43D17B685B6819463F483F
:10E900000BF018F87B685B6819463D480BF012F86D
:10E910007B685B68194639480BF00CF87B685B68CC
:10E92000194638480BF006F87B685B68194633488F
:10E930000BF000F87B685B68194631480AF0FAFF73
:10E940007B685B6819462D480AF0F4FF7B685B68BA
:10E950001A462D492D480BF021FA7B685B681A4650
:10E960002B492C480BF01AFA7B685B681A462A4937
:10E970002A480BF013FABB6801221A70002334E016
:10E980002749F8680DF07DFD0346002B07D1BB68D1
:10E9900001221A70234B01221A70002325E022491C
:10E9A000F8680DF06EFD0346002B07D1BB6801220D
:10E9B0001A701C4B00221A70002316E01B49F868DD
:10E9C0000DF05FFD0346002B06D01949F8680DF0E5
:10E9D00058FD0346002B07D1BB6801221A707868E6
:10E9E00000F0F8F8034600E0002318461037BD4653
:10E9F00080BD00BF60FC0100A0FC0100D4DE01006E
:10EA0000B0FC0100F0FC010004FD010024FD010048
:10EA100054D20100A4D0010030FD010048FD0100E6
:10EA200058FD0100500200206CFD010070FC010047
:10EA300080FD010080B582B000AF78607B685B68C4
:10EA4000194606480AF076FF7B685B681946044859
:10EA50000AF070FF00BF0837BD4680BDD4DE01005C
:10EA600090FD010080B586B000AFF860B9607A60B3
:10EA70003B603B68DB6898470346002B00F09E80B4
:10EA80000023FB753B681B6807F117021046984787
:10EA9000FB7D002B00F08880FB7D082B02D0FB7DE6
:10EAA0007F2B21D1BA68FB689A427CD9464B1B78F0
:10EAB000002B0FD03B681B7C002B0BD03B685B68A6
:10EAC000082098473B685B68202098473B685B6854
:10EAD00008209847BB68013BBB60BB6800221A70E6
:10EAE0007B6801337B605EE0F87DBA68FB68D31A0F
:10EAF0001A4607F11603F9680AF062FF0346002B75
:10EB000023D007E00023FB753B681B6807F1170261
:10EB100010469847FB7D002BF4D12B4B1B78002B24
:10EB2000AED03B681B7C002BAAD03B685B681946C3
:10EB300026480AF0FFFE3868FFF77CFF3B685B68F9
:10EB40001946F8680AF0F6FE9AE71F4B1B78002B6F
:10EB500008D03B681B7C002B04D03B685B68FA7DC7
:10EB600010469847FA7DBB681A70BB680133BB60DA
:10EB70007B68013B7B60FB7D0D2B02D0FB7D0A2B6C
:10EB80000ED1114B1B78002B10D03B681B7C002B47
:10EB90000CD03B685B6819460D480AF0CBFE05E0D7
:10EBA0007B68012B04D96BE700BF02E000BF00E0E7
:10EBB00000BFBB6800221A70012300E00023184642
:10EBC0001837BD4680BD00BF50020020D4DE0100D2
:10EBD000A8DE010080B58AB000AF78607B685B6812
:10EBE0001A46444944480BF0EBF87B685B681A46C8
:10EBF000424943480BF0E4F87B685B68194641489A
:10EC00000AF098FE7B685B6819463F480AF092FE5E
:10EC10007B685B6819463D480AF08CFE3C4B1B78CC
:10EC2000002B01D03B4900E03B497B685B681A46FA
:10EC30003A480BF0C5F800233B7207F10803232282
:10EC4000202118460BF00BFA07F108032F4A202168
:10EC500018460BF0D1F97B685A6807F1080319468A
:10EC60002F480BF0ADF807F108032E4A2021184673
:10EC70000BF09DF907F108033B22202118460BF009
:10EC8000EEF907F10803284A202118460BF0B4F9E1
:10EC900007F108036022202118460BF0EDFB07F175
:10ECA00008031A4A202118460BF0A6F97B685A6817
:10ECB00007F1080319461D480BF082F807F1080315
:10ECC00080222021184600F04BFC07F10803184A67
:10ECD000202118460BF090F97B685A6807F1080369
:10ECE000194614480BF06CF8002318462837BD4627
:10ECF00080BD00BF98FD010024FD0100B4FD0100AE
:10ED0000C0FD0100F8FB0100C8FD0100D4DE0100D8
:10ED100050020020D4FD0100DCFD0100E4FD0100F3
:10ED2000ECFD0100F8FD010000FE01000CFE0100F9
:10ED300018FE010030FE010080B582B000AF78609F
:10ED400039603B689B68194612480AF0F3FD3B683E
:10ED50009B68194678680AF0EDFD3B689B68194688
:10ED60000D480AF0E7FD3B689B6819460B480AF01E
:10ED7000E1FD3B689B68194609480AF0DBFD3B68EA
:10ED80009B68194607480AF0D5FD00BF0837BD4605
:10ED900080BD00BF38FE0100D4DE010058FE010036
:10EDA00060FC010064FE010080B483B000AF7860B5
:10EDB000044A7B681360002318460C37BD465DF893
:10EDC000047B7047BC1C002080B400AF034B1B6861
:10EDD0001846BD465DF8047B704700BFBC1C002090
:10EDE00080B483B000AF0346FB7197F90730002B66
:10EDF0000BDBFB7903F01F02074997F907305B092A
:10EE0000012000FA02F241F8232000BF0C37BD4672
:10EE10005DF8047B704700BF00E100E080B483B080
:10EE200000AF03463960FB7197F90730002B0ADB0E
:10EE30003B68DAB20C4997F907301201D2B20B44A1
:10EE400083F800230AE03B68DAB20849FB7903F053
:10EE50000F03043B1201D2B20B441A7600BF0C37E9
:10EE6000BD465DF8047B704700E100E000ED00E086
:10EE700080B582B000AF0346FB71FB1D012219462D
:10EE8000034809F03FFC00BF0837BD4680BD00BF06
:10EE900000A0064080B584B000AF78600A4B1B68C4
:10EEA00007F10F01002218460CF0E6FB0346012B88
:10EEB00003D1FA7B7B681A7002E07B6800221A702B
:10EEC00000BF1037BD4680BDC01C002080B500AF1C
:10EED000064B1B6818460CF0D4FD0346002B14BFEC
:10EEE00001230023DBB2184680BD00BFC01C0020F8
:10EEF00080B584B000AF00233B601D4809F099FB4A
:10EF0000B860BB6803F08063002B01D00023FB7363
:10EF1000BB6803F02803002B15D0154B9B7DFB73BA
:10EF20000EE013480AF08EFF0346FB71114B186880
:10EF30003A46F91D00230CF0EEFAFB7B013BFB7314
:10EF4000FB7B002BEDD1BB6843F0806343F00803EB
:10EF50001946074809F090FB3B68002B01D003F0ED
:10EF6000F7FABFF34F8F00BF00BF1037BD4680BD1B
:10EF700000A00640C01C002080B582B000AF7860C1
:10EF80007B68022B03D07B68032B15D040E0022264
:10EF9000012122480AF063FF022202211F480AF0E1
:10EFA0005EFF1F4B03F580531B691D4A23F033039B
:10EFB00002F5805213612CE01A480AF013FF032275
:10EFC000002119480AF04BFF174B1B6823F0807390
:10EFD00023F00303144A43F00303136003220121C7
:10EFE00011480AF03CFF104B5B6823F0807323F05C
:10EFF00003030D4A43F003035360094B03F58053A9
:10F000001B69074A23F0330302F58052136100E0C5
:10F01000FEE700BF0837BD4680BD00BF009004403A
:10F02000007004400D00381000D0044080B584B05A
:10F0300000AF0AF031FF3B461846F6F733F94FF4BC
:10F04000E1333B600123FB720123BB720020F4F724
:10F0500069FA02463B4619460B48F5F7C5FFF860CA
:10F06000FB68002B00D0FEE74FF402210648F6F7BC
:10F070004DF905211F20FFF7D1FE1F200AF0CCFE1D
:10F0800000BF1037BD4680BD00A0064080B500AF70
:10F090000022012180200CF0C0F80346084A1360CA
:10F0A000074B1B68002B00D1FEE7054B1B68054989
:10F0B000184603F0FDFAFFF7B9FF00BF80BD00BF9F
:10F0C000C01C0020A0FE010080B586B000AF7860B3
:10F0D00039600023FB757B68002B14D0EFF31080A0
:10F0E00072B6B873184B1B683B61B87B80F310880D
:10F0F0007968386900F030F80346FB73FB7B002B1E
:10F1000001D00123FB753B68002B12D0EFF3108078
:10F1100072B6B8730D4B1A883B681A800C4B1A787C
:10F120003B689A700B4B1A783B68DA70B87B80F3B7
:10F130001088FB7D002B01D01B2300E00023184624
:10F140001837BD4680BD00BF441D0020D0350020CB
:10F15000E5350020E435002080B483B000AF78604E
:10F1600039607B68224AA2FB03235B0DDAB23B685D
:10F170001A707B681E4AA2FB0312520D1D4901FB47
:10F1800002F29B1A7B607B681B4AA2FB03239B0B4A
:10F19000DAB23B685A707B68174AA2FB0312920BE3
:10F1A0004EF6602101FB02F29B1A7B607B68134ADA
:10F1B000A2FB03239B09DAB23B689A707B680F4A73
:10F1C000A2FB031292094FF47A7101FB02F29B1A1F
:10F1D0007B607B680A4AA2FB0323DB08DAB23B6848
:10F1E000DA70002318460C37BD465DF8047B704783
:10F1F000B17C219580EE360073B2E745D34D6210A5
:10F20000CDCCCCCC80B489B000AFF860B9601346E7
:10F21000FB80FB68BB610023FB77BB68013BBB60E5
:10F22000FB88002B2CD1BB68002B29D0FB7F5A1CFC
:10F23000FA771A46BB69134430221A70BB68013B47
:10F24000BB601DE0FA88294BA3FB0213D9080B46CB
:10F250009B000B445B00D31A9BB2DAB2FB7F591CB4
:10F26000F9771946BB690B443032D2B21A70BB68C9
:10F27000013BBB60FB881D4AA2FB0323DB08FB802C
:10F28000FB88002B02D0BB68002BDBD10023BB77AF
:10F290001AE0BB7FBA6913441B78FB75FA7FBB7F0A
:10F2A000D31A013BBA691A44BB7FB9690B4412787F
:10F2B0001A70FA7FBB7FD31A013BBA691344FA7DF7
:10F2C0001A70BB7F0133BB77FB7F5B08DBB2BA7F71
:10F2D0009A42DED3FB7FBA69134400221A7000BF42
:10F2E0002437BD465DF8047B704700BFCDCCCCCC45
:10F2F00080B588B000AFF860B9601346FB80FB684A
:10F30000BB610023FB77FB88DB0BDBB2FB75B7F936
:10F31000063013F5004F05D1434AB968F8680AF082
:10F3200046FE7EE0BB68013BBB60FB7D002B03D04B
:10F33000FB885B429BB2FB80B7F90630002B32D1D1
:10F34000BB68002B2FD0FB7F5A1CFA771A46BB698B
:10F35000134430221A70BB68013BBB6023E0B7F94D
:10F360000620324B83FB02139910D317C91A0B46A0
:10F370009B000B445B00D31A1BB2DAB2FB7F591C13
:10F38000F9771946BB690B443032D2B21A70BB68A8
:10F39000013BBB60B7F90630244A82FB031292108E
:10F3A000DB17D31AFB80B7F90630002B02DDBB68F0
:10F3B000002BD4D1FB7D002B0AD0BB68002B07D0DB
:10F3C000FB7F5A1CFA771A46BB6913442D221A7028
:10F3D0000023BB771AE0BB7FBA6913441B78BB7567
:10F3E000FA7FBB7FD31A013BBA691A44BB7FB96964
:10F3F0000B4412781A70FA7FBB7FD31A013BBA69AB
:10F400001344BA7D1A70BB7F0133BB77FB7F5B0867
:10F41000DBB2BA7F9A42DED3FB7FBA691344002283
:10F420001A702037BD4680BDACFE01006766666677
:10F4300080B588B000AFF860B9607A60FB68BB61E6
:10F440000023FB777B68DB0FDBB2FB757B68B3F1D6
:10F45000004F05D1404AB968F8680AF0A8FD78E085
:10F46000BB68013BBB60FB7D002B02D07B685B422D
:10F470007B607B68002B2FD1BB68002B2CD0FB7FDF
:10F480005A1CFA771A46BB69134430221A70BB68BB
:10F49000013BBB6020E07A68304B83FB021399107C
:10F4A000D317C91A0B469B000B445B00D11ACAB292
:10F4B000FB7F591CF9771946BB690B443032D2B235
:10F4C0001A70BB68013BBB607B68244A82FB031255
:10F4D0009210DB17D31A7B607B68002B02DDBB68C0
:10F4E000002BD8D1FB7D002B0AD0BB68002B07D0A6
:10F4F000FB7F5A1CFA771A46BB6913442D221A70F7
:10F500000023BB771AE0BB7FBA6913441B78BB7535
:10F51000FA7FBB7FD31A013BBA691A44BB7FB96932
:10F520000B4412781A70FA7FBB7FD31A013BBA6979
:10F530001344BA7D1A70BB7F0133BB77FB7F5B0836
:10F54000DBB2BA7F9A42DED3FB7FBA691344002252
:10F550001A702037BD4680BDB4FE0100676666663E
:10F5600080B489B000AFF860B9607A60FB68BB61B5
:10F570000023FB77BB68013BBB607B68002B2BD172
:10F58000BB68002B28D0FB7F5A1CFA771A46BB6950
:10F59000134430221A70BB68013BBB601CE07968E1
:10F5A000284BA3FB0123DA0813469B0013445B009E
:10F5B000CA1AD2B2FB7F591CF9771946BB690B44B2
:10F5C0003032D2B21A70BB68013BBB607B681D4A07
:10F5D000A2FB0323DB087B607B68002B02D0BB68A7
:10F5E000002BDCD10023BB771AE0BB7FBA69134440
:10F5F0001B78FB75FA7FBB7FD31A013BBA691A44AB
:10F60000BB7FB9690B4412781A70FA7FBB7FD31A9B
:10F61000013BBA691344FA7D1A70BB7F0133BB7793
:10F62000FB7F5B08DBB2BA7F9A42DED3FB7FBA690D
:10F63000134400221A7000BF2437BD465DF8047BD6
:10F64000704700BFCDCCCCCC80B586B002AFF8609F
:10F65000B9607A607B68002B08DA7B686333C62B5D
:10F6600004D82D22B968F8680AF0F9FC7B68154ABD
:10F6700082FB03125211DB17D31A1A46B968F868D5
:10F680000AF0E2FE2E22B968F8680AF0E8FC7B680E
:10F69000002B02DA7B685B427B607A68094BA3FB34
:10F6A00002135B09642101FB03F3D31A9AB202230C
:10F6B00000933023B968F8680AF0E7FD00BF1037FF
:10F6C000BD4680BD1F85EB5180B485B000AF78602A
:10F6D0007B68FB60084B1B68FA681344FB6000BF43
:10F6E000054B1B68FA689A42FAD800BF00BF14376E
:10F6F000BD465DF8047B7047041000E080B400AFA5
:10F70000094B1B68084A43F080731360074B0022C3
:10F710001A60074B1B68064A43F00103136000BFE1
:10F72000BD465DF8047B7047FCED00E0041000E08E
:10F73000001000E080B485B000AF786053E07B68D3
:10F7400093F85730102B1ED0102B28DC022B02D040
:10F75000082B0CD023E07B681B68DBB203F00103AD
:10F76000FB737B681B685A087B681A602DE07B6816
:10F770001B68DBB203F00703FB737B681B68DA08C6
:10F780007B681A6021E07B681B68DBB203F00F0323
:10F79000FB737B681B681A097B681A6015E07B683D
:10F7A00019681A4BA3FB0123DA0813469B00134484
:10F7B0005B00CA1A1346FB737B681B68134AA2FBE3
:10F7C0000323DA087B681A6000BFFA7B7B689B68BA
:10F7D000581E796888600E498A5C1A707B68DB69FC
:10F7E0005A1C7B68DA617B681B6A591E7A68116251
:10F7F000002BA4DC7B681B68002BA0D100BF00BFDE
:10F800001437BD465DF8047B704700BFCDCCCCCC2F
:10F81000D8FE01002DE9B043A0B002AFF860B96096
:10F820007A603B600023BB63002387F86930CEE336
:10F830007B685A1C7A601B7887F8733097F87330AE
:10F840001F2B03D997F873307A2B02D900237B67DB
:10F8500007E097F87330203BC44AD35C03F00F03F2
:10F860007B677B6FDB0097F869201344BF4AD35C4A
:10F870001B09DBB287F8693097F86930013B062B2A
:10F8800010D801A252F823F0B9F8000069F900007D
:10F89000D5F80000CFFF000001F9000035F90000A5
:10F8A000F1F9000097F87320FB681146B868984793
:10F8B000BB6B0133BB638AE300233B633B6B7B631E
:10F8C0007B6B3B643B6CFB62FB6AFB63202387F82A
:10F8D00068307CE397F873302A2B05D13B681A1DFA
:10F8E0003A601B687B6372E37A6B13469B00134498
:10F8F0005B001A4697F87330303B13447B6366E332
:10F90000FB6B43F00403FB6397F873302A2B05D19C
:10F910003B681A1D3A601B683B6358E33A6B134619
:10F920009B0013445B001A4697F87330303B134436
:10F930003B634CE397F873306C2B0AD07A2B11D1D0
:10F94000FB6B23F00303FB63FB6B43F00203FB63DE
:10F9500009E0FB6B23F00303FB63FB6B43F0010344
:10F96000FB6300E000BF32E397F87330203B102BBD
:10F970003CD801A252F823F0CFF90000EDF90000C5
:10F98000EDF90000D9F90000EDF90000EDF90000F3
:10F99000EDF90000EDF90000EDF90000EDF90000CF
:10F9A000EDF90000E3F90000EDF90000BDF90000F9
:10F9B000EDF90000EDF90000C7F90000FB6B43F022
:10F9C0000803FB6313E0302387F868300FE0FB6B1C
:10F9D00043F01003FB630AE0FB6B43F02003FB637F
:10F9E00005E0FB6B43F04003FB6300E000BFEEE289
:10F9F00097F87330423B362B70D801A252F823F0AF
:10FA0000A1FD0000EFFB0000DDFA0000DDFA0000C0
:10FA1000DDFA0000DDFA0000DDFA0000DDFA00008A
:10FA2000DDFA0000DDFA0000DDFA0000DDFA00007A
:10FA3000DDFA0000DDFA0000E3FA0000DDFA000064
:10FA4000DDFA0000C5FB0000DDFA0000DDFA000071
:10FA5000DDFA0000DDFA000071FB0000DDFA0000B5
:10FA6000DDFA0000DDFA0000DDFA0000DDFA00003A
:10FA7000DDFA0000DDFA0000DDFA0000DDFA00002A
:10FA80001BFB0000F7FB0000A5FB0000DDFA0000F7
:10FA900013FC0000DDFA0000DDFA0000A5FB000009
:10FAA000DDFA0000DDFA0000DDFA0000DDFA0000FA
:10FAB000DDFA000047FB0000EBFA0000DDFA000071
:10FAC000DDFA0000CDFB0000DDFA0000B5FB000010
:10FAD000DDFA0000DDFA000079FB00000023FB6284
:10FAE00075E1FB6B43F08003FB63FB6B23F00303C7
:10FAF000FB63FB6B43F4007343F00203FB631023CF
:10FB000087F8673008233B632D2387F844303E2372
:10FB100087F8453002233B6459E1FB6B43F40073E3
:10FB2000FB63022387F86730FB6B03F02003002B95
:10FB300000F04881302387F84430622387F845304D
:10FB400002233B643EE1FB6B43F40073FB63082339
:10FB500087F86730FB6B03F02003002B00F0348143
:10FB6000302387F8443001233B642DE1ECFE010093
:10FB7000FB6B43F08003FB63FB6B43F40073FB639D
:10FB8000102387F86730FB6B03F02003002B00F095
:10FB90001D81302387F84430782387F845300223CD
:10FBA0003B6413E1FB6B43F44073FB630A2387F868
:10FBB00067300CE1FB6B43F40073FB630A2387F8A7
:10FBC000673004E1FB6B43F08003FB633B681A1D65
:10FBD0003A601B68BB61BB69002B01D19F4BBB61C5
:10FBE000BB6918460AF0A2FE0346FB62EFE0FB6B1E
:10FBF00043F08003FB6307F110033633BB613B68BE
:10FC00001A1D3A601B68DBB287F846300123FB629D
:10FC1000DDE0FB6B03F00403002B01D106233B6303
:10FC20003B68073323F0070303F108023A60D3E986
:10FC30000023C7E908234FF00002894BC7E90423DA
:10FC400000237B670DE0D7E904014FF00002854BEC
:10FC500004F070FD02460B46C7E904237B6F0133B5
:10FC60007B673B6B7A6F9A42EDDBD7E908014FF077
:10FC700000024FF0000304F0A5FE0346002B2DD038
:10FC8000FB6B43F48063FB63D7E90801D7E90423E6
:10FC900004F06EFA02460B46C7E90823D7E90823A9
:10FCA0001046194604F0B6FE0346BB62D7E9088940
:10FCB000BB6A184604F0AAFB02460B46404649467A
:10FCC00004F056FA02460B46C7E90823D7E9082391
:10FCD000144683F00045C7E9084521E0D7E908014B
:10FCE000D7E9042304F046FA02460B46C7E9082385
:10FCF000D7E908231046194604F08CFE0346BB6280
:10FD0000D7E90889BB6A184604F070FB02460B4627
:10FD10004046494604F02CFA02460B46C7E9082340
:10FD200000237B670DE0D7E908014FF000024D4B3F
:10FD300004F0D6FB02460B46C7E908237B6F01336C
:10FD40007B673B6B7A6F9A42EDDBD7E9082310465D
:10FD5000194604F087FE03463B6107F11003363372
:10FD60002033BB610A2387F867303B6B002B0CD034
:10FD700007F110031846FFF7DDFCBB695A1EBA6194
:10FD80002E221A70FB6A0133FB62FB6B43F4D853DB
:10FD900043F00103FB6300233B63BB6A3B6116E056
:10FDA0003B681A1D3A601B68002B02D02E4BBB61CA
:10FDB00001E02E4BBB61BB6918460AF0B7FD034654
:10FDC000FB6204E000BF02E000BF00E000BFFB6B8D
:10FDD00003F40073002B00F0AB803B6B002B01D1D0
:10FDE00001233B63FB6B03F40063002B33D1FB6BFC
:10FDF00003F00303022B06D0022B39D8002B19D0B5
:10FE0000012B06D034E03B681A1D3A601B683B6149
:10FE10002FE0FB6B03F48073002B05D03B681A1DA9
:10FE20003A601B683B6124E03B681A1D3A601B681E
:10FE30003B611EE0FB6B03F48073002B05D03B6835
:10FE40001A1D3A601B683B6113E03B681A1D3A605B
:10FE50001B683B610DE000BF0BE000BFC0FE01006E
:10FE60000000E03F00002440C8FE0100D0FE010079
:10FE700000BFFB6B03F02003002B04D03B69002B79
:10FE800001D100233B64FB6B03F48073002B18D07B
:10FE90003B69002B06DA3B695B423B61FB6B43F439
:10FEA0008063FB63FB6B03F48063002B09D1FB6B66
:10FEB00003F01003002B04D0202387F844300123E3
:10FEC0003B64FB6B03F48053002B04D107F1100358
:10FED00036332033BB6107F110031846FFF72AFCC5
:10FEE000BB690133BB61FB6B03F48863002B28D033
:10FEF000FB6B03F48063002B01D02D2300E02B2348
:10FF000087F8733097F86830302B06D101233B64B3
:10FF100097F8733087F8443013E0BB69013BBB614D
:10FF2000BB6997F873201A70FB6A0133FB6208E023
:10FF30007B6B002B05D0FA6A7B6B9A4201DD7B6BF1
:10FF4000FB627A6BF96A3B6C0B44D31A7B63396CA6
:10FF5000FB6B03F0800307F11002343200930B4671
:10FF6000B968F8680AF0F9FC0246BB6B1344BB633E
:10FF7000FB6B03F00803002B0AD197F868207B6B1A
:10FF8000B968F8680AF01AFD0246BB6B1344BB63FC
:10FF9000BA69F96AFB6B03F0800300930B46B968FA
:10FFA000F8680AF0DAFC0246BB6B1344BB63FB6BD8
:10FFB00003F00803002B0AD097F868207B6BB96820
:10FFC000F8680AF0FBFC0246BB6B1344BB637B681A
:10FFD0001B78002B7FF42CACBB6B18467837BD46E2
:10FFE000BDE8B08380B582B000AFFB1C012219468A
:10FFF000012001F0B7FA03467B607B68002B4CDDE3
:020000021000EC
:10000000FB78072B16DC002B3CDD013B062B39D897
:1000100001A252F823F000BF3B00010041000100A3
:10002000470001004D00010053000100590001008C
:100030005F000100802B15D024E000F085FB31E04B
:1000400000F03AFC2EE000F015FE2BE000F0DAFDA7
:1000500028E000F057FC25E001F0B0F822E001F0C4
:100060008FF81FE0FB1C01221946012001F07AFAEB
:1000700003467B607B68002B11DDFB78184600F09F
:10008000FFFF0CE0FB785BB2002B0ADAFB1C0122BD
:100090001946012001F066FA03E000BF02E000BF4C
:1000A00000E000BF00BF0837BD4680BD80B58CB002
:1000B00000AF01233B713B1D0133FB61FB69FB6218
:1000C000304B5B69BB620BE0BB6ADAB2FB6A591C5E
:1000D000F96262F07F02D2B21A70BB6ADB09BB62BE
:1000E000BB6A7F2BF0D8FB6A5A1CFA62BA6AD2B29A
:1000F0001A70FB6AFB61244B1B681B09BB61214B17
:10010000DB68BA69D31A7B61FB697B627B693B62FE
:100110000BE03B6ADAB27B6A591C796262F07F02BB
:10012000D2B21A703B6ADB093B623B6A7F2BF0D884
:100130007B6A5A1C7A623A6AD2B21A707B6AFB6195
:100140003B1DFA69D31A1A463B1D1946012001F0DE
:100150008FFA03463B613B69002B09D0094ABB6912
:10016000D360084B1B78013BDAB2064B1A7004E0EF
:10017000044B5B690133034A53613B6918463037CE
:10018000BD4680BD50210020041000E080B58AB03B
:1001900000AFF860B9607A60634B1B78012B10D018
:1001A000614B1B78002B00F0A2805F4B1B78022B69
:1001B00009D1FFF77BFF5C4B1B78012B40F0998046
:1001C00001E000BF00E000BF7B681F2B09D8564B41
:1001D000DA697B6822FA03F303F00103002B40F095
:1001E0008A807B68172B07D8FB68013BFB607B6824
:1001F000DAB2FB681A703DE0BA68FB68D31AFB619B
:10020000FB697F2B12D9FB69DA09FB68013BFB60B4
:10021000D2B2FB681A70FB69DBB2FA68013AFA6085
:1002200063F07F03DAB2FB681A7006E0FB68013BFB
:10023000FB60FB69DAB2FB681A707B687F2B12D90E
:100240007B68DA09FB68013BFB60D2B2FB681A707D
:100250007B68DBB2FA68013AFA6063F07F03DAB2D6
:10026000FB681A7006E0FB68013BFB607B68DAB252
:10027000FB681A702D4B1B681B09BB612A4BDB689E
:10028000BA69D31A7B61BB687B627B693B620BE016
:100290003B6ADAB27B6A591C796262F07F02D2B2A1
:1002A0001A703B6ADB093B623B6A7F2BF0D87B6AA2
:1002B0005A1C7A623A6AD2B21A707B6ABB60BA6818
:1002C000FB68D31A1A46F968012001F0D1F90346F8
:1002D0003B613B69002B03D0134ABB69D3600BE041
:1002E000114B1B780133DAB20F4B1A7004E000BFD8
:1002F00002E000BF00E000BF0D4BD3F884200C4BA0
:10030000D3F888309A420BD0074B9B78002B07D14B
:10031000054B01229A70FFF765FE034B00229A708D
:1003200000BF2837BD4680BD50210020041000E0EA
:100330002C23002080B586B002AFF860B9607A60E7
:100340003B60002300934FF48063144A144901205A
:1003500001F0A0FA002300930823124A104901205B
:1003600001F008FB104B4FF080521A610F4B1B68D5
:100370001B090D4AD3600C4A7B6813620A4AFB686A
:100380005360094ABB689360074A3B685362064B57
:1003900000221A7000BF1037BD4680BD481D0020E6
:1003A00054FF01004821002050210020041000E0EB
:1003B00080B483B000AF7860044A7B68136100BFEB
:1003C0000C37BD465DF8047B704700BF502100200C
:1003D00080B584B000AF7860EFF311834FF0500127
:1003E00081F31188FB6008480AF058FBB8607A680E
:1003F000B968B868FFF7CAFEFB6883F3118800BFCD
:100400001037BD4680BD00BF7C21002080B588B07C
:1004100000AF78603960EFF311834FF0500181F342
:1004200011887B6116480AF039FB38613B69FB6033
:10043000FB68FB613B68BB610BE0BB69DAB2FB693F
:10044000591CF96162F07F02D2B21A70BB69DB09F4
:10045000BB61BB697F2BF0D8FB695A1CFA61BA6992
:10046000D2B21A70FB69FB607A68F9683869FFF7E5
:100470008DFE7B6983F3118800BF2037BD4680BDA8
:100480007C21002080B58CB000AFF860B9607A6044
:10049000EFF311834FF0500181F31188FB61254880
:1004A0000AF0FCFAB861BB697B617B69FB62BB68DF
:1004B000BB620BE0BB6ADAB2FB6A591CF96262F0FC
:1004C0007F02D2B21A70BB6ADB09BB62BB6A7F2BA8
:1004D000F0D8FB6A5A1CFA62BA6AD2B21A70FB6A86
:1004E0007B617B697B627B683B620BE03B6ADAB2D3
:1004F0007B6A591C796262F07F02D2B21A703B6A41
:10050000DB093B623B6A7F2BF0D87B6A5A1C7A621C
:100510003A6AD2B21A707B6A7B61FA687969B86903
:10052000FFF734FEFB6983F3118800BF3037BD4607
:1005300080BD00BF7C21002080B58EB000AFF86088
:10054000B9607A603B60EFF311834FF0500181F3A3
:100550001188FB6132480AF0A1FAB861BB697B617E
:100560007B697B63BB683B630BE03B6BDAB27B6B05
:10057000591C796362F07F02D2B21A703B6BDB09BF
:100580003B633B6B7F2BF0D87B6B5A1C7A633A6BD7
:10059000D2B21A707B6B7B617B69FB627B68BB624A
:1005A0000BE0BB6ADAB2FB6A591CF96262F07F02A7
:1005B000D2B21A70BB6ADB09BB62BB6A7F2BF0D870
:1005C000FB6A5A1CFA62BA6AD2B21A70FB6A7B6181
:1005D0007B697B623B683B620BE03B6ADAB27B6A19
:1005E000591C796262F07F02D2B21A703B6ADB0951
:1005F0003B623B6A7F2BF0D87B6A5A1C7A623A6A6C
:10060000D2B21A707B6A7B61FA687969B869FFF7C0
:10061000BDFDFB6983F3118800BF3837BD4680BD3F
:100620007C21002080B590B000AFF860B9607A609E
:100630003B60EFF311834FF0500181F31188FB61B0
:1006400040480AF02BFAB861BB697B617B69FB63A8
:10065000BB68BB630BE0BB6BDAB2FB6B591CF96385
:1006600062F07F02D2B21A70BB6BDB09BB63BB6B5B
:100670007F2BF0D8FB6B5A1CFA63BA6BD2B21A709C
:10068000FB6B7B617B697B637B683B630BE03B6B54
:10069000DAB27B6B591C796362F07F02D2B21A70B6
:1006A0003B6BDB093B633B6B7F2BF0D87B6B5A1CAE
:1006B0007A633A6BD2B21A707B6B7B617B69FB62A7
:1006C0003B68BB620BE0BB6ADAB2FB6A591CF96299
:1006D00062F07F02D2B21A70BB6ADB09BB62BB6AEE
:1006E0007F2BF0D8FB6A5A1CFA62BA6AD2B21A702F
:1006F000FB6A7B617B697B62BB6C3B620BE03B6AA4
:10070000DAB27B6A591C796262F07F02D2B21A7047
:100710003B6ADB093B623B6A7F2BF0D87B6A5A1C41
:100720007A623A6AD2B21A707B6A7B61FA68796936
:10073000B869FFF72BFDFB6983F3118800BF4037D1
:10074000BD4680BD7C21002080B58CB000AF574BEA
:1007500001221A70EFF311834FF0500181F31188D9
:10076000FB600A225249012000F082FFFB6883F3FC
:1007700011880A20FFF72CFEEFF311834FF0500190
:1007800081F31188BB604B480AF088F978607B6878
:100790003B603B68FB62454B5B68BB620BE0BB6A3E
:1007A000DAB2FB6A591CF96262F07F02D2B21A70A7
:1007B000BB6ADB09BB62BB6A7F2BF0D8FB6A5A1CA1
:1007C000FA62BA6AD2B21A70FB6A3B603B687B621B
:1007D000364B9B683B620BE03B6ADAB27B6A591C82
:1007E000796262F07F02D2B21A703B6ADB093B6227
:1007F0003B6A7F2BF0D87B6A5A1C7A623A6AD2B283
:100800001A707B6A3B603B68FB61284B1B69BB61CC
:100810000BE0BB69DAB2FB69591CF96162F07F0237
:10082000D2B21A70BB69DB09BB61BB697F2BF0D800
:10083000FB695A1CFA61BA69D2B21A70FB693B6053
:100840003B687B6102233B610BE03B69DAB27B6969
:10085000591C796162F07F02D2B21A703B69DB09E0
:100860003B613B697F2BF0D87B695A1C7A613A69FE
:10087000D2B21A707B693B60182239687868FFF73A
:1008800085FCBB6883F31188084B5B6A002B02D0A0
:10089000064B5B6A984700F0EDF900F0B3F900F001
:1008A0008DFC00BF3037BD4680BD00BF5021002009
:1008B00048FF01007C21002080B582B000AFEFF33B
:1008C00011834FF0500181F311887B600B480AF0CF
:1008D000E5F838600A4B1B78002B07D00B223968EB
:1008E0003868FFF753FC064B00221A707B6883F3CD
:1008F000118800BF0837BD4680BD00BF7C210020A5
:100900005021002080B58CB000AFEFF311834FF081
:10091000500181F31188FB6045480AF0BFF8B860C8
:10092000BB687B607B68FB62424B5B68BB620BE031
:10093000BB6ADAB2FB6A591CF96262F07F02D2B27A
:100940001A70BB6ADB09BB62BB6A7F2BF0D8FB6AFB
:100950005A1CFA62BA6AD2B21A70FB6A7B607B6870
:100960007B62344B9B683B620BE03B6ADAB27B6A8A
:10097000591C796262F07F02D2B21A703B6ADB09BD
:100980003B623B6A7F2BF0D87B6A5A1C7A623A6AD8
:10099000D2B21A707B6A7B607B68FB61254B1B6956
:1009A000BB610BE0BB69DAB2FB69591CF96162F00B
:1009B0007F02D2B21A70BB69DB09BB61BB697F2BB6
:1009C000F0D8FB695A1CFA61BA69D2B21A70FB6995
:1009D0007B607B687B6102233B610BE03B69DAB2A1
:1009E0007B69591C796162F07F02D2B21A703B694F
:1009F000DB093B613B697F2BF0D87B695A1C7A612C
:100A00003A69D2B21A707B697B6018227968B8683B
:100A1000FFF7BCFBFB6883F31188064B5B6A002B76
:100A200002D0044B5B6A984700BF3037BD4680BD9B
:100A30007C2100205021002080B592B000AF78606A
:100A4000EFF311834FF0500181F311887B616B4804
:100A50000AF024F838613B69FB60FB687B647B68C3
:100A60001A68674B1B69D31A9B083B640BE03B6C0D
:100A7000DAB27B6C591C796462F07F02D2B21A70D0
:100A80003B6CDB093B643B6C7F2BF0D87B6C5A1CC6
:100A90007A643A6CD2B21A707B6CFB60FB68FB63C1
:100AA0007B689B68BB630BE0BB6BDAB2FB6B591CCA
:100AB000F96362F07F02D2B21A70BB6BDB09BB63D1
:100AC000BB6B7F2BF0D8FB6B5A1CFA63BA6BD2B2AC
:100AD0001A70FB6BFB607B685B6820221946F86824
:100AE00009F08FFFF8600922F9683869FFF74EFBBB
:100AF0003B69FB60FB687B637B681A68404B1B6942
:100B0000D31A9B083B630BE03B6BDAB27B6B591C3F
:100B1000796362F07F02D2B21A703B6BDB093B63F0
:100B20003B6B7F2BF0D87B6B5A1C7A633A6BD2B24B
:100B30001A707B6BFB60FB68FB627B68DB68BB62E7
:100B40000BE0BB6ADAB2FB6A591CF96262F07F0201
:100B5000D2B21A70BB6ADB09BB62BB6A7F2BF0D8CA
:100B6000FB6A5A1CFA62BA6AD2B21A70FB6AFB605C
:100B7000FB687B627B681B693B620BE03B6ADAB215
:100B80007B6A591C796262F07F02D2B21A703B6AAA
:100B9000DB093B623B6A7F2BF0D87B6A5A1C7A6286
:100BA0003A6AD2B21A707B6AFB60FB68FB61002371
:100BB000BB610BE0BB69DAB2FB69591CF96162F0F9
:100BC0007F02D2B21A70BB69DB09BB61BB697F2BA4
:100BD000F0D8FB695A1CFA61BA69D2B21A70FB6983
:100BE000FB601522F9683869FFF7D0FA7B6983F357
:100BF000118800BF4837BD4680BD00BF7C21002062
:100C00005021002080B500AF074B1B6A002B08D095
:100C1000054B1B6A5B68002B03D0034B1B6A5B68A8
:100C2000984700BF80BD00BF5021002080B586B02E
:100C300000AF7860EFF311834FF0500181F311881A
:100C40007B610B4809F02AFF386180227968386996
:100C500009F0D7FEF8600E22F9683869FFF796FAB6
:100C60007B6983F3118800BF1837BD4680BD00BF84
:100C70007C21002090B583B000AF154B1B6A002B80
:100C80001AD0134B1B6A1B68002B15D0104B1B6A24
:100C90001B689847C7E900013C68D7E900014FF09D
:100CA00000024FF000030A00002313461A462146B3
:100CB0000D20FFF7E7FB07E0064B1B681B091946F1
:100CC0000C20FFF7A3FB00BF00BF0C37BD4690BD53
:100CD00050210020041000E080B586B000AFEFF393
:100CE00011834FF0500181F31188FB60194809F01E
:100CF000D5FEB860BB687B60174B1B68C3F3080365
:100D00003B607B687B613B683B610BE03B69DAB22F
:100D10007B69591C796162F07F02D2B21A703B691B
:100D2000DB093B613B697F2BF0D87B695A1C7A61F8
:100D30003A69D2B21A707B697B6002227968B8681E
:100D4000FFF724FAFB6883F3118800BF1837BD460C
:100D500080BD00BF7C21002004ED00E080B582B0A2
:100D600000AFEFF311834FF0500181F311887B60E6
:100D7000074809F093FE3860032239683868FFF7A6
:100D800005FA7B6883F3118800BF0837BD4680BD34
:100D90007C21002080B582B000AFEFF311834FF0CB
:100DA000500181F311887B60074809F077FE3860B5
:100DB000122239683868FFF7E9F97B6883F31188F4
:100DC00000BF0837BD4680BD7C21002080B582B0C1
:100DD00000AFEFF311834FF0500181F311887B6076
:100DE000074809F05BFE3860112239683868FFF760
:100DF000CDF97B6883F3118800BF0837BD4680BDFD
:100E00007C21002080B588B000AF7860EFF31183BB
:100E10004FF0500181F311887B611A4809F03EFEC2
:100E200038613B69FB60184B1B697A68D31A9B08D1
:100E30007B60FB68FB617B68BB610BE0BB69DAB27E
:100E4000FB69591CF96162F07F02D2B21A70BB696A
:100E5000DB09BB61BB697F2BF0D8FB695A1CFA61C7
:100E6000BA69D2B21A70FB69FB600822F968386966
:100E7000FFF78CF97B6983F3118800BF2037BD46EB
:100E800080BD00BF7C2100205021002080B588B0AB
:100E900000AF7860EFF311834FF0500181F31188B8
:100EA0007B611A4809F0FAFD38613B69FB60184B19
:100EB0001B697A68D31A9B087B60FB68FB617B68BF
:100EC000BB610BE0BB69DAB2FB69591CF96162F0E6
:100ED0007F02D2B21A70BB69DB09BB61BB697F2B91
:100EE000F0D8FB695A1CFA61BA69D2B21A70FB6970
:100EF000FB600422F9683869FFF748F97B6983F3DE
:100F0000118800BF2037BD4680BD00BF7C21002076
:100F10005021002080B588B000AF7860EFF31183D6
:100F20004FF0500181F311887B611A4809F0B6FD3A
:100F300038613B69FB60184B1B697A68D31A9B08C0
:100F40007B60FB68FB617B68BB610BE0BB69DAB26D
:100F5000FB69591CF96162F07F02D2B21A70BB6959
:100F6000DB09BB61BB697F2BF0D8FB695A1CFA61B6
:100F7000BA69D2B21A70FB69FB600622F968386957
:100F8000FFF704F97B6983F3118800BF2037BD4662
:100F900080BD00BF7C2100205021002080B58AB098
:100FA00000AF78603960EFF311834FF0500181F3A7
:100FB00011887B61274809F071FD38613B69FB604E
:100FC000254B1B697A68D31A9B087B60FB687B62A0
:100FD0007B683B620BE03B6ADAB27B6A591C796240
:100FE00062F07F02D2B21A703B6ADB093B623B6A55
:100FF0007F2BF0D87B6A5A1C7A623A6AD2B21A7096
:101000007B6AFB60FB68FB613B68BB610BE0BB6913
:10101000DAB2FB69591CF96162F07F02D2B21A7030
:10102000BB69DB09BB61BB697F2BF0D8FB695A1C2C
:10103000FA61BA69D2B21A70FB69FB600722F968DB
:101040003869FFF7A3F87B6983F3118800BF28375D
:10105000BD4680BD7C2100205021002080B483B09B
:1010600000AF7860054B1B697A68D31A9B08184655
:101070000C37BD465DF8047B704700BF502100204F
:1010800080B58CB000AF0346FB713B4B1B68002B57
:101090006DD0394B1B68FB620023BB6208E0FB6A22
:1010A0001B69FB62FB6A002B07D0BB6A0133BB6282
:1010B000FB79BA6A9A42F2D300E000BFFB6A002BC8
:1010C00055D0EFF311834FF0500181F311887B610C
:1010D0002A4809F0E3FC38613B69FB60FB687B62EE
:1010E000FB793B620BE03B6ADAB27B6A591C79629E
:1010F00062F07F02D2B21A703B6ADB093B623B6A44
:101100007F2BF0D87B6A5A1C7A623A6AD2B21A7084
:101110007B6AFB60FB68FB61FB6A9B68BB610BE061
:10112000BB69DAB2FB69591CF96162F07F02D2B285
:101130001A70BB69DB09BB61BB697F2BF0D8FB6907
:101140005A1CFA61BA69D2B21A70FB69FB60FB6A79
:101150001B6880221946F86809F053FCF8601622D3
:10116000F9683869FFF712F87B6983F3118800BFCB
:101170003037BD4680BD00BF782100207C21002093
:1011800080B582B000AF0C4B1B68002B0FD00A4B10
:101190001B687B607B68DB68002B02D07B68DB68A8
:1011A00098477B681B697B607B68002BF2D100BF8E
:1011B0000837BD4680BD00BF7821002080B586B0CD
:1011C00000AFEFF311834FF0500181F31188FB6002
:1011D000174809F063FCB860BB687B607B687B6183
:1011E000144B1B783B610BE03B69DAB27B69591CFD
:1011F000796162F07F02D2B21A703B69DB093B6110
:101200003B697F2BF0D87B695A1C7A613A69D2B26C
:101210001A707B697B601B227968B868FEF7B6FF9D
:10122000FB6883F3118800BF1837BD4680BD00BF3F
:101230007C210020E635002080B58AB000AF7860C0
:10124000EFF311834FF0500181F311887B61274840
:1012500009F024FC386180227968386909F0D1FBF3
:10126000F860FB687B6201233B620BE03B6ADAB209
:101270007B6A591C796262F07F02D2B21A703B6AB3
:10128000DB093B623B6A7F2BF0D87B6A5A1C7A628F
:101290003A6AD2B21A707B6AFB60FB68FB6100237A
:1012A000BB610BE0BB69DAB2FB69591CF96162F002
:1012B0007F02D2B21A70BB69DB09BB61BB697F2BAD
:1012C000F0D8FB695A1CFA61BA69D2B21A70FB698C
:1012D000FB601A22F9683869FEF758FF7B6983F3CF
:1012E000118800BF2837BD4680BD00BF7C2100208B
:1012F00080B500AF0348FFF799FC0348FFF796FC61
:1013000000BF80BD5CFF010084FF010080B500AF1D
:10131000074B1B681809064B1968064B064AFFF76E
:1013200009F84FF00050FFF743F800BF80BD00BF41
:10133000E0010020F1120100E4FF0100F0B585B0EA
:1013400002AF00237B6048E029497A6813469B007E
:1013500013449B000B441B68184602F00BF801462F
:1013600023487A6813469B0013449B0003441033C0
:1013700019601F497A6813469B0013449B000B4475
:1013800018681B497A6813469B0013449B000B4462
:1013900004331968164C7A6813469B0013449B006B
:1013A000234408331C68124D7A6813469B0013448B
:1013B0009B002B440C331D680D4E7A6813469B002E
:1013C00013449B00334410331B6800932B46224682
:1013D00009F0B3FB7B6801337B60064B1B687A68BE
:1013E0009A42B1D300BF00BF0C37BD46F0BD00BF6D
:1013F000602200202823002080B586B002AFF8606C
:10140000B9607A603B6005222B49B8680AF03AFF60
:101410000346002B4BD0294B1B68092B03D92848C6
:10142000FFF70AFF44E0254B1A68264913469B0044
:1014300013449B000B44FA681A60204B1A68214938
:1014400013469B0013449B000B440433BA681A6094
:101450001A4B1A681B4913469B0013449B000B440C
:1014600008337A681A60154B1A68164913469B00B0
:1014700013449B000B440C333A681A600F4B1A68F4
:10148000104913469B0013449B000B441033BA6968
:101490001A600A4B1B680133084A1360BB6900934A
:1014A0003B687A68B968F86809F047FB00E000BF5C
:1014B0001037BD4680BD00BFE0CE010028230020CC
:1014C00094FF01006022002080B582B000AF1F4B66
:1014D0007B607B6803221A617B6803225A617B6808
:1014E0001B4A9A617B681B4ADA617B684FF4805221
:1014F0001A627B6800229A627B6800225A627B68CB
:101500000022DA627B68124A1A667B68124A5A66BF
:101510007B6840229A667B6800221A677B680022FB
:10152000DA667B6800225A677B6807330B491846E6
:101530000AF0B1FF7B680A4918460AF0ACFF7B68E5
:1015400020229A7100BF0837BD4680BD2C230020A1
:10155000ECFF0100D4230020D4330020F8FF010069
:10156000FCFF010080B58CB000AFF860B9607A6014
:101570003E4B3B623B6A1B78DBB2002B01D1FFF78D
:10158000A3FFFA6813465B001344DB006033374A5D
:101590001344FB61BB687B62FB691B69BB62FB692F
:1015A000DB68BB610023FB62BA6ABB699A422BD934
:1015B000FB699A68BB6AD31A7B617A697B6893423C
:1015C00028BF13467B61FB695A68BB6A13443B61C1
:1015D0007A693969786A0AF065FEFA6A7B691344A8
:1015E000FB627A6A7B6913447B627A687B69D31AEF
:1015F0007B60BA6A7B691344BB62FB699B68BA6A09
:101600009A4201D10023BB62BA69BB6AD31A7B61DB
:101610007A697B68934228BF13467B617B69002B04
:1016200019D0FB695A68BB6A13443B617A6939690E
:10163000786A0AF037FEFA6A7B691344FB627A6AB9
:101640007B6913447B627A687B69D31A7B60BA6AD0
:101650007B691344BB62FB6A002B02D0FB69BA6A48
:101660001A61FB6A18463037BD4680BD2C23002026
:1016700080B58CB000AFF860B9607A60BB68FB627F
:10168000FB685A1C13465B001344DB00334A1344C7
:10169000BB62BB6A1B697B62BB6ADB683B627A6ABE
:1016A0003B6A9A424BD8BB6A9A683B6AD31A013BA1
:1016B000FB61FA697B689A4213D300BF00E000BF68
:1016C000BB6A5A683B6A13447B617A68F96A786935
:1016D0000AF0E8FD3A6A7B681A44BB6ADA600123C3
:1016E00037E0FA697B6A1344FB61FA697B689A42C6
:1016F0002ED3BB6A9A683B6AD31ABB61BB6A5A682D
:101700003B6A13447B61BA69F96A78690AF0CAFDD9
:101710007A68BB69D31A7B607B68002B0AD0BB6AEE
:101720005B687B61FA6ABB6913447A681946786919
:101730000AF0B8FDBB6A7A68DA60012309E07A6AC8
:101740003B6AD31A013BFB61FA697B689A42B6D2C5
:10175000002318463037BD4680BD00BF2C23002033
:1017600080B588B000AFF860B9607A60BB68BB61D3
:10177000FB685A1C13465B001344DB001F4A1344EA
:101780007B617B695B69022B29D0022B2ED8002B51
:1017900002D0012B13D029E0786909F08EFA386164
:1017A0003A697B689A4202D20023FB6121E07B68A0
:1017B000FB617A68B969786909F03BFA19E07869E0
:1017C00009F07BFA38617A683B69934228BF134677
:1017D000FB61FA69B969786909F02BFA09E07A685E
:1017E000B969786909F0CAF9F86102E00023FB6180
:1017F00000BFFB6918462037BD4680BD2C23002062
:1018000080B588B000AFF860B9607A600E4BFB61BC
:10181000FB691B78DBB2002B01D1FFF755FEEFF31C
:1018200011834FF0500181F31188BB617A68B96868
:10183000F868FFF795FF7861BB6983F311887B69CE
:1018400018462037BD4680BD2C23002080B584B0CB
:1018500000AF0E4BBB60BB681B78DBB2002B01D125
:10186000FFF732FE0A4B7B607B681B693B607B683D
:10187000DB683A689A4202D00123FB6001E0002352
:10188000FB60FB6818461037BD4680BD2C23002046
:101890008C23002080B588B000AFF860B9607A6012
:1018A0003B60334BBB61BB691B78DBB2002B01D1C2
:1018B000FFF70AFE2E4B7B617B691B691A46FB68AA
:1018C00093424CD2EFF311834FF0500181F3118812
:1018D0003B61FB68002B32D07969FB685A1C1346C8
:1018E0005B001344DB000B44BA681A607969FB683B
:1018F0005A1C13465B001344DB000B4404337A6824
:101900001A607969FA6813465B001344DB000B44E4
:1019100020333A681A607969FA6813465B00134409
:10192000DB000B44283300221A607969FA681346F9
:101930005B001344DB000B44243300221A607969F6
:10194000FA6813465B001344DB000B442C33BA6A7D
:101950001A603B6983F311880023FB6102E04FF0BA
:10196000FF33FB61FB6918462037BD4680BD00BFD1
:101970002C23002080B588B000AFF860B9607A6091
:101980003B60324BBB61BB691B78DBB2002B01D1E2
:10199000FFF79AFD2D4B7B617B695B691A46FB68FB
:1019A00093424BD2EFF311834FF0500181F3118832
:1019B0003B61FB68002B31D07969FA6813465B0004
:1019C0001344DB000B446033BA681A607969FA6823
:1019D00013465B001344DB000B4464337A681A60DF
:1019E0007969FA6813465B001344DB000B446833E3
:1019F0003A681A607969FA6813465B001344DB00A1
:101A00000B44703300221A607969FA6813465B0050
:101A10001344DB000B446C3300221A607969FA68C6
:101A200013465B001344DB000B447433BA6A1A603C
:101A30003B6983F311880023FB6102E04FF0FF3321
:101A4000FB61FB6918462037BD4680BD2C23002072
:101A500080B58AB000AFF860B9607A603B60BB685F
:101A60003B6201237B620123FB6107E03A6A7B68EA
:101A7000B2FBF3F33B62FB690133FB613A6A7B68BB
:101A80009A42F3D23A68FB699A4201D93B68FB61FA
:101A90007B6B03F00103002B25D13B6B002B22D085
:101AA0007B6B03F00203002B05D03B68002B02D1B7
:101AB0003023FB7601E02023FB760BE03B6B013B00
:101AC0003B63FB7E1946F86809F054F9FB68DB6854
:101AD000002B07DB3B6B002B05D0FA693B6B9A426E
:101AE000ECD300E000BFFB68DB68002B55DB3B68F4
:101AF000012B03D93B68013B3B6009E0BA687B6A74
:101B0000B2FBF3F37B617A697B689A4200D205E00D
:101B10007B6A7A6802FB03F37B62E8E7BA687B6A58
:101B2000B2FBF3F37B617B697A6A02FB03F3BA6869
:101B3000D31ABB601B4A7B6913441B781946F868AB
:101B400009F018F9FB68DB68002B08DB7A6A7B6810
:101B5000B2FBF3F37B627B6A002BDFD100E000BFB6
:101B60007B6B03F00103002B17D03B6B002B14D0D1
:101B70000AE03B6B013B3B632021F86809F0FAF86F
:101B8000FB68DB68002B07DB3B6B002B05D0FA6999
:101B90003B6B9A42EDD300E000BF00BF2837BD4643
:101BA00080BD00BF0400020080B5A2B002AFF860A3
:101BB000B9607A6007F110033B6540237B65002321
:101BC000BB65FB683B660023FB65BB681B7887F839
:101BD0007F30BB680133BB6097F87F30002B00F08B
:101BE0009F8197F87F30252B40F08D8100233B6744
:101BF0000123BB67BB681B7887F87F3097F87F307D
:101C0000233B0D2B3ED801A252F823F0751C010096
